:020000040800F2
:10000000F87F00108501000895010008950100089F
:100010009501000895010008950100080000000006
:100020000000000000000000000000009501000832
:100030009501000800000000950100081129000842
:100040009501000895010008950100089501000838
:100050009501000895010008950100089501000828
:100060009501000895010008950100089501000818
:100070009501000895010008950100089501000808
:1000800095010008950100089501000895010008F8
:1000900095010008950100089501000895010008E8
:1000A00095010008950100089501000895010008D8
:1000B00095010008950100089501000895010008C8
:1000C00095010008950100089501000895010008B8
:1000D00095010008950100089501000895010008A8
:1000E0009501000895010008950100089501000898
:1000F0009501000895010008950100089501000888
:100100009501000895010008950100089501000877
:100110009501000895010008950100089501000867
:100120009501000895010008950100089501000857
:100130009501000895010008950100089501000847
:100140009501000895010008950100089501000837
:100150009501000895010008950100089501000827
:100160009501000895010008950100089501000817
:100170009501000895010008950100089501000807
:1001800095010008DFF808D000F020F800F0A6B9CB
:10019000F87F0010FEE70000814230B515D002F074
:1001A0000304034622F00302D51AE84204D053F8B0
:1001B000045B41F8045BF7E701391A19934204D054
:1001C00013F8010B01F8010FF8E730BD284BD3F805
:1001D000882042F47002C3F888205A6922F402721F
:1001E0005A61244B1A6842F001021A601A6890079B
:1001F000FCD500229A601A6822F0A0621A601A6880
:1002000042F480321A601B4A13689903FCD51A4BDA
:100210001B68DBB2112B194B0CBF40F2056240F298
:1002200005721A60134B164A5A601A6842F08072BF
:100230001A601A689201FCD549F202429A604FF4A2
:1002400080121A6300225A639A634FF080521A6434
:100250004FF480425A641A6822F001021A60094A77
:10026000012111601A6B42F07F021A63704700BFD0
:1002700000ED00E000380240002004E0003C0240B5
:100280000C5A410F00380140012910B513D80C4811
:100290000C4B53F8213050F82110012010701944F4
:1002A0004FF6FF70994208D933F8024B8442F9D0D7
:1002B0000020107010BD092010BD002010BD00BF2F
:1002C0007C0D0308840D0308012926D8144B53F82C
:1002D000212002F17842930B032B88BF530C114A63
:1002E000116988BF04330029BCBF0F4951604FEA30
:1002F000C303BCBF01F18831516043F0020143F4F4
:10030000803343F00203116113611361054BDA6816
:10031000D203FCD44FF000421A610920704700BF9D
:10032000840D0308003C02402301674573B516465F
:1003300000220C4601921D466BB101AA084B98475A
:1003400060B921462644023D8E4205D931F8023B70
:1003500025F8023FF8E7022002B070BD0920FBE754
:10036000F909000873B5164600220D4601921C4695
:10037000002B2CD001AA184B984750BB174B1A6979
:10038000002ABFBF164A5A6002F188325A602E44D2
:1003900040F201122946114D1A6123468E4210D9AE
:1003A00031F8022B1C88A24201D10233F6E721F872
:1003B000024CEA68D203FCD41A88A242F5D0082085
:1003C00003E0064B4FF000421A6102B070BD0220FC
:1003D000FBE70920F9E700BFF9090008003C0240EB
:1003E0002301674570B52B4D86680446A847014632
:1003F0002046B047266AA8474FF080414268264D04
:100400002046B047254B9847A668A8470146204696
:10041000B047266AA84722494268224D2046B04785
:10042000214B9847A668A84701462046B047266A50
:10043000A8471E4942682046B0471D4B98471D4BB0
:10044000A568984701462046A8471B4B98471B4B79
:10045000A568984701462046A847194B9847194B6D
:10046000A568984701462046A847174B9847174B61
:10047000A568984701462046A847154B9847154B55
:10048000A568984701462046A847134BBDE8704031
:10049000184700BF69060008CD080008D907000802
:1004A00002000040610C00084109000804000040FF
:1004B00071100008F1110008A9150008B91B000807
:1004C000111F000875200008D9250008C92D000853
:1004D0005D320008653C0008ED430008F0B52F4B85
:1004E0002F4D304C85B0984702A901A82E4B984754
:1004F000029901982D4B98474FF4A06200232C4994
:100500002C48A047A84784693021A3682046984713
:10051000236A022230212046984703AA236930210A
:1005200020469847E368302120469847039B224C99
:10053000012B0CBF214B224B98470021A047214B98
:100540009847214B04469847204B06469847204B36
:10055000074698473A460346314620461D4CA04779
:10056000A84784693121A36820469847236A02225C
:1005700031212046984703AA236931212046984714
:10058000E368312120469847039913484B1E59428E
:100590005941124B9847002005B0F0BD09260008CC
:1005A000610C0008B94C0008F5250008C16100087D
:1005B000820C03088E0C0308E9610008653C000802
:1005C000C92D0008850900086116000829180008CF
:1005D000992700080D600008E5030008556A000827
:1005E00010B51448415C0023C45C8C421CD1124BF2
:1005F000D86C5963103901299FBF104C606840F4D2
:1006000000006060986840F080409860186880073B
:10061000FCD501299FBF0948416821F400014160D0
:10062000DB6C1360002010BD0133102BDCD10320E4
:1006300010BD00BFF60C030800200140002301405C
:10064000102070470C2070470020704740F6FF7064
:10065000704700207047002914BF04200020704715
:10066000B1FA81F040097047144B1548002230B5AB
:100670005A60144A9A60144ADA60144ADA61144AD9
:100680001A61144A1A62144A5A62144A9A62144A43
:10069000DA62144A9A61144A5A61144A0260144A8E
:1006A00042604FF080420261002400250122186060
:1006B000C0E902454261836130BD00BF580C002093
:1006C000880C00201D070008AD070008610600081F
:1006D000E1050008490600084D0600084506000827
:1006E000410600085306000857060008990C030845
:1006F000AE0C0308074A115C0023D05C814202D192
:10070000054B585C70470133102BF6D14FF0FF308A
:10071000704700BFF60C0308E40C03082DE9F8430A
:100720001A4E1B4F16F801E01A481B4ADFF8748076
:10073000DFF8749000244FF0010C335D9E451ED10C
:100740007B6C13F480730CD17D6C45F480757D64F3
:100750004360D3625360C2F808C0C2F80C80C2F88C
:100760001090BEF10F0F0ADC08460C4B0C4C98475A
:10077000002201231146A0470020BDE8F883013480
:10078000102CDAD10320BDE8F88300BFF60C030873
:10079000003802400023014000200140F506000817
:1007A000390F00089224490292244912074B5B5CDE
:1007B0000F2B10B507DC0846054B064C9847002365
:1007C0001A461946A047002010BD00BFF60C0308CA
:1007D000F5060008390F000870B5054E054D0024D8
:1007E000214630460134A847102CF9D170BD00BF16
:1007F000580C0020AD070008C2F30B02034B11B1E7
:100800005A61002070479A60FBE700BF0074004007
:10081000022070470C2070470020704740F6FF70A0
:100820007047000070B50E1D0D46002031460D4B7F
:100830009847044680B90C4A136C43F00053136484
:100840000146024601233046084EB047084B1A685D
:1008500025B142F480321A60204670BD42F0010298
:10086000F9E700BF150C000800380240390F0008F6
:100870000074004070B50D1D0E46002029460F4B38
:1008800098470446A8B90E4B1A68A6B122F48032E4
:100890001A6000231A46194628460A4DA847084BF5
:1008A0001B6813F0011F01BF074A136C23F00053AC
:1008B0001364204670BD22F00102E9E7251000080C
:1008C00000740040390F000800380240104B1148F6
:1008D000002230B55A60104A9A60104ADA60104A15
:1008E0001A61104A1A62104ADA61104A5A61104AB3
:1008F0009A61104A0260104A4260104A0261002464
:10090000002501221860C0E902454261836130BDC3
:10091000A80C0020D00C002025080008750800084D
:10092000F907000811080008150800081908000850
:100930001D080008990C0308060D0308020000407A
:1009400070B5054D054C00212846A0472846234692
:100950000121BDE870401847A80C00207508000868
:1009600001230B7000207047002070470348086087
:100970000349116002221A6000207047840D0308A9
:100980007C0D0308114B1248002230B55A60114A01
:100990009A60114ADA60114A1A61114A5A61114A81
:1009A0009A61114ADA61114A1A62114A0260114AC7
:1009B00042604FF0005202610024002501221860BD
:1009C000C0E902454261836130BD00BF100D0020C7
:1009D000F00C002061090008690900082D030008D7
:1009E00065030008C9020008890200086D090008B3
:1009F000990C03083C0D030801F1774101F57401DE
:100A00000023B1F5802F13603CBF4FF40033136017
:100A100010680028CCBF002001207047014B53F81C
:100A2000210070470C10002010B5054B054A064CFC
:100A300003EBC101D1E900010023A04710BD00BFB5
:100A40005011002020BF0200F5FC02085020704722
:100A50002DE9F74F02AD012001F00F0845F8080D10
:100A60008A464FEA880909F00C01144600FA08F694
:100A70000F224FEA2A192846344B4FEA980702FA08
:100A800001FB09FA01F99847002C49D0BB0003F19A
:100A9000804303F59C339A680BEA0202914509D022
:100AA0002B4A126816424ED19A6822EA0B0242EA99
:100AB00009029A60274B2849284A4FEA481803EB55
:100AC000080703F808A001EBCA0A3A610023244A88
:100AD000DFF89C80DAE90001C047224B78607C6136
:100AE00000209847C7E90201194B9968F243114069
:100AF0009960D9680A40DA60DA683243DA609A6845
:100B000032439A605E615C693440FBD11A681643D7
:100B10001E602846144B9847204603B0BDE8F08F6E
:100B20000237124B53F827300BEA03039945F0D1F3
:100B3000074A136823EA0606064B166003EB4818BB
:100B4000C8F81440E5E70C24E3E700BF35170008B8
:100B5000003C0140380D002050110020380F0020CB
:100B600020BF0200C52600085517000800380140C4
:100B7000F5FC02084F2911DC0B119B0203F18043A5
:100B800003F5003301F00F011869C84010F00100AF
:100B90001DBF0123002013601060704703207047C1
:100BA0004F2910DC0B119B0201F00F0003F1804371
:100BB000012103F50033814089B2012A0CBF19835A
:100BC000598300207047032070474F2904DC032A13
:100BD0008CBF002001207047002070474F2910B5BE
:100BE0000C460FDC511E42F20E7399420CD8D317FB
:100BF000002006498847064B03EBC403C3E9000104
:100C0000002010BD052010BD0F2010BD25280008B4
:100C10005011002037B502AC012344F8083D0D46C1
:100C200020460C4B98474F2D0FDC0B4A32F81530FD
:100C3000012B0CD043F0010322F81530002520468B
:100C4000064B9847284603B030BD0525F7E70C252D
:100C5000F5E700BF351700086C0F00205517000896
:100C6000144B1548002230B55A60144A9A60144A51
:100C7000DA60144A9A61144A1A61144A5A61144A91
:100C8000DA61144A1A62144A5A62144A9A62144A7D
:100C9000DA62144A1A63144A0260144A4260144A1F
:100CA00002610024002501221860C0E9024542616A
:100CB000836130BD380F0020D0130020150C0008D0
:100CC00025100008CB0B0008750B0008A10B0008CD
:100CD0001D0A0008CD0F0008290A0008DD0B0008D6
:100CE000510A00084D0A0008990C03088C0D0308EE
:100CF000040000402DE9F341214B02AE01251B68A1
:100D00000446984746F8085D05FA04F830461D4D3C
:100D10001D4B6401984704F118021C4B295D2A44BD
:100D2000002098471A4B2F19C3F814807B69F3B140
:100D30007B68B3B10020DFF86880C047D7E90223A1
:100D4000801A61EB03012A5D124B03EBC203D3E966
:100D50000023994208BF904209D30020C047C7E949
:100D600002012B19295D5F699A691869B8470A4B16
:100D70001B6898473046094B984702B0BDE8F081A0
:100D80006C140020380D002035170008750B000882
:100D9000003C014050110020681400205517000845
:100DA000C52600080020014B184700BFF50C0008BD
:100DB0000120014B184700BFF50C00080220014B31
:100DC000184700BFF50C00080320014B184700BF6F
:100DD000F50C00080420014B184700BFF50C000873
:100DE000084B70B55C691B68074E1C40C4F3441483
:100DF0000525E30701D52846B047640805F101053C
:100E0000F7D170BD003C0140F50C0008084B70B5EF
:100E10005C691B68074E1C40C4F385240A25E30760
:100E200001D52846B047640805F10105F7D170BD2A
:100E3000003C0140F50C000800F00F02930003F0A5
:100E40000C019308023310B50B4C54F823400F23C8
:100E500000098B408840234098420BD1074801216C
:100E60000368914023EA01030360054B03EB421240
:100E700000235361012010BD00380140003C0140B7
:100E8000380D00202DE9F04F041100F00F05012668
:100E9000A40204F1804405FA06F00327022A85B073
:100EA00004F5003406FA05FB07FA00F703D0032A1D
:100EB00014BF002602260DF11008012248F8082D63
:100EC000814086401A4A01914046C3F3031A0093B9
:100ED000904720680199009BFA431040014321602C
:100EE000E1680A401643E660A2684FEA8509ED1002
:100EF000174304EB8505A7602A6A0F2109F01C0936
:100F00000AFA09FA01FA09F922EA090242EA0A028E
:100F10002A6213F0010F636814BF4BEA030323EA4C
:100F20000B0363604046034B984705B0BDE8F08F64
:100F3000351700085517000838B504464F2C0846E9
:100F4000114611DC03F00F02012A0BD0002A18BF52
:100F500002210246054D2046A8472046044B9847EB
:100F6000002038BD0321F4E7032038BD850E0008BA
:100F7000390E00084F2870B50A4604460EDC0146BB
:100F8000074B084D00209847002320461A460121B0
:100F9000A8472046044BBDE87040184770BD00BF0D
:100FA000A10B0008850E0008390E000870B500235B
:100FB00004460A46034D1946A8472046024BBDE8A1
:100FC00070401847850E0008390E00084F2937B5C4
:100FD0000C4615461CDC032A18D8DFE802F0120282
:100FE00012120C4B01AA984701994B1E59425941C4
:100FF0002046094B9847094B43F82450002003B082
:1010000030BD11462046064B9847F4E70420F6E72A
:101010000520F4E7750B0008750F00080C10002080
:10102000AD0F0008F7B502AD012345F8083D0E46A7
:1010300007460B4B284698474F2E0EDC094B0024E1
:1010400023F81640224631463846074B9847284633
:10105000064B9847204603B0F0BD0524F7E700BFD4
:10106000351700086C0F0020CD0F00085517000839
:101070002DE9F0410024174F174E254627F814504C
:101080002146142200200134B047502CF6D1134BD6
:10109000134C1D60002213490620A047002212496C
:1010A0000720A047002211490820A047002210492C
:1010B0000920A04700220F490A20A04700220E491C
:1010C0001720A047234600220C492820BDE8F04104
:1010D000184700BF6C0F0020DD0B0008003C0140EA
:1010E000CD160008A50D0008B10D0008BD0D0008C3
:1010F000C90D0008D50D0008E10D00080D0E00080F
:10110000012A08D052B9E123054A13711B0A537111
:1011100011600020704748F22603F5E7042070476D
:101120001014002010B51F200A4CA0472020A04713
:10113000094B0A4A0A4C00201880136C23F4001350
:1011400013641721A04710B91621A04700B1192038
:1011500010BD00BFF91600080054004000380240DE
:101160002510000838B5172100201B4CA04710B1EE
:101170000C24204638BD1621A04704460028F7D18C
:101180000246164D432302211720A8472246432337
:1011900002211620A847124B12491A6C124D42F434
:1011A00000121A644FF400121A621C62A3F5F233A3
:1011B0002D229A80E1229A832E221A844FF48042B3
:1011C0001A8101221A801F202246A8472246074979
:1011D0002020A847CDE700BF150C0008390F0008F4
:1011E0000038024075140008CD16000839140008B4
:1011F0000F4B1048002230B55A600F4A9A600F4AD0
:10120000DA600F4A1A610F4A5A610F4A9A610F4A0F
:10121000DA610F4A02600F4A42600F4A02610024FD
:10122000002501221860C0E902454261836130BD9A
:10123000F013002048140020651100082511000853
:1012400001110008AD1200080D1300086D1300080D
:10125000990C0308C30D030805000040114A517999
:101260001379114A03EB0123918B89B28B420AD087
:1012700013F4004F4FF000019BB21180938314BF11
:101280000E232E231384084B01221A8000229A82F7
:101290009A8892B242F440729A8040F201521A80C7
:1012A000704700BF1014002000540040F8B51546E8
:1012B0001E46124B124C596001221A702A689A601D
:1012C00000229A705A70DA6023600E4B0E4F9847D6
:1012D0002368987820B94FF47A720023B847F7E76B
:1012E000DB682A68934204D1002232602B60002020
:1012F000F8BDFBD2002BF9D00122F6E7181400202C
:10130000401400205D120008B5260008F8B5154607
:101310001E46124B124C5960002229681A709960BF
:101320009A705A70DA6023600E4B0F4F984723680B
:10133000987820B94FF47A720023B847F7E7DB6852
:101340002A68934204D1002232602B600020F8BD4D
:10135000FBD2002BF9D00122F6E700BF2C140020AD
:10136000401400205D120008B52600082DE9F04762
:101370001E4C1F4DDDF82080616017460022396841
:10138000A160E2606B60DFF87090D8F80030AB606D
:101390000121184B099E2270A27061702970AA70F9
:1013A0006A70EA60C9F800409847DFF850A0D9F8A1
:1013B0000030987820B94FF47A720023D047F6E7CE
:1013C000E26839688A4202D03A60012306E0EA689E
:1013D000C8F80020DB689A4202D10023336002E0A3
:1013E00001D9002BF1D10020BDE8F0872C1400209A
:1013F000181400205D12000840140020B5260008D3
:101400000B4B1A8B910702D51A8892050AD59A8838
:1014100022F4E0621204120C9A80064B1B6801222F
:101420009A7070471A8892B242F400721A80EEE7FE
:101430000054004040140020094B10B51B68984729
:10144000084B00229A82084B1B680BB102221A61DA
:10145000064B9847064BBDE810401B68184700BF75
:101460006C140020005400404014002001140008B7
:1014700068140020454B2DE9F0411B68444D984706
:10148000444A2C68918A2678138B1388A06889B205
:101490009BB201F00107002E5BD01E4697B10128D8
:1014A0000BD123F480639BB213803B4B394A1B68FA
:1014B0005B00DBB2013313823AE00228F5D143F43A
:1014C0000063F1E78F0716D5012809D143F40073B3
:1014D0001380304A93889BB243F48063938005E085
:1014E000022825D123F480639BB213802B4BBDE8E7
:1014F000F0411B6818474B0618D502280FD146F457
:101500000076B3B21380E3686168178ACF54E3684A
:10151000918A01330138E360A06089B2EBE70328C8
:10152000F1D14F07E2D526F48066EAE70128D0D052
:101530000028DBD163782BB3164A938823F48063A9
:101540001B041B0C938040F201531380144B2B603F
:10155000CCE72FB1104B1B685B0003F0FE03AAE73A
:1015600060B10E060AD5E3686168C95C1182918A90
:1015700001330138E360A06089B2F1E74B0758BF3F
:101580000130D5E7074B9847B0E700BF6C14002047
:101590004014002000540040101400206814002063
:1015A000181400200114000808B50748074B984795
:1015B000074A0023136013715371064A9360D36086
:1015C000054A9360D36008BDF01300202511000880
:1015D00010140020181400202C140020104B4FF081
:1015E000FF3210B5C3F88020C3F88420C3F88820E8
:1015F000C3F88021C3F88421C3F88821094A0A4B23
:10160000D3630A4B0A4CDC609A605A6A42F4E022C7
:101610005A62084B1860084B0020196010BD00BFCB
:1016200000E100E0000000201129000800ED00E0CA
:101630000007FA056C140020681400200020704791
:10164000EFF3108000F00100704762B6704772B689
:101650007047EFF3108362B630BF83F31088704792
:101660000F4B1048002230B55A600F4A9A600F4A5B
:10167000DA600F4A1A610F4A5A610F4A9A610F4A9B
:10168000DA610F4A02600F4A42600F4A0261002489
:10169000002501221860C0E902454261836130BD26
:1016A0009014002070140020DD1500083D1600087D
:1016B0004B1600084F160008531600084116000884
:1016C000990C0308F90D0308010000200346094A9C
:1016D000103042F8201003F01F025B119B0003F151
:1016E000604303F56143012000FA02F2C3F8802150
:1016F0001A60704700000020421100F01F032032E2
:101700000120034900FA03F341F82230704700BF7B
:1017100000E100E00368426893430CBF0120002011
:101720007047426803681A4203D1EFF310834360A5
:1017300062B67047EFF31083436072B670470000E3
:1017400090E80C0032EA030301D1014B18477047BF
:1017500035170008426803681A4200D162B6704724
:10176000014B024ADA60FEE700ED00E00400FA05F2
:1017700000207047012910B506D0022937D0244A2D
:10178000136843F004033FE0224B1B6803B1984702
:10179000214A1F49136943F0040313610B6843F4A2
:1017A000017343F001030B6030BF1C4B196841F417
:1017B00080311960116921F0040111611A689103E7
:1017C000FCD51A6842F080721A60144B1A689201B4
:1017D000FCD59A6842F002029A601A6822F001026F
:1017E0001A600F4B1B688BB1BDE810401847094BBE
:1017F0001B6803B19847084A136943F00403136157
:10180000034A136843F00603136030BF10BD00BFE6
:1018100000700040C814002000ED00E000380240D5
:10182000CC140020002070470D4B0E48002230B52C
:101830005A600D4A9A600D4ADA600D4A1A610D4AE3
:101840005A610D4A02600D4A42600D4A026100244D
:10185000002501221860C0E902454261836130BD64
:10186000B0140020D01400202518000871170008BB
:101870006117000875170008990C0308350E030856
:1018800002000020426858235343154A11F0010F0B
:10189000D3580CBFFF204FF47F408A0755BF1A8BE7
:1018A0009A8B03F1180103F11C0192B222EA0002A3
:1018B0000A80198B9A8B0A4392B272B909490A4A73
:1018C00013F4803F18BF0A46C3F384231168012034
:1018D00000FA03F321EA030313600020704700BFFE
:1018E0000004002044380240403802404268084961
:1018F000582353431A1D14330A440B44002052F852
:10190000041F013118BF01309A42F8D1704700BF5F
:1019100000040020000000004268582353430A4A94
:10192000D358DB0302D49FED040B70479FED040BEB
:10193000704700BFAFF30080000000002A758541AA
:10194000000000002A7595410004002000000000FE
:101950009FED010B704700BF000000000000F03F4A
:101960002DE9F04F47683C4D924658233B4A7B4354
:1019700002EB030B2DED028BB0EE408AF0EE608A95
:10198000DBF85090D458364B83B048460E46984703
:1019900053EC182BCDE90001A847324B2F4D984747
:1019A000DBF85430013B9BB2238509F1FF338145BD
:1019B000E36207F10103C84628BF8046022BDFF827
:1019C00098903ED176BBC4F83480B2000223934095
:1019D000228CBAF1000F3BD013439BB223840B231C
:1019E00003FB076305EBC303D3E90C23DDE9000127
:1019F000C8471C4B984740451CBF0123A38258236E
:101A000003FB07533344002083F818A00B2303FB88
:101A1000076605EBC60585ED0C8B03B0BDEC028BAC
:101A2000BDE8F08F012E02D1C4F83880CDE7022E38
:101A300002D1C4F83C80C8E7032EC6D1C4F8408068
:101A4000C3E704F134031FFA88F223F82620BCE729
:101A500092B222EA0303C1E7C5F5020800040020A0
:101A6000D9F4020875FB0208F8B5436858225A43B6
:101A70000D4623498C5816225E1C02FB0353023389
:101A8000002051F823101F4B9847002837D11E4BD8
:101A90001E4A14F4803F18BF1A4601211768C4F388
:101AA000842301FA03F31F4213D117683B431360E9
:101AB0008E424FF084032380A18201D0082E08D1EA
:101AC000B4F844306FEA43436FEA53439BB2A4F83F
:101AD000443004F13403002223F8252015F0010FCF
:101AE0000CBF68214FF4D041AB0755BF238BA38BAC
:101AF00004F1180204F11C029BB20B431380F8BDE1
:101B000000040020150C0008443802404038024010
:101B1000436870B51620114E0C4658225A4300FBFC
:101B20000343B118981CB5584B6856F820000C4E6A
:101B300000210122B047A4002B8C012202FA04F4F8
:101B40001C43A4B22C842B889BB2D9075CBF1343DF
:101B5000AA824FF0000058BF2B8070BD0004002007
:101B6000390F00084368124858225A4370B5855807
:101B7000104E2C8C162202FB03130233890050F8FE
:101B80002300012303FA01F1A4B2002324EA010493
:101B90001A4619462C84B04741F211131C4205D154
:101BA0002B8823F001031B041B0C2B80002070BD2D
:101BB00000040020390F00082DE9F0431C4A1D4D98
:101BC0001D4CDFF89C90DFF89C80DFF89CC0DFF8AC
:101BD0009CE01A4F1A4E0021302048432B182A50FF
:101BE00018481862184844F8213059605862013189
:101BF000164898620E291648C3F81C90C3F808804E
:101C0000C3F80CC0C3F810E05F619E61D862E3D1F5
:101C1000104B1360104B53600026104B13610027CC
:101C2000C2E90267516194610148BDE8F08300BFD9
:101C3000C817002028150020F0140020651B00089C
:101C4000611900085119000819190008311D000810
:101C5000ED180008990C03086D0E030806000040FB
:101C6000811E0008691A000885180008111B000869
:101C70002DE9F84F55EC104B07460E46DFF89CB0A7
:101C8000214BDFF89CA0DFF89C90DFF89C800022BD
:101C900010EE100A2946D84770B122462B4616A1ED
:101CA000D1E90001D047194B0022C847C047184B63
:101CB00038603360BDE8F88F0022164B2046294675
:101CC000D84722462B4650B10DA1D1E90001D0479B
:101CD0000E4B0022C847C0470F4B3860E9E7002091
:101CE0000949D047094B0022C847C0474FF47A73CF
:101CF0003860DEE7AFF300800000000065CDCD4125
:101D00000000000080842E4100408F400000E03F32
:101D100000CA9A3B0000F03F40420F00D1FA02088F
:101D200019F8020861F2020875FB020800000000C1
:101D30002DE9F04F2DED028B87B006A9D0F804B045
:101D4000474D002341F8043D0493582303FB0BF354
:101D5000EA1892ED0A8BEC58B0EE480AF0EE680AE9
:101D6000404B04A89847404A4049DDF8149002953A
:101D700014F480330CBF884690460BF10106DDF861
:101D800010A0B8FBF9F545B15446B5F5803F15D91B
:101D9000002C33DB6D086400F7E7002B344B354C27
:101DA000B9FBF4F40CBF5A25B4259A459DBF0AFB34
:101DB00005F5B5FBF4F40125BAFBF4F4022E22D0AC
:101DC000052E20D0B4F5803F1DD3B5F5004F15D8B2
:101DD0006D006408F6E7029A9DED007B582303FB33
:101DE0000B2B8BED087BCBF85040CBF854509DED7E
:101DF000000B07B0BDEC028BBDE8F08F9FED167BAA
:101E00008DED007BF3E7002CF8D0B8FBF5F31A4A10
:101E100003921F46B3FBF4F3B9FBF3F8B9FBF8F0F8
:101E20009047D045CDE9000107D353EC182BDDE9ED
:101E30000001124EB0470028CDD00134B7FBF4F3B7
:101E4000B9FBF3F8B8F1000FD8D0B9FBF8F0039B59
:101E50009847E6E7AFF300800000000000000000B4
:101E600000040020711C00080095BA0A804A5D0534
:101E7000C1166C0140420F00D9F40208E5FA0208CD
:101E80002DE9F84F43681D4F1D4CD1E900895825B5
:101E90005D4307EB050B06468A4642464B46DBE9A7
:101EA0000A01A047044610B10020BDE8F88FCBE935
:101EB0000A893046134B984705F104098AED000B57
:101EC00005F13008DFF840A0B944B84459F8043FA0
:101ED000013305D10134042C08F10808F6D1E3E7F9
:101EE00063193B4498ED000B1A7E21463046D047DB
:101EF0000028EFD00820BDE8F88F00BF00040020C4
:101F000095FA0208311D0008611900080000000060
:101F10002DE9F84F2DED028B9FED1B8B1C4CDFF84C
:101F200078800026DFF874B004F12C074FEA860AA7
:101F3000A146002559F8043F01330ED029465AF82E
:101F40000800D847134B5AF8080029469847231F22
:101F50002B44002287ED008B1A760135042D07F102
:101F60000807E7D1013600230E2E84ED098B84ED9E
:101F7000078BE364236504F15804D3D1BDEC028BD5
:101F8000BDE8F88FAFF30080000000000000000003
:101F90000404002085180008F0140020651B0008C8
:101FA00010B54468012C09DC054800EB441083613E
:101FB000029B01614261C361002010BD082010BD79
:101FC000F01700200120704700487047006CDC02C9
:101FD0005020704743680B4A70B5D65C0A4A0B4CD8
:101FE000D55C0B4A0020D15CA04708B1062070BD2B
:101FF0003146A0470028F9D12946A0470028F5D14D
:1020000070BD00BFF40E0308F60E0308150C00089F
:10201000F80E03084368094A70B5D65C084A094CB3
:10202000D55C094A0020D15CA04731460020A0477A
:1020300029460020A047002070BD00BFF40E030811
:10204000F60E030825100008F80E030810B5084620
:10205000144639B112680549054B022A28BF0222ED
:102060009200984702232360002010BDD008002072
:10207000CF0103082D4B2E492E48DFF8E0C02DE993
:10208000F04F2D4C9C62002203F1340B2B4C1A7143
:102090005A719A71DA71DFF8C8A0DFF8C890DFF8DA
:1020A000C880DFF8C8E0264F264E274DDC62C1F815
:1020B00004B0264C83F8392083F83A2083F83B207B
:1020C0004FF0010B1C4A0B601860C3F808A0C3F85E
:1020D0000C90C3F81080C3F814C0C3F818E0DF6197
:1020E0001E625D621C63586383F838B0C3F83CA07D
:1020F000C3F84090C3F84480C3F848C0C3F84CE02C
:102100001F655E659D65DA650C4A1A665C66104B54
:102110000360104B4360104B036100220023C0E9B1
:102120000223022343618161BDE8F08F3018002053
:10213000E817002098180020C51F0008C91F0008D4
:1021400071240008B1250008D11F00084D200008A7
:10215000990C0308A30E030807000040E1240008BF
:10216000D51F000815200008A11F000845250008FC
:102170002DE9F843024605280FD8DFE800F00309EF
:102180006E73787D43494B6C43F480534B6404E099
:1021900040490B6C43F480430B643F4C3F4B56016A
:1021A000A11953F822708B69C969102B40F644338A
:1021B00018BF4FF45173022963D0032964D0012959
:1021C00001D143F00103A1194AF6C8704D6945F2E7
:1021D000E47E4FF47A7195FBF1F5511E01298CBF15
:1021E00001467146B1EBC50F84BF090943F02003D6
:1021F000B1EB450F84BF890843F01003A94288BFA3
:1022000043F008039BB23B80254B985C254B13F8A9
:102210000290254B022A13F8028038D140F2522353
:1022200040F26225B8F1360F08BF1D461F4F2B46FE
:1022300001220021B84700222B461146484634446B
:10224000B8472B46012200214046B8472069184B69
:10225000002198470120BDE8F8830E490B6C43F438
:10226000004399E70B494B6C43F400538EE709494F
:102270004B6C43F4801389E706494B6C43F400131D
:1022800084E743F002039EE743F003039BE740F239
:102290005225CBE700380240F0170020DC0E03087F
:1022A000F80E0308F40E0308F60E0308390F0008B1
:1022B000750F0008F8B5254B53F8203004461889EF
:1022C00010F08000FBD1224D188005EB441501224F
:1022D0002969204B9847EB691F4D032B1F4B1F5D4E
:1022E0001F4B1E5D1F4B14BF03210221185DA84721
:1022F00003213846A84703213046A847052C0FD8AC
:10230000DFE804F0030910151A1F174A536C23F471
:102310008053536404E0144A136C23F48043136421
:102320000120F8BD104A136C23F40043F7E70E4A6E
:10233000536C23F40053ECE70B4A536C23F48013E3
:10234000E7E7094A536C23F40013E2E7DC0E0308C5
:10235000F0170020A10B0008AD0F0008F40E0308D1
:10236000F60E0308F80E030800380240194B1A490C
:1023700053F8202040010B18F0B50E5899685F689B
:10238000D3F80CE0C1B100233C78A0B290810020CA
:102390000130814214DD8645C8BF3C5C1589ED07DC
:1023A000FCD59589002BADB21FFA84FCA2F80CC0B5
:1023B000A8BFF5540133EBE771464FF00043E3E764
:1023C0001189C907FCD59289002B92B2A8BFF2549B
:1023D0000120F0BDDC0E0308F0170020224BF0B501
:1023E00053F82040214B40011A181D585668D268F6
:1023F000034412F0010F99684FEA520218BF0132EC
:1024000011F001034FEA51011FD10029084604BF12
:102410004FF0004310463788A781002101318842E0
:1024200016DD8A42C8BF36F81170B4F808E01EF015
:10243000010FFAD0B4F80CE0A781002B1FFA8EFE32
:10244000A8BF25F813E00133E8E7481C0023E2E7C2
:102450002289D207FCD5A289002B92B2A8BF25F809
:1024600013200120F0BD00BFDC0E0308F017002090
:102470002DE9F8434468012C88461746994602DD49
:102480000820BDE8F8832046104B98470028F7D075
:102490000F4E089B650170191B6883603B68C36021
:1024A0008369C0F80480102B46F8059020460BD1B4
:1024B000084B98470028E3D02046074B9847002850
:1024C000DED00020BDE8F883044BF2E7712100085C
:1024D000F0170020DD230008B52200086D23000856
:1024E000F8B54468012C0F46164601DD0820F8BDFA
:1024F00020460F4B98470028F8D00E4D32686001F7
:102500002B182F509A6000225A60DA609B69102BBA
:1025100020460AD1084B98470028E7D02046074BB1
:1025200098470028E2D00020F8BD054BF3E700BF34
:1025300071210008F0170020DD230008B5220008F3
:102540006D2300082DE9F0414468012C88461746A8
:1025500002DD0820BDE8F0812046104B9847002896
:10256000F7D00F4E3A686501731900209860C3F8E0
:102570000480DA609B697051102B20460BD1094B07
:1025800098470028E5D02046074B98470028E0D020
:102590000020BDE8F081054BF2E700BF7121000883
:1025A000F0170020DD230008B52200086D23000885
:1025B00070B51D46064B049E0446984730B9324616
:1025C00029462046034BBDE870401847082070BDDF
:1025D00045250008E124000870B5044D044C286826
:1025E000A04768682346BDE870401847E8170020F8
:1025F00015200008024A034B02609B1A0B607047CB
:1026000000900020F8EF022010B50A4A0A490B4852
:102610000B4CA0470B4A0C490C48A0470C4B0D4AE9
:1026200023F0030300211BB142F8041F043BFAE727
:1026300010BD00BF0000000008750020A073030853
:10264000990100085808000000040020456B0308A9
:10265000AC680000540C00200420704710B50A2418
:10266000A2FB040104FB0311B4220023014CA04788
:1026700010BD00BFF5FC020810B5104619460A222D
:102680000023054CA047B424A0FB042304FB013322
:102690001046194610BD00BFF5FC02080020704727
:1026A000034A136823F0010313600020704700BF42
:1026B00010E000E0B420A2FB00010538004B1847F1
:1026C0007B0C030873B502AE012346F8083D144B9A
:1026D0003046984713480168826811F4803F22F021
:1026E0007F42114902D18B689A4203D322B14368D9
:1026F000886803449B1A00E08B688A60D1E9004532
:10270000E41845F100053046084BC1E900459847FB
:102710004FF0FF304FF6FF712040294002B070BDEE
:102720003517000810E000E01019002055170008C8
:102730002DE9F74302AE1C46012346F8083D8046CA
:10274000124B134F3046154698474046B847B421C0
:10275000A5FB012301FB0433002B08BF042A81469B
:1027600011D3D41E43F1FF354046B847A0EB090012
:10277000C1178D4208BF8442F6D23046054B9847B8
:1027800003B0BDE8F08300240025EDE7351700080D
:10279000C526000855170008134B1448002230B511
:1027A0005A60134A1A61134A9A61134ADA61134A4A
:1027B0005A61134A1A62134A5A62134A9A60134AB8
:1027C000DA60134ADA62134A9A62134A0260134AC1
:1027D0004260134A02610024002501221860C0E90A
:1027E00002454261836130BDC0180020F01800200E
:1027F000592600085D26000879260008C52600082D
:102800005D290008892800089D260008A1260008E7
:1028100031270008B5260008990C0308FA0E0308B2
:102820000300002010B5034CA2FB040104FB0311BC
:1028300010BD00BF20BF02000A4B6FF07F42002096
:102840000021C3E900019A60DA60074B013A5A603F
:10285000064AF02182F8231000229A6007221A60AB
:10286000012070471019002010E000E000ED00E0AA
:10287000034B9860034B0138002258609A60704700
:102880001019002010E000E0F7B502AE1D4601234C
:1028900046F8083D0746174B304614469847164BF6
:1028A00038469847154BC3E900454FF6FF739D42E4
:1028B0004FF0FF3208BF9442114B05D16FF07F40BB
:1028C000D860104B984705E0A94208BFA04207D343
:1028D0001B69984730460C4B9847002003B0F0BD69
:1028E000201AD860094B984288BF6FF07F40054B93
:1028F000E8E700BF35170008C5260008B818002013
:10290000101900207128000855170008FEFFFF006D
:102910000C4B10B51B6898470B4B002098470B4B8E
:10292000D3E90023994208BF904207D3084B1B69A3
:102930009847084BBDE810401B681847064900201F
:102940008847F6E76C140020C5260008B818002058
:1029500010190020681400208928000870B50B4D5C
:102960002C690E4684B90A4B4FF6FF714FF0FF30C9
:10297000C3E90001074B98476FF07F40064BE860C2
:1029800098472E61204670BD082070BD10190020A8
:10299000B818002039280008712800080020704766
:1029A0004368044A4FF44B7000FB03230020C3F834
:1029B00020137047381900204368044A4FF44B70C5
:1029C00000FB03230020C3F82413704738190020AC
:1029D00007207047072070470A4A38B543684FF40C
:1029E0004B7101FB032393F81C234AB1064D1C468F
:1029F000D4F8000328B1012200230020A847F7E7FC
:102A0000062038BD38190020B52600080720704779
:102A1000072070470720704707207047072070473E
:102A200007207047072070472DE9F34102AD0123CD
:102A300045F8083DD0F80480214B224C28460F462B
:102A4000164698474FF44B7000FB08F0221892F896
:102A50001C1359B33368D2F80C23934226BF00F5F8
:102A60004370001930463946036833604FF44B73A6
:102A700003FB084300243068CA1B90421ED9D3F8D8
:102A800014231A4492F8002101F8012BD3F81423DF
:102A9000D3F80C0301320138B2F5007FC3F81423D8
:102AA000C3F80C03E7D1C3F81443E4E7062428462F
:102AB000054B9847204602B0BDE8F0810024F6E7B8
:102AC000351700083819002055170008F7B5466873
:102AD000032E07464FF0010022DC02AD114B45F8F2
:102AE000080D28469847104A4FF44B7303FB062302
:102AF0000E4AC3F82873002452F82620C3F8004376
:102B0000C3F80443C3F80843C3F80C43C3F81043A5
:102B1000C3F81443C3F818232846054B98472046AA
:102B200003B0F0BD3517000838190020680F0308FE
:102B3000551700082DE9FF4104AC012344F8083D76
:102B40004568304B304E204690460F4698474FF42C
:102B50004B7303FB056393F81C23002A4FD0D3F873
:102B60000033D8F80020C3F580739342019394BFDB
:102B700001AB43461B68C8F800304FF44B7303FBAE
:102B80000563D3F80023B2F5807F1AD039464FF0A1
:102B9000000ED8F80020C81B824222D9D3F80403C3
:102BA00011F8012B1A540130D3F80023B0F5807FBF
:102BB00002F1010208BF7046C3F80023C3F8040302
:102BC000E7E7D3F820233AB9002520460F4B984772
:102BD000284604B0BDE8F0810421D3F828039047CB
:102BE000F2E7002AF0D04FF44B7303FB0565D5F8EC
:102BF000182393899BB243F080039381E4E7062571
:102C0000E3E700BF35170008381900205517000802
:102C10002DE9F0414468069F079D5B48052C5DD176
:102C2000466C46F0200646645848594E00EB510069
:102C3000B0FBF1F14FF44B7000FB046089B2D0F8A7
:102C400018030181002B5CD040F20C6E40F20C4165
:102C50000132012B14BF0B467346092A53D143F4AA
:102C60008053012F838153D0022F0CBF02230023F6
:102C70001B03012D03824DD002D3032D40F281802E
:102C80000023032C83824348434F50F82400B4BFF1
:102C90004FF072084FF08208434600220221B847E5
:102CA0003E4843460122002150F82400B847012D38
:102CB0000DD13B4800221146434650F82400B84746
:102CC000384843462A46002150F82400B847052CCE
:102CD00028D8DFE804F02242464A4E521CB9466C1E
:102CE00046F010069FE7042CD0F840E0D4BF4FF424
:102CF00080364FF08076A64046EA0E0606642A48E3
:102D000093E70C23A9E7082AABD00120BDE8F081A6
:102D10000323ADE74FF44073B3E724490022252095
:102D2000234B98474FF44B7303FB0464012384F84F
:102D30001C33D4F818339A8992B242F080029A81F7
:102D40009A8992B242F020029A819A8992B242F410
:102D500000529A810020BDE8F0810022154926200A
:102D6000DEE7002214492720DAE700221349342045
:102D7000D6E7002212493520D2E700221149472028
:102D8000CEE70420BDE8F08100380240804A5D05AE
:102D900038190020880F0308390F0008980F03081E
:102DA000A80F0308B80F030840A5AE023D31000884
:102DB000CD1600086D3100089D310008CD310008A6
:102DC000FD3100082D3200082DE9F043244A254D3D
:102DD000254CDFF8DC90DFF8DC80DFF8DCC0DFF8C2
:102DE000DCE0224F224E0021502048432B182A506D
:102DF0002048186220485862204898622048D862CB
:102E00002048186320485863204898632048D863B6
:102E100020481864204844F8213059605864013132
:102E20001E48986404291E48C3F80890C3F80C8013
:102E3000C3F810C0C3F814E09F61DE61D864D3D139
:102E4000184B1360184B53600026184B1361002772
:102E5000C2E90267516194610148BDE8F08300BF97
:102E600028270020E825002028190020292A00080A
:102E7000352B00089D290008A1290008B929000860
:102E8000192A00080D2A00081D2A0008212A000816
:102E9000252A0008112A0008152A0008D12900084F
:102EA000D5290008990C0308310F030808000040D9
:102EB000CD2A0008A52F0008112C0008D9290008E8
:102EC0001F4B70B51B68044698471E484FF44B7360
:102ED00003FB0403D3F818239588D3F80C23B2F529
:102EE000007FADB208D1D3F820233AB30221D3F842
:102EF0002803BDE870401047D3F810134E1C013270
:102F0000B6F5007FC3F80C2308BF0022C3F8106396
:102F1000194408BFC3F810234FF44B7303FB040498
:102F200081F80051D4F824331BB10121D4F82803CF
:102F30009847054BBDE870401B68184770BD00BF3F
:102F40006C1400203819002068140020094B4FF43D
:102F50004B7202FB0030D0F81823938921B19BB249
:102F600043F080039381704723F080031B041B0C04
:102F7000F8E700BF38190020094B4FF44B7202FBF1
:102F80000030D0F81823938921B19BB243F020037D
:102F90009381704723F020031B041B0CF8E700BF4C
:102FA0003819002073B502AE012346F8083D0446E7
:102FB0002C4B2D4D3046984764684FF44B7303FB00
:102FC00004530022D3F818339A81052C07D8DFE880
:102FD00004F0032E303234362520244B984700214C
:102FE0002046234B9847234B002120469847052C29
:102FF000214B26D15A6C22F020025A644FF44B73B5
:1030000003FB045400253046C4F80053C4F80453AD
:10301000C4F80853C4F80C53C4F81053C4F814533C
:1030200084F81C53154B9847284602B070BD2620E3
:10303000D3E72720D1E73420CFE73520CDE747205D
:10304000CBE71CB95A6C22F01002D6E7042C1A6C9C
:10305000D4BF4FF480314FF08071A14022EA0102C9
:103060001A64CBE73517000838190020F916000854
:10307000792F00084D2F000800380240551700082E
:1030800007B50D4A4FF44B7303FB0023D3F81833F5
:103090009B8A9B050ED5094B01AA53F82010084BBB
:1030A00000209847019810F1FF3018BF012003B0AD
:1030B0005DF804FB0120FAE738190020A80F030887
:1030C000750B0008184B70B51B68044698472046DE
:1030D000164B9847F8B1164A4FF44B7303FB042381
:1030E000D3F80013E1B1D3F80803451C0139B5F555
:1030F000807FC3F8001308BF0021C3F80853185C91
:1031000008BFC3F808134FF44B7303FB042283B2C8
:10311000D2F818239380074BBDE870401B6818470E
:103120002046054B9847F6E76C14002081300008D4
:1031300038190020681400204D2F0008084B10B5E6
:103140001C88A4B2A20602D50020064B984723068D
:1031500004D50020044BBDE81040184710BD00BF47
:1031600000100140C12E0008C5300008084B10B502
:103170001C88A4B2A20602D50120064B984723065C
:1031800004D50120044BBDE81040184710BD00BF16
:1031900000440040C12E0008C5300008084B10B59F
:1031A0001C88A4B2A20602D50220064B984723062B
:1031B00004D50220044BBDE81040184710BD00BFE5
:1031C00000480040C12E0008C5300008084B10B56B
:1031D0001C88A4B2A20602D50320064B98472306FA
:1031E00004D50320044BBDE81040184710BD00BFB4
:1031F000004C0040C12E0008C5300008084B10B537
:103200001C88A4B2A20602D50420064B98472306C8
:1032100004D50420044BBDE81040184710BD00BF82
:1032200000500040C12E0008C5300008084B10B502
:103230001C88A4B2A20602D50520064B9847230697
:1032400004D50520044BBDE81040184710BD00BF51
:1032500000140140C12E0008C530000870B5054EAD
:10326000054D002456F824000134A847042CF9D158
:1032700070BD00BF28190020A52F0008014B0020B9
:1032800019607047F8290020014B00201960704731
:10329000FC29002038B5B0F8C05090F8A330D0F821
:1032A000BC109D420446A8BF1D462A46114BD0F8CB
:1032B0009C009847D4F8BC30B4F8C02084F8A050E3
:1032C0002B44C4F8BC3094F8A3309D4208BFB4F836
:1032D000C230A9B20CBF5B1A0023A4F8C230B4F804
:1032E000C230521AA4F8C02003B1034BC4F8B8305E
:1032F00038BD00BFCF0103089532000808B5024869
:10330000024B9847002008BD04090020CF010308A4
:1033100008B50248024B9847002008BDE00800208D
:10332000CF01030803290CD8DFE801F0020D1721B3
:10333000144B02F1400152F8040B43F8040B8A428B
:10334000F9D100207047104B02F1400152F8040BF4
:1033500043F8040B8A42F9D1F3E70C4B02F1400128
:1033600052F8040B43F8040B8A42F9D1E9E7084B01
:1033700002F1400152F8040B43F8040B8A42F9D1E0
:10338000DFE700BFAC090020F2090020200900207F
:103390006609002003460022006810B49A601A6093
:1033A0005A600C681C600A605A684C685C604A602D
:1033B0009A688C689C608A6018B1034B5DF8044B76
:1033C00018475DF8044B7047394B000810B50123CE
:1033D00004460360014B9847204610BD351700088E
:1033E00037B50C4608B300EB8103DB68FBB1451829
:1033F00095F86C30DBB90F4B68469847610101F1D5
:10340000A041D1F8003B002B0BDB95F85C3043F476
:103410000023C1F8103BD1F8003B43F00443C1F84E
:10342000003B6846044B9847012003B030BD0020A4
:10343000FBE700BFCD330008551700082DE9F3471F
:10344000294C2A4BDFF8D4A0DFF8D4804FF49477CE
:103450004743814668469847282200212046D047A6
:10346000234B6360002680221A76DE77214BA3600F
:10347000214BE360214B2361214B6361214BA3610D
:10348000214B224AE36108EB0705214B22602362AE
:10349000C422204B636231462846D04701220421D2
:1034A000FF234020A5F8AC2085F8B41008F80720C9
:1034B00085F80290AC606B7085F8A3002A4631460F
:1034C0006C180131102982F87C3082F87D3084F844
:1034D0005C0002F10202F3D168460F4B98470120CD
:1034E00002B0BDE8F08700BF28280020CD330008D7
:1034F000E0080020A6090020EC0900201A0900209D
:1035000060090020482700205E27002004090020D1
:10351000902700200410030855170008190203081B
:10352000D028002030B585B0094B0193094B029398
:1035300004AB094A43F8042D084A4468156801A9F8
:1035400002AAA8472046064B9847002005B030BD88
:10355000482700205E27002090270020FC2900201B
:103560003D34000837B50C4B054668460C46984775
:103570000A484FF4947303FB050045682C43A542A9
:10358000446003D0064B00201B6898476846054BF3
:103590009847284603B030BDCD330008D02800201E
:1035A000F82900205517000837B50A4B044668462D
:1035B0000D46984708484FF4947303FB0400074BEB
:1035C000446824EA0505456068469847204603B0EC
:1035D00030BD00BFCD330008D028002055170008AB
:1035E0002DE9F341194B04460D46684617469847A6
:1035F00035B9D7B96846164B984702B0BDE8F08197
:10360000DFF8508004F10C06002556F8043B43B166
:10361000621992F86C2022B91A685A60294620462D
:10362000C0470135102DF0D1E3E704F10C0304F19C
:103630006C024C3453F8041B19B1107808B10868B7
:103640004860A34202F10102F4D1D3E7CD33000870
:1036500055170008E133000810B5437890F8A22010
:103660009A42044618D0052B03D1012211460B4B78
:10367000984794F8A230637013B1052B05D010BDA4
:10368000A4F8C030C4F8B83010BD20460022012193
:10369000024BBDE81040184710BD00BFE1350008DF
:1036A00091F8A23081F82631062381F8A23008462D
:1036B000004B184759360008D0F8043823F00103AE
:1036C000C0F8043891F8263181F8A2300846014B41
:1036D000184700BF593600082DE9F0474FF0FF3377
:1036E0004361402343624FF0401383620D4691F8DB
:1036F000B4700023FF244FF080419A1CBB424FEA74
:10370000821211DA03F1400642F4800240F82620CA
:1037100000EB43120133C2F80849C2F8084BC2F863
:103720000019C2F8001BE8E74FF4866303614FF409
:103730000043C0F80039B5F82441C0F8003B00232D
:10374000C0F81039DFF8C4C0DFF8C4804FF0C043C0
:10375000C0F8103BA41005F15D06022701234FF0CD
:10376000011164B314F0030213D096F800E096F848
:1037700010904EEA8242B9F1000F0FD048EA835E02
:103780004EEA020203F1480E4FEA4E1E394340F85A
:103790000E200133A4087F000136E2E700EB431955
:1037A0004EF4002EC9F810EB03F1580E4FEA4E1EEE
:1037B00042EA0C0240F80E2041EA0741E9E70126FF
:1037C0000923C0F81068C0F814380D4BC0F81C1855
:1037D0008361D0F8003823F4FE63C0F800384FF05E
:1037E000FF312046074B9847032385F8A230C5F8E0
:1037F000A86085F8A1402846034BBDE8F04718476C
:1038000010180C80A9350008593600080080009473
:10381000008000184B8882B00BB101202AE0CB88D1
:10382000022BFAD190F8A220032AF6D00B7803F0ED
:103830000F03012B20D012D3022BEED1042A8B8848
:1038400001D1002BE9D103F07F038B8090F8B420E5
:103850009342E2DAD0F8B02002EB430301E000F13A
:10386000AC03C0F8BC300223A0F8C030054BC0F850
:10387000B830002002B07047052ACED10DF1060302
:10388000EFE700BF953200084B887F2B10B5044648
:103890001BDC8A88CAB9CA88BAB990F8A220042A5F
:1038A00013DCDBB280F8A1306BB9032384F8A230BB
:1038B0002046074B98470023A4F8C030054BC4F8B6
:1038C000B830032010BD0423F0E7012010BD00BF75
:1038D000593600089532000810B54B88ABB98C8872
:1038E0009CB9CA88012A10D190F8A21003290CD0E3
:1038F00000F1A403C0F8BC30054BA0F8C020A0F82C
:10390000C220C0F8B830204610BD012010BD00BF55
:103910009532000838B58B8804461546EBB9CB883C
:10392000DBB990F8A230032B17D04B88012B14DCA5
:10393000DBB280F8A43073B9042384F8A2302046A7
:10394000074B98472DB10023A4F8C030054BC4F8AD
:10395000B830052038BD0523EFE7012038BD00BF92
:10396000593600089532000870B5836817484668D4
:1039700053F8040B0478022C1BD005D81CB3012C7F
:10398000F6D10129F4D170BD032C15D0FF2CEFD155
:1039900005791478A542EBD145795478A542E7D151
:1039A000C5885488A542E3D105899488A542DFD112
:1039B00070BD34788C42E5E70329D9D15488457825
:1039C000E4B2A542DEE72046DDE700BF282800205C
:1039D00010B5CB8804460A460BB1012010BD90F803
:1039E000A230052BF9D10B7813F00F031BD0022B5B
:1039F000F3D18B8803F07F038B80002BEDD090F800
:103A0000B4108B42E9DA51880029E6D1D0F8B00031
:103A100030F8131021F0010120F81310938884F876
:103A2000B530042011E04B88012BD6D102210A4B7E
:103A300098470028D1D0C37A9B06CED5B4F8AC30D5
:103A400023F00203A4F8AC3006200023A4F8C03011
:103A5000024BC4F8B83010BD69390008953200082F
:103A600010B5CB8804460A460BB1012010BD90F872
:103A7000A2100329F9D0137813F00F0325D0022BDD
:103A8000F3D10429938801D1002BEED103F07F03F9
:103A90009380002BE9D094F8B4108B42E5DA51887A
:103AA0000029E2D1D4F8B00030F8131041F0010140
:103AB00020F81310938884F8B53004200023A4F86C
:103AC000C0300B4BC4F8B83010BD5388012BCCD19B
:103AD0000221084B98470028C7D0C37A9B0605D51A
:103AE000B4F8AC3043F00203A4F8AC300620E5E7AC
:103AF000953200086939000838B5CB884A88A0F8A3
:103B0000C23004460D4618462BB9A4F8C030364BD7
:103B1000C4F8B83038BD94F8A230032B0CDCD4F8CC
:103B2000A8304BB10023C4F8A83094F8A3309842D1
:103B300028BF1846A4F8C2000023C4F8BC30A4F87B
:103B4000C0306B78062B25D1110A022912D0032927
:103B50003BD001291ED12A462046244B9847C8B1A4
:103B6000031DC4F8BC300379B4F8C220934228BFC7
:103B700013460DE02A4620461C4B984750B1031DC2
:103B8000C4F8BC30C288B4F8C2309342A8BF134610
:103B9000A4F8C030D4F8BC3093B92A46FF2120469F
:103BA000124B9847E8B100F10A03C4F8BC304388CF
:103BB000B4F8C2200A3B934228BF1346A4F8C03091
:103BC000094BC4F8B830002038BD12F0FF0FC2D145
:103BD000074BC4F8BC30B4F8C230042B28BF042310
:103BE000D6E7012038BD00BF9532000869390008CA
:103BF000DC08002090F8A030D3B1D0F89C104B78AE
:103C0000092B13D8DFE803F005071209120B121273
:103C10000D0F084B1847084BFCE7084BFAE7084B19
:103C2000F8E7084BF6E70122074B1847074BF1E787
:103C30000220704715380008D1390008613A0008A1
:103C400089380008D938000815390008F93A000801
:103C500000EB8101CB6809CB1B1A432BD8BF002096
:103C600070470000154B1648002230B55A60154ABF
:103C70009A60154ADA60154A1A61154A5A61154A5E
:103C80009A61154ADA61154A1A62154A1A63154A89
:103C90005A63154A5A62154A9A62154ADA62154AF7
:103CA0000260154A4260154A026100240025012283
:103CB0001860C0E902454261836130BD9828002048
:103CC0007828002025350008DD430008454300081A
:103CD000253E0008114B0008793F0008954900086F
:103CE0007D32000889320008FD32000811330008D7
:103CF00025330008990C0308C80F03080900004089
:103D000010B50446006808B1014B9847204610BD25
:103D1000394B00082DE9F0434FF494733A4C434378
:103D200087B0E65C05460F46002E66D00F2968DC9A
:103D3000364B01A89847942303FB057304EB430318
:103D400093F87C90B9F1FF0F18D04A2303FB059339
:103D500004EB8303DB688BB11A685A6000232C4A9A
:103D60000393049305930C2009F1FF3300FB032018
:103D700003A9284B984703A8274B9847942303FB94
:103D800005733C3304EB4303FF221A71234A12F8F4
:103D9000091021F0010102F8091093F80590B9F11A
:103DA000FF0F904618D04A2303FB059304EB8303CF
:103DB000DB688BB11A685A600023154A0393049399
:103DC00005930C2009F1FF3300FB032003A9114BDD
:103DD000984703A8104B9847942303FB057504EB01
:103DE0004505FF2385F87D3018F8093023F00103DD
:103DF00008F8093001A80A4B9847304607B0BDE8DB
:103E0000F0830026F9E700BFD0280020CD3300085A
:103E10005028002095330008013D0008D8080020F4
:103E20005517000808B54068014B9847002008BDA9
:103E3000153D0008426838B50B4644318A420446B5
:103E400008D0521A064D9010454303D01846054D30
:103E5000A84703466268443A6260184638BD00BF0E
:103E6000F1F0F0F0E50103082DE9F04F87B00F29DC
:103E70008246914600936FDC384B4FF4947202FBFC
:103E80000032019292F8A220052A65D1942202FB09
:103E9000001103EB410191F87C80B8F1FF0F5BD07A
:103EA0004A2606FB008603EB8603DC6804B304A8FD
:103EB0002B4B98470024DDF800B003962546009B65
:103EC0009C4212D22549039B029101EB8303DB68DC
:103ED0000CCB9B1A432B01DD75B9154665B9012141
:103EE00001FA08F150461F4B984704A81E4B98470B
:103EF000204607B0BDE8F08F029B2E684FF4947700
:103F000007FB0A374744484697F84C10174B761A78
:103F10005E4528BF5E46043132462944984797F8EB
:103F20004C302A683344DBB2934287F84C30B144BA
:103F30003444ABEB060BC2D1029B039A03EB820322
:103F40000025D86887F84C500168094B98474146CE
:103F50000198084B9847B2E70024C9E7D028002011
:103F6000CD330008A935000855170008CF01030814
:103F7000353E0008E133000838B54068034D1C4663
:103F80001B68A8472060002038BD00BF693E0008BC
:103F90002DE9F7434FF494762B4D4643AC190F4669
:103FA000B4F8240110B36846284B98470FB3002299
:103FB000114640F2A223264D0B20A847002240F2D2
:103FC000A22311460C20A8474FF0A042D2F8043893
:103FD00023F00203C2F80438012384F8A2302046FB
:103FE0001C4B984768461C4B9847012003B0BDE81E
:103FF000F0834FF0A0421036D2F80438DFF85C802E
:1040000043F002033544C2F804380126274697F8E6
:10401000B4309E4213DA2B6873B1A31993F86C3055
:1040200053B1DFF83C90012231462046C04718B119
:1040300028680168C847F6E701360435E7E700233A
:1040400087F8A230CBE700BFD0280020CD3300088E
:10405000390F00085936000855170008513C000870
:10406000353E000873B50546002842D1224A234E4A
:10407000536B43F080034FF0A04453636846204BDA
:1040800098470223C4F804388023A3601D4BE360E3
:104090004FF41023A363D4F800381B4943F0030303
:1040A000C4F80038A36B43F400134FF47A72A3638F
:1040B000284600238847154B0121284698472A4661
:1040C00013494320B0472A4611492A20B0474FF0F0
:1040D000FF3363614FF48053A361C4F83458A3687D
:1040E00043F00103A36068460A4B9847012002B0E1
:1040F00070BD0020FBE700BF00380240CD1600086D
:10410000CD330008400C004031270008913F0008E3
:104110002D480008551700082DE9F04F4FF494730F
:10412000814E434389B016F803A00746BAF1000F49
:1041300002D14FF0000AEFE0012AFAD9022A40F03A
:10414000E080FF25794800222C4690F900305FFA84
:1041500083FE1EF0010F09D1FF2C0DD11EF0020FBE
:1041600000F0DE8043F00103037014460132042A9C
:1041700000F10100E9D10DE0FF2D07D11EF0040F81
:1041800004D043F0010303701546EFE7002CEDD097
:10419000002DEBD0FF2D05D1FF2CCAD0631E0E2BB6
:1041A00005D9C6E76B1E0E2BC3D8FF2CF6D14FF4F2
:1041B000947909FB07694B461022FF2D07D093F82D
:1041C0007C00A842B5D093F87D00A842B1D0FF2C66
:1041D00007D093F87C00A042ABD093F87D00A042BA
:1041E000A7D0013A03F10203E7D194200A60784393
:1041F0000B680F2B0EDCC2183C3206EB420292F821
:1042000004E0BEF1FF0F02D15279FF2A04D001333E
:104210000B60EDE7102B8CD094207843034406EB21
:104220004303EAB283F87C200B68184406EB400095
:104230003F4B80F87D405B68598803F116060B44BC
:104240000193B9F82431002E59D001998E4256D2EB
:104250007178052953D13178072950D1B078802859
:104260003FD164F07F013048B1704FF4947101FB8D
:1042700007012144012081F86C00A046B8F1000F2D
:104280002CD002932B4B039208F1FF3B0C2101FB36
:104290000B3B0021059106910791584605A9264B35
:1042A0009847264B05A89847DFF87CE0029B039AC5
:1042B0004A2101FB07810EEB8101C1F80CB0F078B7
:1042C0004FEA480100F0030088404FF4947101FB6D
:1042D00007E18844B18888F85C10034331780E44C4
:1042E000B1E70028FAD1DFF840E0B2704FF49471E2
:1042F00001FB07E12944A84681F86C00BEE7A9F854
:104300002431094A4FF4947303FB07235B78FF2B96
:1043100002D138460A4B9847504609B0BDE8F08FA5
:10432000FF2D7FF435AF29E7D0280020D8080020E2
:10433000282800205028002095330008013D00085F
:104340006540000813B5064B40680C4601A9984724
:1043500020B1019B2360002002B010BD0620FBE7C6
:104360001941000838B50546074C2A20A0474320CC
:10437000A04700212846054B9847054A536B23F078
:1043800080035363012038BDF9160008913F0008EF
:104390000038024013B50B4B044668469847204648
:1043A000094B98474FF494736343084A0849002027
:1043B000D054084A002388476846074B9847012095
:1043C00002B010BDCD33000865430008D02800209E
:1043D00031270008A08601005517000808B540687D
:1043E000014B9847002008BD954300082DE9F04196
:1043F0000A4FDFF830800A4E00247B69A3420AD9B5
:104400000025294620460135C047102DF9D1204608
:10441000B0470134F1E7BDE8F08100BF7828002003
:1044200095430008153D00082DE9F8434FEA42186E
:1044300000EB08031546D3F80829D20748BF01222C
:1044400000EB080748BFC3F80829D7F80039002B4C
:1044500006460C4610DB8DB9D1F8B83033B10846AA
:104460009847D4F89C3094F8A01093BBD7F8003943
:1044700043F00063C7F80039BDE8F88301EB85031A
:10448000DB68002BF2D04B1993F86C90B9F1000F58
:10449000ECD0012229462046144B98470028E5D04D
:1044A0000168031DB04441F40022C8F81029D7F870
:1044B000002942F00442C7F800296A1C06EB0236C4
:1044C0001A46881A1844002805DD52F8040B30609B
:1044D000F7E7A946E6E7B9F1000FCDD004EB850474
:1044E000034BE06801689847BDE8F883513C000839
:1044F000353E00082DE9F041214B044608460D46A3
:1045000098470228074635D003280FD0012815D137
:10451000D4F8003943F40013C4F80039D4F8003B50
:1045200043F40013C4F8003BBDE8F081D4F8003830
:1045300095F8A12043EA0213C4F80038114E002276
:1045400029462046B047052F374617D105F11008F8
:10455000012695F8B430B34210DD58F8043B3BB166
:10456000AB1993F86C301BB1324629462046B84748
:104570000136EEE70023C5F8B830DFE7BDE8F0818B
:10458000F53B00082944000870B454010519D5F81A
:10459000083BDE0744BF0126C5F8086B1B0742BF76
:1045A00003190825C3F8085B82B991F8A33043F0DA
:1045B000C04343F40023C0F8103BD0F8003B43F065
:1045C0000443C0F8003B70BC084B1847114420441A
:1045D00091F85C3043F40023C0F8103BD0F8003B66
:1045E00043F00443C0F8003B70BC7047F54400083A
:1045F0002DE9F84390E81800E41AA3101C4C5C4322
:1046000014BF23460123E41807468846194B01D2FC
:104610009C4229D91C4644206043174B98470646C4
:10462000D7F800907D68A5EB0905701903D04422E6
:104630004146124B98470E4AAB105A4304D02A46C3
:10464000494630460E4B984744353544B9F1000F82
:1046500002D048460B4B9847442303FB04643E605A
:104660007D60BC60BDE8F883002CD4D12646D7E736
:10467000F1F0F0F0C3C3C303294B0008CF010308D6
:10468000E5010308394B000838B582684368934256
:10469000044608D023B118464422044DA8470346D7
:1046A0004433636038BD024B984738BDCF010308DF
:1046B000F1450008F0B500EB810493B005460E46C5
:1046C000E068084B01A917469847E3685C68002337
:1046D0003B700121B140A878034B9847443C2046E9
:1046E00013B0F0BD894600086535000873B505466E
:1046F0001E46084614468AB901F1C402C1F89C203E
:1047000080F8A030013405EB04341146731A1344C9
:10471000002B0BDD236841F8043BF7E70DF107029E
:104720002146034B9847021D0660EBE702B070BDBF
:10473000B54600082DE9F743324B334F1B6804465A
:104740000E4698476846314B9847656915F0100842
:104750000ED0226A02F4B013B3F5802F06D1C2F353
:104760000A13314602F00F022046B8476569EDE7AB
:104770006A030FD5D4F81878DFF8A890BFB24FB10C
:10478000FB0703D5424631462046C84708F10108D9
:104790007F08F4E7280311D5D4F81878DFF888905B
:1047A0003F0C4FF000084FB1F90703D542463146A0
:1047B0002046C84708F101087F08F4E7EA040FD54E
:1047C000134B3146204698474FF480536361114B99
:1047D0001B6898476846104B984703B0BDE8F083C4
:1047E0002B0506D50D4B3146204698474FF4006304
:1047F0006361002DEBDA0A4B3146204698474FF0B3
:104800000043E3E76C140020ED460008CD330008B8
:10481000D93600086814002055170008A136000892
:10482000B936000829440008894500080249034BAD
:104830004FF0A040184700BFD0280020354700089F
:104840002DE9F7430E460446002837D090F8B430DF
:104850008B4233DD04EB86076846194B9847FD68A9
:104860002DB3A31993F86C500DB3D4F8B03033F8CE
:104870001630DB070CD5DFF85C90DFF85C80012296
:1048800031462046C84790B1F8680168C047F6E74E
:1048900068460C4B984720B121464FF0A0400A4B88
:1048A0009847324621464FF0A040084B984768464B
:1048B000074B9847284603B0BDE8F0830025F9E789
:1048C000CD330008151700083547000829440008B3
:1048D00055170008513C0008353E00080F292DE906
:1048E000F04738DC274C4FF4947505FB004595F8EC
:1048F000A220052A02D00120BDE8F087942202FB05
:10490000001104EB410191F87D60FF2E23D04A2273
:1049100002FB0060023004EB8004606878B390E82A
:104920000C009B1A184ADFF868809B1002FB03F901
:104930001E27636893E80600521A432A0EDD002FF3
:104940000FDC5960D7E76422002300200F49884715
:10495000013FD146EDE70020BDE8F087002FCADC1B
:10496000EFE731462846C04762680CCA9B1A064AE0
:104970009B1002FB03FAD145E5D01E27E9E7BDE80D
:10498000F08700BFD0280020F1F0F0F0B526000835
:104990004148000808B54068014B9847002008BD11
:1049A000DD4800082DE9F04F99B00F298046924666
:1049B000019300F39580002B00F09080002A00F016
:1049C0008F80494E4FF4947303FB0063029393F876
:1049D000A230052B40F08480942303FB001106EBEA
:1049E000410191F87D70FF2F7AD04FF04A0B0BFBFD
:1049F000007B0BF1020B06EB8B0BDBF80430002B7A
:104A00006ED005A8394B98470025DDF80490CDF805
:104A10000CB02C46039B07A95868354B9847039B5D
:104A20005B68D3F804B0BBF1440F21D04FF494730A
:104A300003FB08633B4493F85C504D4528BF4D464B
:104A40002DB12A465146ABF140002A4B98474FF40E
:104A5000947303FB0863DA19A9EB050992F85C204B
:104A60004BF8445CAA42AA442C442ED80025D1E736
:104A70000135642D0BD9019A4A4501D11A685A6053
:104A800005A81D4B9847204619B0BDE8F08F05A832
:104A90001A4B984783460028F2D14FF4947303FBD6
:104AA000086393F8A230052BEAD139460298144BDB
:104AB000984705A8134B98475846322200231249BD
:104AC000884705A8114B9847A4E793F8A230052B17
:104AD000D6D1394602980A4B9847D1E7019CD2E7D4
:104AE0004FF0FF34CFE700BFD0280020CD330008BF
:104AF00089460008CF01030855170008151700085C
:104B00004148000823170008B5260008411700088F
:104B100038B54068034D1C461B68A847206000203C
:104B200038BD00BFA5490008004B1847E94B0008F5
:104B3000004B1847E94B0008004B1847854B00080D
:104B4000004B1847854B00080148024B011D1847D0
:104B5000042A00202D4C0008074B5B685BB150B164
:104B600010F8183C202B02D00120044B18470121DB
:104B70001838034B18477047042A0020154C0008CA
:104B80000D720008004B1847594B0008114B37B500
:104B90005C680546B4B902A90F4B41F8044D68465C
:104BA00000949847019B9D4205D901200B4B9847E3
:104BB000204603B030BD0A4B00981C6825441D6098
:104BC0002044F6E741F00401064B98470028F0D056
:104BD0001830EEE7042A00202D4C0008154C000880
:104BE000002A0020A57100080021014B184700BFD2
:104BF0008D4B000838B5054B05469847044618B15B
:104C00002A460021024B9847204638BD8D4B0008AC
:104C10001902030882B000230193019B1BB9019B79
:104C2000019A1344F8E702B070470000034B1A687A
:104C30005B68026004339B1A0B6070473C0A0020DB
:104C400007B5002301933223ADF8043001238DF81A
:104C500007300198034B98470348044B03B05DF8B5
:104C600004EB1847D16F000808100308E15D000845
:104C70002DE9F04305460D480D4B04680679477948
:104C800090F8068090F8079085B0204698470194E8
:104C90000290CDF80090284643463A463146054CEE
:104CA000A047012005B0BDE8F08300BF340A002012
:104CB000B55B0008599D000837B5CDE90023134BBB
:104CC00005460C469847E0B9EDB1E4B1104B1149E7
:104CD0001D60114B1C60DDE90023C1E900230F4B6F
:104CE0009DF800205D620E4B1A719DF801205A71EB
:104CF0009DF802209A719DF803201C60DA7103B0C0
:104D000030BD0820FBE70220F9E700BF255F00085F
:104D10000C2A0020102A0020182A00203C0A00201B
:104D2000340A002070B5ADF5007D134605460A46ED
:104D3000194C4FF400716846A04705F47F43B3F562
:104D4000A06F044616D0B3F5C06F09D00246002309
:104D500028466946114DA84720460DF5007D70BDD7
:104D60000F4B1B68002BF7D000220DF8002068467F
:104D70009847F1E70B4B98470B49C369984706469C
:104D80000028E9D00025A542E6DAB3696946304635
:104D900098470135F7E700BF190603087D8B000827
:104DA0001C2A002075910008030000402DE9F84FEF
:104DB000D1E90067344B354CDFF8DCB081468846DA
:104DC0003046924639460022A047D84704460D4651
:104DD00030463946D8472E4E0A220023B047052ACE
:104DE00073F10003B34627DB013445F10005264685
:104DF0002F460A22002330463946D847134317D19D
:104E0000012E77F1000317DB304639460A220023D2
:104E1000D847002908BF012806460F46E9D1DAF82D
:104E20000030002B22D007DD013BCAF8003003E040
:104E3000002F08BF012EF2D00A2200232046294667
:104E4000D847134309D10023204629460A22D847D0
:104E500004460D4654EA0503EED1204629460D4B83
:104E60009847C8E900010020BDE8F88FD9E9002380
:104E7000013243F10003C9E9002300220023C8E9FD
:104E800000230120BDE8F88F0000244019F8020833
:104E900055FC020869F5020825FD02082DE9F04FCE
:104EA00099460C46034685B02343CDE9000193465D
:104EB00054D02D4F012400250A26002908BF0A28B6
:104EC00008D300230A22B84706FB05F3A4FB0645D6
:104ED0001D44F2E7D9F8003003939B453EDADFF832
:104EE0008880012600274FF0000AD3450FDD0A22F3
:104EF000002320462946C0470A230A227B43A6FBFB
:104F0000026704460D460AF1010A1F44EDE72246F6
:104F10002B46DDE90001C0470A22002304460D4666
:104F2000C047002B08BF052A02D30A3445F100050B
:104F30000A21A6FB012301FB07339D4208BF9442CF
:104F400005D303990131C9F8001014461D460A2201
:104F5000002320462946C047CDE90001DDE90001D4
:104F600005B0BDE8F08F00BFF5FC02082DE9F04167
:104F7000904606461A460F465C1E002140460D4BE1
:104F80000D4D984756EA070310D0304639460A229D
:104F90000023A847013C303208F804203046394647
:104FA0000A220023A84706460F46EBE72046BDE845
:104FB000F08100BF19020308F5FC02080CB413B518
:104FC00004AB054C53F8042B0193A04702B0BDE895
:104FD000104002B0704700BF190603082DE9F04FDA
:104FE000A1B01F469DF8AC809DF8B030039001251C
:104FF000B8F1470F049116462A9C0193069509D0F3
:10500000A8F167014B424B41B8F1580F059302D10B
:10501000029505E00595A8F17802534253410293A9
:105020009B4B6322002107A89847029B2BBB019B47
:1050300033B1002E77F1000322DA764267EB47079F
:10504000304639464FF0010900234FF0010A4FF076
:10505000000B002908BF0A284A4609F1010911D3AB
:105060000A2200238B4DA8470A230A2203FB0BF3D5
:10507000AAFB02AB9B440123EBE700230193DFE78C
:10508000029BFBE703B10692059B002B00F0948086
:10509000069DB8F1470F0CBF45236523A542059334
:1050A0001EDCDFF8F08100240DF11C09AC4266DA49
:1050B00052465B4630463946C047303004F8090056
:1050C00052465B4630463946C0475046594616461A
:1050D0001F460A220023C047013482468B46E5E77B
:1050E000304639466C4DDFF8AC8106AB2246A84706
:1050F000012681468A4600270A25002908BF0A287A
:1051000045D200254FF02E0BAC4238DD20ABEB181A
:105110003246029348463B46514605F101085D4D33
:10512000A847029B303003F8640C32463B464846A1
:105130005146A847304691469A46394600230A22EE
:10514000A84759EA0A0306460F4629D120AB9844DE
:10515000029A9DF8143008F8643C2B2302F8623C54
:10516000069B029C5A1E0A2192FBF1F303F13000C8
:1051700001FB1323303304F8610C04F8603C07ABE7
:10518000464A47490198002818BF0A4665E00023AF
:105190000A22C04705FB07F3A6FB05671F44ACE7DF
:1051A0004445D3D0B8F1010F04D18DF81DB00134BE
:1051B0004FF002084546A7E7029BE3B9DFF8D4A009
:1051C00062250DF11C09002F08BF0A2E05F1FF33DF
:1051D0004AD31D46304639460A220023D047303292
:1051E00009F80520304639460A220023D047013C01
:1051F00006460F46E7E7B8F1580F0CBF4620662079
:10520000002C08BF0124622107AB0F3856EA0702C1
:1052100008D1081B224618443025002A17DD013A20
:105220008554FAE706F00F02092A88BF121801F127
:10523000FF3194BF3032D2B25A54320942EA077277
:105240003D09002C16462F46E0DD013CDEE7002C30
:10525000ACBF0C1B0C46114A234404990398114C13
:10526000A04721B0BDE8F08F20AA1A44303602F8DA
:10527000646C641B3022E118002906DDB8F1440F8C
:1052800003D1013B09F80320F5E74B4478E700BF61
:1052900019020308F5FC02089D4E00081C100308C3
:1052A0001B100308BD4F00082DE9F04FC5B0A24BFD
:1052B0000590901C5BEC10AB1646069198479F4CEE
:1052C0000790632230212BA8A0476322302112A827
:1052D000A047504600287BF100034FF00002B8BF02
:1052E0000BF100438DF8AC208DF84820BFBF52462B
:1052F0009B4692460123B4BF04930492904F5046BC
:105300005946B847731C04460D46073613F8012F5B
:10531000472A00F0C283672A00F0EB839E42F5D152
:10532000884E894B002250465946B0470646002811
:1053300028D1864BDFF82C92CDE90E452046294630
:1053400098470B46024659465046C847079B0D965C
:1053500082468B46CDE910AB002B40F0DD82002267
:105360007B4B7C4CA0470DAACDE910017A4B10A9CC
:105370000EA89847794A7A4904980E9B002818BFCE
:105380000A465CE065230993DFF8FC91704DDFF875
:10539000FC810026002422462B4650465946C84729
:1053A00040B15046594622462B46C04701368246F8
:1053B0008B46F0E750465946B847644B694C6A4FF4
:1053C000984702460B4650465946A0470022002304
:1053D00004460D46B84710B105F100431D4650A3E1
:1053E000D3E90023204629465A4CA0475F4B604C26
:1053F000984712AA6323A047594604465D4B50467E
:105400009847099B019312AB1C44009403460296F3
:10541000594A06990598594CA04745B0BDE8F08F08
:10542000079B9C4210DA4D4A049B4D4C5046002B82
:1054300008BF144659464F4B9847224603460699E3
:1054400005984E4CA047E8E737A3D3E90023504620
:105450005946454D4FF00104A84700B90446E3B250
:105460000A93002B00F0D3803F4D454F394CD04676
:10547000D94600260022434B40464946A84700280B
:1054800000F0C8800022002340464946B847002863
:1054900040F0C0804046494600222D4BA0470136CF
:1054A00080468946E6E7079B089A284F9A42244B94
:1054B00002DA032E40F34481404649469847CDE93D
:1054C0000E01B847274C02460B4640464946A047C6
:1054D00080468946CDE91089002401220D94274693
:1054E00023460B920B9A07998A4251DA10A3D3E90B
:1054F0000023404649461C4DA84708B10137012406
:10550000134B144D404649460022A8470B9B0133DC
:105510000B93804689460123E4E700BFAFF3008088
:1055200000A0D885573476432D431CEBE2361A3F52
:105530009A9999999999B93F8B0003081902030820
:1055400025FD0208E5FA02080000E04369F50208BB
:1055500000002440C5F50208AD4D00087110030895
:105560001F1003085DF20208A9FA020855FD02089F
:105570006D4F000825FB020869100308BD4F0008A5
:1055800095FA02080000F03FD1FA020819F8020863
:105590000BB1CDE9108904B10D97DDE910890D9C9F
:1055A00000270B948EA3D3E90023404649468E4D35
:1055B000A847002850D000220023404649468B4D82
:1055C0000134A84700283DD00FB10B9B0D9300225A
:1055D000874B884C40464946A047874BCDE9100190
:1055E0000DAA10A90EA898470A9B002B38D00E9B35
:1055F0000A2B35D100227E4B50465946A04776A350
:10560000D3E900237D4CA04750B300230A93D04632
:10561000D946002600237A4F0893784C744B002219
:1056200040464946A047044600283FF43CAF704B33
:10563000404649460022B847089B013380468946C8
:105640000893EAE7404649460022694B694DA8475E
:10565000012780468946A4E7002FB8D00D94B6E70D
:10566000DDE9108900220023404649465F4CA047EF
:10567000002838D10D9B622BC4BF62230D930D9F70
:10568000604B2BAC3A4630212046984744AB1F4430
:10569000002307F8643C40465B4B5C4F4946984703
:1056A000632312AAB8475A4F8EB1099B029312ABDB
:1056B0001844584A0E9B5849039601900094049848
:1056C000002818BF0A4606990598B847A5E6089B22
:1056D0000393099B029312AB1844019000940E9B14
:1056E0004E4A4F49EBE7DDE90E014E4C00230A28F4
:1056F00071F1000209DB0A220023A04706B1013E36
:10570000089B013308930123F1E70BB1CDE90E01AA
:105710003F4C6EB1099B444A4449009301960346AD
:105720000498002818BF0A4606990598A04774E611
:10573000089B0193099B00933D4A3E490346EFE7CE
:1057400050465946984780468946CDE90E89B84764
:10575000394E0B46024659465046B047B8F1010F44
:1057600006460F4679F10003CDE910670D94C0F2AB
:105770008480079B089ADFF874B0DFF86CA09D1A4C
:10578000013DA046A146002D5ADCB9F1000F01D021
:10579000CDE910670CB1CDF83480DDE910010022AD
:1057A000134B144C114EA0470DAACDE91001124B1A
:1057B00010A90EA89847DDE91045002200232046D5
:1057C0002946B04700287FD0DDE90E011B4B9847E2
:1057D00082468B467DE100BF2D431CEBE2361A3F2B
:1057E0009A9999999999B93FA9FA020895FA0208E4
:1057F00000002440C5F50208AD4D0008D1FA0208AA
:1058000019F802081902030855FD02086D4F000837
:10581000BD4F0008241003082310030834100308A8
:105820003310030855FC0208441003084310030812
:105830004F1003084E1003085DF2020869F50208D4
:105840000022002330463946D84700289DD1AAA31C
:10585000D3E9002330463946D04710B108F101089A
:10586000012430463946A64EA64B0022B047013DE2
:1058700006460F464FF0010985E7079DDFF8B4A201
:10588000DFF8A8B2A046A1460022002330463946E0
:10589000D04700287FF479AF97A3D3E9002330469F
:1058A0003946D84718B108F10108013501243046BE
:1058B0003946934E934B0022B047013D06460F46B2
:1058C0004FF00109E0D163E70D9B622BC4BF622357
:1058D0000D930D9E8C4B2BAF3246302138469847A6
:1058E00044AB1E44002306F8643C2046874B884C9A
:1058F00029469847632312AAA04712AB184485494A
:105900000190854A04980097002818BF0A460E9B0C
:1059100006990598814C09E7DFF8188200220023D8
:10592000C047D8B1079F784C622FA8BF62272BAB26
:105930003A4630211846A04744AA1744002207F8E7
:10594000642C009004987649764A0E9B734C00288C
:1059500018BF0A4606990598A0475EE5724B089065
:105960000446054606460993079B089A9A4219DAA7
:1059700061A3D3E90023504659466C4FB84708B19C
:10598000013501246A4B504659469847099B984770
:1059900002460B4650465946C84700220023C047DE
:1059A000002845D00EB1CDE910AB04B10D95DDE96D
:1059B00010010022534B524C5E4EA0470DAACDE978
:1059C00010015D4B10A90EA89847DDE91045002293
:1059D000002320462946B04780460028A2D1079FD1
:1059E000494B0D9EDFF860A1622FA8BF62270DF121
:1059F000AC093A4630214846984744AB1F442046FC
:105A000007F8648C29464A4B984701240746884684
:105A100000254FF00A0B0A2871F1000315DB002363
:105A20000A22D0470BFB05F3A4FB0B451D44F2E70C
:105A3000344B334E504659460022B047089B013341
:105A400082468B46089301268EE7DFF8FCB04E4471
:105A50000A2C75F100031CDB22462B4638464146D2
:105A6000D8473030307022462B4638464146D04722
:105A700020462946174698460A220023D047044666
:105A80000D4654EA050306F10106E1D1CDF8009078
:105A900058E707F130033370E5E745230993002207
:105AA000264B274E50465946B04700287FF46CAC31
:105AB00020461D4B234C2946984702460B4650462C
:105AC0005946A047002200231A4CA04700283FF463
:105AD000BBAC50465946164B1B4D984700240A282C
:105AE00071F10003FFF69CAC0A220023A8470134A1
:105AF000F5E76523D2E700BF9A9999999999B93F3B
:105B0000C5F50208000024401902030855FD0208EB
:105B10006D4F0008591003085A100308BD4F0008C4
:105B2000621003086310030869F50208A9FA020865
:105B300025FD020895FA0208AD4D00080000E0437B
:105B4000E5FA02085DF2020855FC020870B5084B40
:105B5000044610EE100A0D4616469847324641ECB0
:105B6000100B044B29462046BDE87040184700BF83
:105B70001DF50208A952000810B4024CA4465DF8B5
:105B8000044B60471906030838B50C46114638B176
:105B900031B12CB15D1CAC424FF0000402D2047054
:105BA000012038BDC4541A46014B9847204638BDE1
:105BB00069040308034613F8012B002AFBD1181AC5
:105BC0000138704738B50D460446114660B15AB1E8
:105BD00055B11046054B98470130854204D3204605
:105BE000034B9847002038BD012038BDB55B000845
:105BF0005904030810B510F8013BA3F14102192A1A
:105C00000AD911F8012BA2F14104192C06D90BB1C4
:105C10009342F0D0981A10BD2033F2E72032F6E715
:105C200070B5064B04469847256AA36A224601468A
:105C3000AC46606ABDE87040604700BF75910008DF
:105C40002DE9F84F91460E4601B3114B1B78EBB18D
:105C5000104BDFF844B0DFF844A093E82001A845DA
:105C600014D055F8044B23694B45F8D16068D847E8
:105C70003146074602466068D0470028EFD1F35D01
:105C80000BB15C2BEBD12046BDE8F88F0024FAE77E
:105C9000342A0020442B0020B55B0008B101030822
:105CA0000846014B184700BFE94B00080846014B66
:105CB000184700BF854B000838B50C680D4664B125
:105CC0002046074B984710B12046064B9847204680
:105CD000054B98470020286038BD022038BD00BF22
:105CE000879000087D8E0008854B00080120014B3D
:105CF000184700BFC5B500080420014B184700BF76
:105D0000C5B50008F8B516461F460D4651B1084600
:105D1000054B984720B932463B46284603498847F9
:105D20000020F8BD0220F8BD87900008098E000809
:105D30002DE9F041804617461E460D46B1B1302090
:105D40000D4B98470446A0B10562C0F824808762D5
:105D50000A4D4EB10123037622460949A847069B06
:105D600000201C60BDE8F0810676F5E70220BDE862
:105D7000F0811520BDE8F081E94B0008E9900008AA
:105D8000215C000808B1014B18477047394B0008E7
:105D9000036853F82130F0B58BB11C68176862684E
:105DA00097420CD0226862B1566845682346144673
:105DB000B6FBF5F205FB12629142F0D000231846C3
:105DC000F0BD1346FBE70000024B03491B68034884
:105DD0009B6818478C2A0020F55E0008B55E000815
:105DE0000FB470B5C2B046ABFF2153F8042B01933A
:105DF00002A80A4C0A4DA0470A4C0646A068A847CC
:105E00003246002302A9A068074EB047A068A84701
:105E100042B0BDE8704004B0704700BF795B000835
:105E2000218C00083C0A00207D8B00080FB407B5C8
:105E300004AA064B52F8041B019240F20150984705
:105E400003B05DF804EB04B0704700BF254D0008B7
:105E5000034A52F82030013342F82030704700BF27
:105E6000202A0020034A52F82030013B42F820301B
:105E7000704700BF202A0020034B53F82000002861
:105E8000D4BF002001207047202A002013B5064B04
:105E90000446684698472046044B98476846044B9A
:105EA000984702B010BD00BF09750108515E000897
:105EB0004175010810B5044C0120A047234602207B
:105EC000BDE81040184700BF8D5E000813B5064BB3
:105ED0000446684698472046044B98476846044B5A
:105EE000984702B010BD00BF09750108655E000843
:105EF0004175010810B5044C0220A047234601203B
:105F0000BDE81040184700BFCD5E000810B5034B38
:105F100098470349C369BDE81040184775910008C8
:105F200004000040014B1878704700BF342A00205D
:105F3000014B1878704700BF002B0020014B1878E8
:105F4000704700BF640A002041B14B69934205D9F4
:105F5000012B886903D050F8220070470020704759
:105F600070B516461C461A46054B0546984723460B
:105F7000044C32460146A4462846BDE870406047BE
:105F8000415C0008495F00082DE9F8430C46804653
:105F90005C212046164B914698470646E8B1071B00
:105FA000781C144B9847054618B900242046BDE8D4
:105FB000F8833A462146104B104C98470023EB5586
:105FC000701C0F4B98474B46024629464046A04757
:105FD0000C4B044628469847E8E70B4B4A462146B7
:105FE000404698474369012BDFD18469DEE700BF53
:105FF00029040308E94B0008CF010308615F00088A
:106000008B000308854B0008415C00082DE9F74F21
:106010008DE80C004A4B1E7882468946002E40F0DF
:106020008A80002800F08780002900F08480002A00
:1060300000F08180019B002B7DD0424BDFF8348142
:1060400098474FF00053324651468346C0473E4B77
:106050000446324649465846C0473C4B00993246B2
:1060600005465846C0473A4B0199074632465846BE
:10607000C047002C5FD0002D5DD0002F5BD00028E2
:1060800059D0A368002B58D0E368002B55D0236962
:10609000002B52D06369002B4FD0A369002B4CD04A
:1060A000E369002B49D0236A002B46D0AB68002B54
:1060B00043D0EB68002B40D02B69002B3DD06B699F
:1060C000002B3AD0AB69002B37D0EB69002B34D0D2
:1060D0003B69002B31D07B69002B2ED08368002BCD
:1060E0002BD0C368002B28D0036933B3436923B393
:1060F000836913B3C36903B3436AF3B1036AE3B1BA
:10610000836AD3B1C36AC3B1124B009AC3F800A02B
:10611000114BC3F80090114B1A60114B019A1A6091
:10612000104B1C60104B1D60104B1F60104B186013
:1061300003B0BDE8F08F0820FAE70220F8E700BFBF
:10614000342A002075910008010000200200002080
:1061500003000020842A0020782A0020DC2A002066
:10616000D82A0020902A00208C2A0020882A00208B
:106170007C2A0020495F0008014B1868704700BF67
:10618000902A0020014B1868704700BF8C2A00201D
:10619000014B1868704700BF882A0020014B18681F
:1061A000704700BF7C2A0020014B1868704700BF71
:1061B000802A0020014B1868704700BF582A002031
:1061C000074A13683BB9074B1B7833B91060084482
:1061D000506018467047042070470820704700BF81
:1061E0003C0A0020342A0020F8B5234B1B780446D3
:1061F0000E46002B37D1002837D08369002B36D0CC
:106200004369002B33D08B4231D907691B4B9F4226
:106210001BD001339F422CD1194B01F20125984725
:1062200021463B463246174CA047174C036B174993
:106230002060984720681649436B9847154B00200B
:106240009D605D619D61DD61F8BD0D4B01F2011541
:10625000984721463B4632460A4CA0470E4A836A7D
:1062600010600E49E9E70820F8BD0220F8BD0120C2
:10627000F8BD0420F8BD00BF002B0020080000403E
:1062800075910008495F0008582A0020F95C000851
:106290004D6D00083C0A0020802A0020ED5C0008BB
:1062A000F8B58468084F054624B126682046B847EB
:1062B0003446F9E76A682868044B920021469847FB
:1062C000EC60AC60F8BD00BF394B00081902030850
:1062D000034653F8180B984201D0014B18477047FA
:1062E000394B0008F0B52A4B2A4D2B4F89B09847FF
:1062F0002A4B002418685C601C609C60A8472046FC
:10630000A8472146264B1C2201A8984703940694CF
:10631000244C012307AE0293A06801964FF07E53F0
:10632000059318B10568B8472846FAE71D481E4D81
:10633000A84705AA92E80300019A1C4BB24283E8E1
:10634000030001BF08332360079BA361039B18BFB1
:1063500022600499029A6260A360E16043B15968C7
:10636000B1FBF2F302FB13132268114942F8231028
:10637000002301220693029207930393049301A83A
:106380000C4B0196984701A8A84709B0F0BD00BF83
:1063900015880008855D0008394B0008442B002053
:1063A000190203085C2A0020D16200086C2A002030
:1063B000642A0020A162000807B5124B9847124BCF
:1063C0009847124B9847124B9847124B9847124BDD
:1063D000984701A96846114B9847019A0098104BBD
:1063E000002198470F4B98470F4B98470F4B984702
:1063F0000F4B98470F4B98470F4B984703B05DF8EA
:1064000004FB00BF91900008858C00081110020861
:106410007DB50008C95D0008DD7401082D4C000839
:1064200019020308494B00084DF90108BD0802088C
:1064300069DA000875950008E562000870B5124B2E
:10644000124C134D9847134B98471348A047134BD2
:106450002846596AA0472846114D1249A0472846A8
:106460001149A04728461149A0470121104B4EF67B
:106470006020984701210F4B0220984701210846D0
:106480000D4BBDE870401847C10E02082D5E000894
:1064900076100308B9630008741003083C0A002052
:1064A000961003087E1003088A100308A010030842
:1064B000A16D0008A56D00089D6D000810B50D4B7D
:1064C00098470D4B98470D4B98470D4B98470D4BF0
:1064D00098680D4B98470D4B1B68DB6898470C4B31
:1064E00098470C4B98470C4B98470C4BBDE8104015
:1064F000184700BFE5620008C308020855F9010803
:10650000C97401083C0A0020498B00088C2A00202D
:10651000B1B500082110020845910008E18F00087C
:106520002DE9F84390E81800E41AA41014BF23469C
:106530000123E4180646894602D2B4F1804F22D3E3
:106540006FF04044A000124B98470746D6F80080F1
:106550007568D9F80030A5EB0805EF4218BF7B51EC
:10656000AB0804D02A46414638460A4B98470435C2
:106570003D444046084B07EB8404984737607560FC
:10658000B460BDE8F883002CDCD12746DEE700BF0D
:10659000294B0008E5010308855D00082DE9F04F4F
:1065A00085B00D46039100293FD0D1F804A0BAF17F
:1065B000000F3AD00B68002B37D08B69002B34D0FA
:1065C0001D4B1B78002B32D01C4E1D4B7468376856
:1065D000A4EB07094FEAA9094FF00008C84516D0F7
:1065E000029757F804BB01935146DBF80400984723
:1065F000019B029A40B9DBF810102B69994218D11F
:10660000156005B0BDE8F08F08F10108E6E7B36852
:106610009C4205D004B12560043474600020F0E78A
:1066200003A90648074B9847F8E70220E9E7082046
:10663000E7E70F20E5E700BF342A0020442B0020C5
:106640004504030821650008436810B50C680A4634
:10665000B4FBF3F103FB1141034B984708B1006809
:1066600000B9002010BD00BF915D000807B5084BC0
:1066700001911B781BB9002003B05DF804FB01A950
:106680000448054B98470028F5D08068F4E700BF20
:10669000342A00205C2A00204966000870B5054BAA
:1066A0000D46044698472A460146034B2046BDE85E
:1066B000704018476D660008895F0008F8B5044609
:1066C0004B6840682568B3FBF0F200FB123355F8C5
:1066D000236032461768B94223D1964223D10F680E
:1066E0004FB1D7F804E0BEFBF0F600FB16E08342A2
:1066F0000CD045F8202055F8236004F108008642AC
:106700004FF0000008BFA76045F823000B68136036
:1067100008460B4B0D689847E368013BE360284649
:10672000F8BD3A46D6E70E68002EEFD07768B7FB83
:10673000F0F600FB1670834218BF45F82020E5E70D
:10674000394B000870B50C4600294AD0284D2A68FC
:106750006968881A0011002813462CDD1268A242CD
:1067600003D05A68A24217D1043399422ED051F86F
:10677000040C1A68186041F8042D1E4869601E4B0D
:1067800004F110019847054620B1616880681B4BF1
:10679000984740B3002070BD9A68A24201D10833E7
:1067A000E3E703F1100252F8046CA64201D10C3366
:1067B000DBE70138CFE78A1A9210022A0CD0032AAD
:1067C00006D0012A02D11A689442CED0052070BDAD
:1067D0001A68A242C9D004331A689442C5D004335F
:1067E000F1E7022070BD2946054B02489847D1E7E2
:1067F000442B00205C2A0020496600084504030859
:10680000BD6600082DE9F04385B01F4601230093C3
:10681000C368394E04460D46904600F110014268A7
:1068200002A8B0479DF80830002B42D0039D012DEF
:106830001FD12646002346F8183FA6460020A3682D
:106840004EF8080F63B35968B1FBF5F205FB12125D
:10685000D3F800C056F82210D9B9A1681960A36016
:1068600046F822E0196809B146F820306346104620
:10687000E8E7B5F1804F01D3204B98474FEA8509EF
:1068800048461F4B98474A4600211E4B06469847EC
:10689000D3E70968196056F8222013600246E5E73D
:1068A000194B20469847B8FBF5F36560266005FB59
:1068B0001385236853F82520AE005AB112683A6058
:1068C00053F825301F60E36838460133E36005B0B4
:1068D000BDE8F083A2683A60A76042B13A68616897
:1068E0005068B0FBF1F201FB120243F8227004F190
:1068F00008029A51E7E700BF05970208B19702081E
:10690000294B000819020308D162000873B5164626
:106910000191002A2ED0184B1B7813B9082002B021
:1069200070BD0C460A46154B314698470028F5D0F5
:1069300013484368B4FBF3F503FB154501AA294648
:10694000104B984708B1006880B90F4B0C2098474E
:10695000034608B1002202601A1D1EBF00225C60BF
:106960009A60294622460648084CA047083006602F
:106970000020D4E70220D2E7342A0020415C00083E
:106980005C2A0020915D0008294B0008056800087A
:10699000234B2DE9F0474FF0010983F80090214B7C
:1069A000214DDFF8A8A0DFF8A880204F204E98479F
:1069B000204B19680446A8471F4B20461968A84772
:1069C0001E4B20461968A8471D4B20461968A8474A
:1069D00051462046A84741462046A847394620460A
:1069E000A84731462046A847164DDAF80420494604
:1069F0002046A847D8F8042002212046A8477A68F4
:106A000003212046A847726800212046A8470E4B64
:106A10001B681BB12046BDE8F0471847BDE8F0876A
:106A2000640A0020759100089D650008B82A0020BE
:106A3000982A0020842A0020782A0020DC2A0020BE
:106A4000D82A00200D690008502B0020382A002089
:106A5000E02A0020554B2DE9F0411C788846002C97
:106A600040F0A180524A1268002A00F09C80514AEE
:106A70001268002A00F097804F4A1268002A00F03E
:106A800092804E4A1268002A00F08D804C4A1268AB
:106A9000002A00F0888001251D704A4B4A4E18607C
:106AA0004A4B98474A4B4B4999604B49D9604B49EF
:106AB00019614B4959614B4999614B49D9614B491E
:106AC00019624B494B4A59624B4999624B4956608E
:106AD00000270026D9624A491160C2E9026783E8AB
:106AE0001400156155619361464ADFF864E1464B35
:106AF000C2F808E0DFF85CE1C2F80CE0DFF858E12A
:106B0000C3F804E082E818009A614FF0020E3F4A91
:106B1000C3F810E0DFF844E11960C3E902675D6182
:106B2000C2F808E03A4BDFF838E1C2F80CE0DFF8D1
:106B300034E182E81800C2F810E0DFF82CE19A6135
:106B4000C3F804E0334A5D614FF0030EC3F810E070
:106B5000C3E902678260304AC260304A0261304A4B
:106B60004261304A8261304AC261304A1960026231
:106B70002F4B304A4262304A80E8180019605A6050
:106B800098611C61C3E902675D612C4B98472C4BEF
:106B900098472C4B83F800802B4B1D702B4B98474C
:106BA0002046BDE8F0810820BDE8F081342A0020AD
:106BB000902A00208C2A0020882A00207C2A00208D
:106BC0003C0A0020502B0020A910030875910008F2
:106BD000042B0020C189000889870008DD8800088F
:106BE00081750008E97500080D7600081B7600081D
:106BF00099760008382A0020257700088577000854
:106C0000990C0308342B0020E02A0020542B00208C
:106C1000B82A00209D65000845670008415C00080F
:106C2000895F0008615F00089D6600080D69000823
:106C3000982A00206D660008531103083D6400087F
:106C400091690008640A0020002B0020414C0008D4
:106C5000A15C0008AD5C0008E3100308315D00088A
:106C6000B95C0008055D00081C11030808B5064B57
:106C70009847064A106028B183689847B0FA80F0B8
:106C8000400908BD0620F9E7B5610008682B00201F
:106C900008B5054B186828B1C3689847B0FA80F06A
:106CA000400908BD0620F9E7682B0020064908685E
:106CB00008B538B10369022204319847B0FA80F070
:106CC000400908BD0620F9E7682B002008B5064BEF
:106CD000186830B1426959689047B0FA80F04009AD
:106CE00008BD0620F9E700BF682B002013B501910D
:106CF00005490246086818B18469496801ABA04794
:106D0000019802B010BD00BF682B002013B501919F
:106D100005490246086818B1C469496801ABA04733
:106D2000019802B010BD00BF682B002008B5064BCB
:106D3000186830B1026A59689047B0FA80F040098B
:106D400008BD0620F9E700BF682B00200F4809683E
:106D500038B500F1140450F8045B41F8045BA0421C
:106D6000F9D1008808800A49126801F1300051F811
:106D7000044B42F8044B8142F9D10988118018680C
:106D80000449054B9822984738BD00BF8911030874
:106D90009F110308D1110308CF0103080020704799
:106DA000002070470020704770B5074D074C084918
:106DB0002846A04707492846A047284623460649B3
:106DC000BDE87040184700BF042B0020C1890008AF
:106DD000582E0308D0170308142203082DE9F04F9A
:106DE0006A4D87B006AB286800220292039243F8EE
:106DF000082D046A03AA02A9A047002840F0C18018
:106E0000049B002B00F0BD80029A1468039AA146EF
:106E100002EB83039A4203D052F8041B8944F9E73A
:106E20002F7957B901217C20594B984706460028F5
:106E30004FD07C223946574B9847DFF88CA14C4500
:106E400008D22B796BB92868334607697C22214622
:106E5000B84738B12C7914B930464F4B98470020C9
:106E600091E0264630467C34D04718BB029B049FF5
:106E70001B68DDF80CE0B84231DA5EF82010A3425E
:106E800003EB010228D8944226D201911C46019BB3
:106E90001C44A145DED92B7923BB286833460769FA
:106EA0007C222146B8470028D4D130467C34D047D4
:106EB0000028CFD0736E033323F003082B799BB9DE
:106EC0000C214046354B9847074670B93046324B47
:106ED00098474FF07A4056E013460130CBE7A34283
:106EE000D5D0B7E72646E0E700272B797C3CA3B94D
:106EF00028683B46D0F810B042462146D8470028C3
:106F0000A8D13846264B4444984740B92B79002BEA
:106F1000A0D13846204B98479CE72746F1E7214807
:106F2000DFF8A880C04705A938461F4B98470028BE
:106F3000ECDB059BD8691D4B98478346B8B1059B90
:106F40009A695169426891420FD01948C047059B20
:106F50001848D969C0471848C047059BDBF804109A
:106F60009B6916485A69C047D0E782681A62144B79
:106F7000059914489847059A536943F008035361EB
:106F80005DE74FF07F4007B0BDE8F08FD0330020C1
:106F90008D4B000819020308594B0008F54B0008F7
:106FA000311A020815130308E11B0208558700086F
:106FB000B85E0308301303087C130308D3130308D7
:106FC000552D020880300020D5190208754A0108A5
:106FD0002DE9FF474D4F4E4C03901FFA80F9C0F347
:106FE00007454FEA10683E464A4BDFF85CA19847D8
:106FF00000230093052219464748B8474748B84739
:10700000AAF800908AF802508AF803804448B847EA
:107010001DB1236843F0004323602046414B98474D
:10702000002836DB4048B047404B984701230021F9
:107030003F488AF804303F4B98473F4B98473F48BA
:10704000B0473F48B0473F4B3F4898473F48B0475D
:107050003F48404B9847011E07DB3F483F4B98474E
:107060003B483F4B9847011E07DA3E48B04710E0C7
:107070003D4B04B0BDE8F04718473C48B0473C4B97
:10708000984720B14A46002120463A4B98473A4853
:10709000B047236813F0005316D1226822F44062EF
:1070A0002260226842F400622260344A126810684A
:1070B00028B10122009209211A46314DA847B8F1A2
:1070C000000F01D02F4B9847236899001AD5A56867
:1070D000EA07CDD520482C4B98472C4B98470023E6
:1070E0008AF804302A4B98472A4B98472A4B9847EE
:1070F0002A4B984705F00505294B98476B1F5D42C1
:107100005D4171E704B0BDE8F08700BF754A010832
:10711000002E0020ABFA0108691203088B12030845
:10712000991203083DB80008A712030899940008B3
:1071300040420F00750F0208A96D0008BB1203083A
:10714000C8120308DD6D0008702B0020E912030847
:10715000803000205D3C020808300020C74601084E
:1071600095350208FE1203085DF901080C130308A7
:107170003D5F000819DD0008F6120308D02B00203F
:107180008579010869940008C5460108B9BB000863
:10719000BD640008C9740108B9630008DD74010802
:1071A000916900080A4600F11803500710B547BF5F
:1071B0000548064C0648074C2021A04710B1002383
:1071C0008360C36010BD00BF0C2C0020F94B020887
:1071D000002E002041C1000870B504461D46084637
:1071E000094B04991646984750B112220123C4E96D
:1071F0000023A06000238660C5600361184670BD4F
:107200004FF07A4070BD00BFA57100080023836075
:10721000C36019B10146024B02481847704700BFCE
:10722000A54A02080C2C0020C36803B11847704718
:10723000836903EB011100200B7A13707047836997
:1072400003EB011100208B6813607047836903EB27
:107250000111002091F9083013707047836903EB26
:1072600001110020B1F9083013807047836903EBE6
:10727000011100208B6813607047836903EB0111D3
:1072800000208B6813607047836903EB01118868E5
:10729000CB6882E80900002070470901836958180B
:1072A0005B5C122B0DD1836843B1597D012908D154
:1072B0001969516018331360002070474FF0214066
:1072C00070474FF0224070470901836958185B5C92
:1072D000122B0DD1836843B1597D042908D1196956
:1072E000516018331360002070474FF02140704701
:1072F0004FF0224070470000004B1847C972000849
:107300000901836958185B5C122B0DD1836843B166
:10731000597D012908D11969516018331360002083
:1073200070474FF0214070474FF0224070470901ED
:10733000836958185B5C122B0DD1836843B1597D6A
:10734000022908D119695160183313600020704771
:107350004FF0214070474FF0224070470901836988
:1073600058185B5C122B0DD1836843B1597D0429F9
:1073700008D11969516018331360002070474FF02D
:10738000214070474FF0224070470000004B1847E3
:107390005D7300080901836958185B5C122B0DD1DD
:1073A000836843B1597D082908D1196951601833A0
:1073B0001360002070474FF0214070474FF022408B
:1073C00070470901836958185B5C122B0DD18368E3
:1073D00043B1597D042908D11969516018331360EC
:1073E000002070474FF0214070474FF02240704717
:1073F0000901836958185B5C122B0DD1836843B176
:10740000597D082908D1196951601833136000208B
:1074100070474FF0214070474FF022407047000006
:10742000004B18479D8500080222014B184700BFFA
:10743000918400080522014B184700BF9184000881
:107440000722014B184700BF918400080A22014B14
:10745000184700BF9184000807B502A961E902231B
:10746000024B984703B05DF804FB00BF4585000858
:107470000322014B184700BF9184000838B50C4621
:1074800081691D46204601EB0211044B98470028F4
:10749000A2BF08342C60002038BD00BFC14F0208D5
:1074A00038B50C4681691D46204601EB0211044B9C
:1074B00098470028A2BF08342C60002038BD00BFC8
:1074C000C14F020808B50B468169184601EB02114D
:1074D000024B0022984700EAE07008BDF95202080A
:1074E00083699868704700EB01100830704700EB23
:1074F00001100830704700EB01100830704700EBB6
:10750000011008307047000001380D2834D8DFE83A
:1075100000F0070C0F1215181B1E2124272A2D30EE
:10752000164B1B680B6000207047144B5B68F9E733
:10753000124B9B68F6E7114BDB68F3E70F4B1B69B7
:10754000F0E70E4B5B69EDE70C4B9B69EAE70B4BF1
:10755000DB69E7E7094B1B6AE4E7084B5B6AE1E795
:10756000064B9B6ADEE7054BDB6ADBE7034B1B6BD5
:10757000D8E7024B5B6BD5E70F20704798310020AE
:107580001368112BF7B5154603D3122B0AD9152B07
:1075900002D00F2003B0F0BD54682378162B03D11E
:1075A000A4680CB90720F5E701A9A8680B4B984718
:1075B00090B92E690A4BEF6801AA314620469847D8
:1075C00050B936B1A068074B427D39467243183036
:1075D0009847A3681833EB600020DBE709750008C3
:1075E00059610208CF01030812681B689A4209D149
:1075F000152A09D80123934013F4181F0CBF0F203C
:1076000007207047012070470F2070471223136036
:107610008B699B6853600020704784B010B503A845
:1076200080E80E00039B0999122B2BD1049A72B3A8
:10763000089B1B01D018D25C0346162A1BD19B68FD
:107640001A78FAE7122A11D0152A1BD11A78152AAE
:1076500007D11A7D03F118041B69CC600B614860E7
:107660008A6000200FE008334B60FAE79B681C78C3
:1076700015229442F8D1112A0A600AD0E2D8013AC0
:107680000D2AF0D90F20BDE8104004B07047022049
:10769000F9E70720F7E70000096870B515461C46B2
:1076A00009B9022070BD00231A461B481B4EB04783
:1076B00000282DD029461A4B98470028F1D002788F
:1076C0000346162A1BD19B681A78FAE7122A11D0B2
:1076D000152A1BD11A78152A07D11A7D03F1180132
:1076E0001B69E16023616060A260002070BD083307
:1076F0006360FAE79B68197815229142F8D1112A44
:10770000226007D0E2D8013A0D2AF0D90F2070BDCF
:10771000052070BD072070BD803000208D2D02082F
:10772000652C020810B5896912018818895C024627
:1077300016291BD192681178FAE7122911D0152960
:107740001BD11178152907D1117D02F11804126996
:10775000DC601A6158609960002010BD08325A60E0
:10776000FAE79268147815218C42F8D11129196032
:1077700005D0E2D801390D29F0D90F2010BD07201E
:1077800010BD0000F7B54B6C15460A6C9A420E46C8
:1077900002D30120204B9847346C04F1100333646A
:1077A00012220123C4E900230023A3602A68112ABE
:1077B00030D005D8531E0D2B20D90F2003B0F0BDBB
:1077C000122A24D0152AF8D101A9A868134B98478A
:1077D000D8B92E69124BEF6801AA31462046984766
:1077E00098B936B1A0680F4B427D394672431830C4
:1077F00098476C60A3681833EB6006E0002343F001
:107800000103C4E9002308346C600020D6E76B68EC
:10781000A360FAE70720D1E7154C000809750008B6
:1078200059610208CF0103080378122B07D1806841
:1078300030B10078A0F1370358425841704700201A
:107840007047000038B54B68012B05460C4602D046
:107850000120034B984794E80F0085E80F0038BDDE
:10786000154C0008026C436C9A4210B5044602D3D2
:107870000120034B9847206C00F11003236410BDD6
:10788000154C000838B5044B0D4698472946044668
:10789000024B9847204638BD6578000845780008B7
:1078A0002DE9F74F8E68D1F804A0F77AB37A0193E7
:1078B00003373B44B2F1000BC8BF5B44092B9EBFAA
:1078C0000A37FF1A0A23D0F86081644C05468946BE
:1078D0000633002223216248A0470446002800F016
:1078E000B680D5F86C314362056100F12C0399E84C
:1078F000070083E80700019A5A4804F16003E36136
:1079000003EB021303EB071767640027636123642B
:10791000A761554BA764E76498477368606513F4E3
:10792000003362D0514BA363A762E76315F5AA75D4
:107930000CD0AC420AD0E268A36802B1936003B1F4
:10794000DA60EB68E360A560EC609C60B37A2BB111
:1079500033465246E1694348454DA847736813F0E2
:10796000407F0BD0D90142BFA26A42F48072A2626A
:107970009A0142BFA36A43F48053A362E268D368CA
:107980000BB1136D01332365364B1B69F3B1226BC9
:10799000A38DD2F88820D35C9B0742BFA36A43F033
:1079A0000043A362236993F8743153B9A36A002B8F
:1079B00007DBD8F80C30002B35D0D8F82830002B56
:1079C00007DA3022214627482A4B9847D8F80C304E
:1079D0004BB3D8F83820A36B9A4224D1A36A13F48E
:1079E0004C5F1DD143F4C0231CE0DAF820201AB10B
:1079F000A18D52F821206ABB1F4B7288A3634FF6FA
:107A0000FF739A4202D14FF077401DE00123A36239
:107A1000DAF81830D96D0A441344E363236285E72A
:107A200043F48023A362BBF1000FB9BF727AD8F888
:107A30004030636CA361BCBFA3EB0213A3614FF0A2
:107A40000000B8BFC8F8403003B0BDE8F08F4FF079
:107A50007A40F9E7A263A362DFE700BFDD4B0208CB
:107A60000C2C0020002E00201DD8000829590108E8
:107A700009C4000879D500085D5A01082DE9F84FBE
:107A80009B46C36C0A9E04468946924623B14FF03A
:107A900000084046BDE8F88FB568436CDBF800206D
:107AA000A97A9A1A6B7A0B44E97A0B440233B3EB46
:107AB000221FECDA826B494B9A42E8D16B6823F0C3
:107AC0008042B2F5805FE2D2DA06E0D473681B6AC6
:107AD00023B1328853F82230002BD8D16A884FF670
:107AE000FF739A42D3D004F14C013D483D4B984777
:107AF00080460028CBD07368E76C9A696B88D16D9B
:107B00000B441344D9F80020FA61E26B3A62E2694F
:107B10003A60A2697A6004F12C0E9EE8070007F132
:107B2000100C8CE807006269BA600B9AFA60DBF807
:107B300000201032CBF800207268CAF800200B9A9F
:107B4000C9F80030A26195F80AC0676CA7EB0C1762
:107B5000E76196E807008EE807006764DBF800201D
:107B60006261DBF80020E3631032D9F80030226450
:107B70002362BCF1000F05D072681B481B4E2B46D8
:107B80003946B047A36A43F00802A2622A7A22B1BA
:107B900043F4801343F00803A362236D013323658C
:107BA000114B1B69002B3FF474AF226BA38DD2F8ED
:107BB0008820D35C9B0742BFA36A43F00043A362C3
:107BC000236993F874311BB9A36A002BBFF661AF28
:107BD000302221460448064B98475AE75D5A01086F
:107BE0000C2C0020214C0208002E002009C40008A3
:107BF00079D5000830B5C46C6268826122460346BC
:107C000052F8101BC161416B887A596C01EB00116D
:107C1000596407CA03F12C0585E80700E2691A6276
:107C2000226ADA63A2685A61E2681A6430BD000011
:107C300038B50446144B056C9847A36ADB0208D597
:107C400023691B6C2BB9114B294620469847104BD2
:107C50009847104BE16C104898470023E364226971
:107C6000A36A92F8742123F4801323F00803A3621B
:107C70000AB9002B04DA002221460848084B98472D
:107C8000236D013B236538BDF57B0008857800082E
:107C9000895502083B4C02080C2C0020002E0020C5
:107CA00025D400084A6830B582610A460C4652F86D
:107CB000101BC161034600F12C0507CA85E80700C7
:107CC000E2691A62226ADA63A2685A61E2681A6497
:107CD0005A6B917A5A6CA2EB01125A6430BD30B5DE
:107CE00082694A600D46C26945F8102B00F12C02EA
:107CF00003460C4607CA85E807001A6AE261DA6B98
:107D000022621A6C5B69E260A36030BDF0B50123AA
:107D100087B01222CDE9022300230493836AC56849
:107D2000016913F0006704462AD04B6A9A0702D40F
:107D300001203A4B984723695B6A1B0702D4012054
:107D4000364B984723691B6C13B90120334B984776
:107D500023691B6C9A68324BDB6E9A4202D0012079
:107D60002E4B9847606D2F4B984710B101202B4B3D
:107D700098472269536A23F00A035362002640E0C1
:107D80000A6C002A2FD113F0806312D1426B296C48
:107D9000577A0193012300938269234E686D3B4615
:107DA000A1EB0711B047061E32DB2B6CA3EB0713C8
:107DB0002B64636B1B7A002BE0D01C4B1C4E2846B7
:107DC000984712220123C0E9002300238360216C1D
:107DD000024607461039686DB047061E18DB384664
:107DE000144B9847CAE7124E686D3B4602AA3831D9
:107DF000B047061E0CDB3E4620690F4B02A9383007
:107E00009847696D0D4B0E489847304607B0F0BD56
:107E10002A46314602A80B4B9847EDE7154C00085F
:107E200098310020B9250208F5230208657800087A
:107E300015220208895502084578000811D8000863
:107E4000002E0020659901082DE9F7431F468B6835
:107E500004465E7A1E4B104689461546984710B96F
:107E600001201C4B9847D5F808801B4B404698478B
:107E7000002829DB324649462046184B98470028FF
:107E800022DBD4F86041D8F80C00A36A606523F4C3
:107E9000802343F08053A36229460023A269104D3A
:107EA000A847002810DBA269002501950095731EE4
:107EB00010323946606D0B4EB047002804DB616D0F
:107EC00009480A4B9847284603B0BDE8F08300BF35
:107ED00029780008154C0008ED5E0208A17800081A
:107EE00015220208F5230208002E002011D80008F0
:107EF0002DE9F047426B0446507A8EB0002866D0D8
:107F0000216B384B384E08A898470C9BA4699B06F8
:107F100004A908A848BF1034B047002857DBDFF891
:107F2000E480324FDFF8E09010340D9B002BA4F179
:107F3000100555DD04A908A8B047002847DB059BBC
:107F4000002B01DD1034F0E714F8103C122B18D18F
:107F500007A901A8C847039B254A93F80FA0182337
:107F600003FB0AF3D258234B134053B12846224B4C
:107F70009847014670B3037853451CD128461F4BE0
:107F800098479DF81830142BDCD19DF81030002B49
:107F9000D8D114F8103C122BD4D154F8083C002B43
:107FA000D0D01B78142BCDD12A4629464046B8475D
:107FB0000028C7DA0BE054F8083C9A68079B9A42FD
:107FC0000BD101A928460E4B98470028D9DA0EB0EC
:107FD000BDE8F0874FF02140F9E74FF02240F6E787
:107FE0000020F4E7A11202083D30020879C600081B
:107FF0003055030808002000B152020845780008F7
:1080000025520208002E0020951302082DE9F04F9A
:1080100091B001AC84E80E00DDF80CB01A9DDBF8DD
:1080200004309BF809A0122203F010080123CDE9C7
:10803000082300230A93814608A90CA8514B9847AE
:10804000DBF8047017F480576AD0214605A84E4E1D
:10805000B04715B101204D4B9847214605A8B047C0
:1080600010B90120494B984705AA08A94848494B2F
:108070009847061E61DB08A94846474B984708AD5C
:10808000B8F1000F53D000271C9B9A455CD1DBF858
:10809000043013F4107F1BD015B901203B4B9847D7
:1080A000B8F1000F02D00120384B984704A92846A8
:1080B0003A4B9847061E40DB05AB224604A93848D8
:1080C000384EB047002836D005A92046364B984791
:1080D000B8F1000F04D12846344B9847002836D118
:1080E000039BD9F810005A7A314B21469847061E57
:1080F00023DBD9F81030D3F86041B8F1000F03D179
:108100002946A0692B4B9847BAF1000F30D0A069DF
:108110001B99294B4FEA0A1200EB0710984727E0FA
:10812000B8F1000FB0D115B94FF0214605E00AF1C2
:10813000FF3A0127A8E74FF022460CA81F4B9847AB
:10814000304611B0BDE8F08F4FF07D46F5E721468F
:108150001B9BD9F810001A4C2A46A047061EECDBE0
:10816000D9F81030D3F86041A36A43F08063A3626A
:108170002046144B984710EA200638BF4FF07B4644
:10818000DBE700BFC5DF0008C9130208154C000873
:10819000002E0020C9C10008857800086519020872
:1081A0000C2C00200D4C0208191602082978000832
:1081B000A178000845780008CF01030809E000080D
:1081C000497E0008F17E000870B504468CB00D466B
:1081D000002A26D0214B22489847036B0646B3B1AC
:1081E00012200121CDE908010A9308A9626A002D35
:1081F0002FD04FF0FF3400200CAB6FF0004563E947
:108200000A450090174C1648A0470CB070BD164A9E
:108210001348164B08A998470028F6DB0A9B3363DE
:10822000E3E7436B5B68DB0611D5C36A026B99B267
:10823000D2F884201B0C32F811201B040CA9134324
:1082400041F8103D04A80A4B984704A9CEE781697C
:10825000CCE7084B02489847D7E700BF1DD8000875
:10826000002E002061CB0008E0310020E1C50008AD
:10827000894E0208A1CB0008F0B5036993F8743168
:1082800093B0044613B9836A002B04DA0022214616
:108290006B486C4B9847A36A44F24442134223D084
:1082A00059060BD5A56B43F08003A36235B1664B2D
:1082B00098478DE811009DE80300A847A36A5A0576
:1082C00007D523F480630022A362114620465F4B4A
:1082D0009847A36A5F0407D523F48043A362012271
:1082E00000212046594B9847E568E968002950D09D
:1082F000AB6A002B04DA2A6A5148554B2946984745
:10830000AB6ADE0616D5A169524B28469847064649
:10831000514B98473378162B04BF12233370AB6A46
:1083200023F01003AB62A36AD8000ED54B4B01209B
:1083300098470AE0A36A4A4A13421BD0190304D49F
:10834000DA0002D52046474B98472069D0F8203103
:108350001BB100222146444B9847636A99688B6899
:1083600013B14B699C4266D021464048404B984728
:1083700013B0F0BD636B1B7A002BE6D023691B6C36
:10838000002BE2D1216C334B103928469847324BF1
:10839000CEE72069D0F87021002AD6DB284BD3F82D
:1083A000B031002BD1D01D699542CED95D7D02FB45
:1083B00005351835036CA96012260127C5E9006749
:1083C0000BB1AB60C1E7626B137A002BBDD0216BA0
:1083D000284B06A89847216C274B10392846984708
:1083E00002A906A8254B9847002802DA01201B4B5A
:1083F000984705A90CA8224B9847002802DA0120CB
:10840000164B98472278182353431E4AD3589B0291
:1084100005D40F9BDB8A03F03003302B95D10DA9D7
:108420002846194B984700288FDA01231222C5E904
:1084300000230023C5E701220869144B984793E7FE
:10844000002E002025D4000875910008C98100087D
:1084500089D600088578000889550208154C00085F
:10846000000008100D7D0008715301080C2C00203D
:10847000A54A0208A1120208457800083D3002080A
:1084800025170208305503080551020859FB010859
:1084900038B5064B0D46144698470023E2B243F028
:1084A0000103C0E90023856038BD00BF657800087E
:1084B00008B5074B2DED028BB0EE408A9847092294
:1084C0000123C0E9002380ED028ABDEC028B08BDC8
:1084D0006578000800B52DED028BB0EE408AF0EE15
:1084E000608A83B0104B98478DED008B01230E22DC
:1084F000C0E900239DF8003003729DF801304372FB
:108500009DF8023083729DF80330C3720C30002353
:108510000DEB03021279C2540133042BF8D103B0DE
:10852000BDEC028B5DF804FB6578000810B5044BC8
:108530000C46984707220123C0E90023846010BD40
:108540006578000810B5064B0C4698470C220123AD
:10855000C0E9002394E80C008260C36010BD00BF36
:108560006578000810B5044B0C4698470822012393
:10857000C0E90023846010BD6578000810B5064B83
:108580000C4698470D220123C0E9002394E80C0013
:108590008260C36010BD00BF6578000810B5044B51
:1085A0000C46984701220123C0E90023846010BDD6
:1085B0006578000810B5044B0C4698471222012339
:1085C000C0E90023846010BD6578000810B5044B35
:1085D0000C4698472146034BBDE81040184700BFA2
:1085E0006578000851760208026C52F8083CB3FA2C
:1085F00083F3012001215B0942E9040142F8083CB0
:108600007047026C52F8083CB3FA83F35B0942F8F6
:10861000083C70472DE9F341866C054688461746AD
:10862000CEB9104B984712220123C0E9002386607F
:108630000446D8F808200C480C4B69469847002897
:108640000DDB0C220123C4E900239DE80C00E3604C
:108650000123A260AB646B6908333B60002002B069
:10866000BDE8F08165780008002E0020F9CE0008F2
:108670002DE9F14F0446C06C284D294E04F1300B12
:1086800004F1340A04F1380904F13C0804F120072C
:1086900000282CD01430A847E06C1830A847E06CB4
:1086A0002030A847E06C1C30A8475846A8475046E1
:1086B000A8474846A8474046A8473846A847E36C1D
:1086C0009A695868517AB047E36C9A691868917A48
:1086D000B047E36C216C9868091A0911B047636BC5
:1086E000E069997A334601B0BDE8F04F1847584623
:1086F000A8475046A8474846A8474046A847384696
:10870000A847636BA069597AB047636BE069997AAF
:10871000B0476069216C091A0911E3E779EA00089A
:1087200031EA000808B5436B1B7A13B10021024BF4
:1087300098474FF04A4008BD2D85000808B1014B0D
:1087400018477047394B000808B1014B184770476C
:10875000394B00082DE9F041054678B1084B094F27
:1087600093E84001B04509D056F8044B28462168EB
:10877000B8470028F6D12046BDE8F0810024FAE78A
:10878000842B00204504030870B500293ED0204DFD
:108790002A686868841A2411002C134620DD1268A8
:1087A0008A4203D05A688A420BD10433984222D0BD
:1087B00050F8041C1A68196040F8042D6860002005
:1087C00070BD9A688A4201D10833EFE703F11002C5
:1087D00052F8046C8E4201D10C33E7E7013CDBE731
:1087E000821A9210022A0CD0032A06D0012A02D142
:1087F0001A689142DAD0052070BD1A688A42D5D035
:1088000004331A689142D1D00433F1E7022070BDDD
:10881000842B002038B50A4B0A4D186800241C60D0
:108820005C609C60A8472046A847074B074D186826
:108830005C601C609C60A8472046A847204638BD65
:10884000842B00203D870008782B002049870008F2
:1088500070B500283ED0204D2A6869688C1A241112
:10886000002C134620DD1268824203D05A688242EF
:108870000BD10433994222D051F8040C1A681860C5
:1088800041F8042D0020696070BD9A68824201D1D0
:108890000833EFE703F1100252F8046C864201D16D
:1088A0000C33E7E7013CDBE78A1A9210022A0CD06E
:1088B000032A06D0012A02D11A689042DAD0052094
:1088C00070BD1A688242D5D004331A689042D1D064
:1088D0000433F1E7022070BD782B00202DE9F04F22
:1088E000904687B099460F4609B31349DFF850A068
:1088F00091E82008AB451CD055F8046B3946306A26
:10890000D04704460028F5D1149B0493DDE91223D7
:10891000CDE90223DDE910233046CDE900234146AD
:108920004A46064B9847204607B0BDE8F08F022024
:10893000FAE70520F8E700BF782B0020656F0208F2
:10894000450403082DE9F84390E81800E41AA41040
:1089500014BF23460123E4180646894602D2B4F127
:10896000804F22D36FF04044A000124B9847074637
:10897000D6F800807568D9F80030A5EB0805EF42FD
:1089800018BF7B51AB0804D02A46414638460A4BF3
:10899000984704353D444046084B07EB840498470C
:1089A00037607560B460BDE8F883002CDCD12746E1
:1089B000DEE700BF294B0008E50103083D870008FA
:1089C00013B5019121B3144B984778B1019913481D
:1089D0000968134C00231A46A04738B18269019BED
:1089E00051695A68914215D19B6803620D488268AB
:1089F00043689342024607D0019903B119600433DA
:108A00005360002002B010BD01A9074B9847F8E75A
:108A10000220F7E71620F5E7315F000880300020DC
:108A20008D2D0208842B0020458900082DE9F8438C
:108A300090E81800E41AA41014BF23460123E41898
:108A40000646894602D2B4F1804F22D36FF04044EB
:108A5000A000124B98470746D6F800807568D9F8F1
:108A60000030A5EB0805EF4218BF7B51AB0804D0DE
:108A70002A46414638460A4B984704353D4440460D
:108A8000084B07EB8404984737607560B460BDE815
:108A9000F883002CDCD12746DEE700BF294B000815
:108AA000E5010308498700082DE9F74307460190CF
:108AB00028B3D0F82080B8F1000F20D0114DDFF896
:108AC0004C906C682E68B442334608D01B6841460F
:108AD000186A0436C8470028F5D1082007E0AB68BB
:108AE0009C4207D004B1276004346C60002003B0BE
:108AF000BDE8F08301A90348034B9847F6E702203D
:108B0000F5E700BF782B00202D8A000845040308F4
:108B100000F47F40B0F5807F10B504D0B0F5007F41
:108B200005D0002010BD054BBDE810401847044B90
:108B300098470028F5D0034BF6E700BF59420208DA
:108B40006D6C0008AD6C000800F47F40B0F5807FCC
:108B500010B504D0B0F5007F05D0002010BD044B47
:108B6000BDE810401847034B9847034BF8E700BF98
:108B70008D420208CD6C0008916C00082DE9F84F79
:108B800003F10109DFF864A0DFF864B00E46154672
:108B900000F47F484C4600275DB1002C09DDB8F594
:108BA000807F09D0B8F5007F11D0013CD04700B1DB
:108BB00094B93846BDE8F88F29463046D847002892
:108BC000F7DBF2D02D1A064407444C46E4E7294669
:108BD0003046044B9847F2E7002101220846024B39
:108BE0009847D9E7ED6C00081DB60008B17401087C
:108BF000A942020800F47F40B0F5807F0B46114681
:108C000004D0B0F5007F04D0002070471846024B16
:108C100018471846014BFBE7C94202080D6D0008D2
:108C200000F47F40B0F5807F04D0B0F5007F03D022
:108C300000207047014B1847014BFCE7E94202084E
:108C40002D6D000883680BB1C0681847704700009D
:108C500080B584B000AF78607B681B7E002B05D0A8
:108C60007B68FB60F868054B984703E07B68184613
:108C7000034B984700BF1037BD4680BD458C0008A8
:108C8000A590000880B500AF0248034B984700BF8D
:108C900080BD00BF902B00202190000890B585B0CA
:108CA00000AF3B4618461B4B98471B4B1B681846AA
:108CB0001A4B9847F860FB681B681846184B984792
:108CC000B860BB68002B1DD01020164B9847FB687E
:108CD0001846154B9847BB681B681846104B9847B9
:108CE0000346002B03D0BB68D3E9043403E04FF004
:108CF000FF334FF6FF74184621460C4B9847F8682F
:108D00000B4B98473B4618460A4B984700BF143711
:108D1000BD4690BD09750108902B002065900008A4
:108D200065900008C5B500082D900008A10E020846
:108D3000518C00084175010890B589B000AFF8600A
:108D4000C7E90023D7E90034234302D10120264B91
:108D5000984707F110031846244B9847FA68D7E95B
:108D60000034C2E90434224B1B681846214B984753
:108D7000F861FB691B6818461F4B9847B861BB69CF
:108D8000002B14BF01230023DBB2002B0CD0FB69A6
:108D9000D3E90434D7E90012A24208BF994202D3B2
:108DA000BB69FB61E5E700BFFB681946F869134B37
:108DB0009847FC680E4B1B6818460E4B98470346B5
:108DC0009C420CBF01230023DBB2002B03D0D7E968
:108DD00000010B4B984707F110031846094B9847C1
:108DE00000BF2437BD4690BD154C00080975010829
:108DF000902B00206590000865900008679000089F
:108E0000A10E02084175010890B589B000AFF86065
:108E1000C7E900230C4B9847C7E90601D7E90001D1
:108E20000A4B9847C7E90401D7E90612D7E9043489
:108E30005B1844EB02041A462346F8680449884745
:108E400000BF2437BD4690BD8D0E02086D0E02088E
:108E5000398D000890B583B000AF786039603B6809
:108E60004FF000041A46234678680349884700BF3C
:108E70000C37BD4690BD00BF098E000890B589B083
:108E800000AF786007F10C0318461A4B98471A4B4D
:108E90001B681846194B984778617B681846184B31
:108EA00098477A697B689A421BD11348154B9847BB
:108EB0000346002B06D04FF0FF334FF6FF74C7E98F
:108EC00006340AE00C4B1B6818460C4B9847786137
:108ED0007B69D3E90434C7E90634D7E906010A4BB4
:108EE000984707F10C031846084B984700BF2437F2
:108EF000BD4690BD09750108902B002065900008C3
:108F00002D90000841900008A10E0208417501084B
:108F100090B58BB000AFC7E902017A6001233B62D4
:108F20000223FB610423BB61284B1B681846284BB6
:108F3000984778617B691B681846264B984703461B
:108F4000002B0CBF01230023DBB2002B02D0052332
:108F50007B620DE07B69D3E90434D7E90212A242B7
:108F600008BF994202D203237B6201E000237B62A7
:108F70007B6A03F00103002B03D0D7E90201164BF3
:108F80009847D7E90E237868144988477B6A03F02D
:108F90000603002B16D00D4B1B6818460C4B984748
:108FA00078617B6A03F00203002B03D07B69D3E96D
:108FB000043403E04FF0FF334FF6FF7418462146A8
:108FC000054B984700BF2C37BD4690BD902B002025
:108FD0006590000865900008A10E020871F901086B
:108FE00080B584B000AF3B1D1846094B984709482F
:108FF000094B9847F860FB68002B00D0F7E700BFEB
:109000003B1D1846054B984700BF1037BD4680BD35
:1090100009750108902B00204D900008417501084A
:10902000031D03600023436080607047426803684B
:1090300002B1136003B15A600023036043607047BC
:10904000031D0068C31A58425841704710B50468A0
:10905000206818B12046024B9847204610BD00BF3B
:109060002D900008704768B161B188420AD04A6803
:109070000B6802B1136003B15A60436881E80900CC
:109080004160196070470068003018BF01207047C8
:10909000034B1A1D1A6000225A609B60704700BF84
:1090A0009C2B0020836813B50446A3B10B4B684684
:1090B00098470B4B63B19C420AD06168226801B1AA
:1090C0000A6002B151605A68626023605C6014609B
:1090D0006846044B984702B010BD00BF09750108EF
:1090E000A02B0020417501080023036043608160CC
:1090F000C260704737B50D4B684698470C480D4B1A
:10910000984788B18468C5680B4B684698470CB18E
:109110002846A0476846094B984701246846084BF3
:109120009847204603B030BD0446F7E709750108AB
:109130009C2B00204D9000088974010825750108BA
:109140004175010837B5074B074D084C68469847ED
:109150002846A0470028FBD16846054B984703B036
:1091600030BD00BF097501089C2B00204D90000800
:109170004175010800487047A82B00207FB50146C3
:109180000A4B6846984700280EDB039BDA7B1823BE
:109190005343074AD05800F4C020A0F5C0235842DA
:1091A000584107B05DF804FB0020FAE7D517020824
:1091B000305503082DE9F04389B0884616461F460E
:1091C000DDF84090054600283ED00C68002C75D094
:1091D000002A75D004F1B0030B60B022394B002196
:1091E0002046002F08BF2F46984727602B786360E2
:1091F0006B78A3606B68E360B9F1000F17D0D9F802
:109200000030C4F898306368013B1B2B1CD8DFE8A2
:1092100003F0161616161616161616161616161627
:1092200016161D35404044351B1B1B1B164E294688
:1092300002A8254B98470028E5DB039BE1E755F89A
:10924000083F23616B68636101201FE0AD68C4F8CB
:1092500094507DB128461D4B98477F280346C4F89B
:10926000900028BF7F232A46802104F11000184C6B
:10927000A047E9E7C4F890502574E5E7CDF80090E1
:109280000023721E4146A868FFF794FF09B0BDE8AD
:10929000F083AB68C4F89830D6E72B69C4F89C30EB
:1092A0006B89C4F8A030EB68C4F8A430CCE7AB6895
:1092B000C4F8A830EB68C4F8AC30C5E72046E5E751
:1092C0001046E3E719020308D5170208B55B00084A
:1092D000895B000838B50C46054610B10378162B9B
:1092E00035D0256025B12B78122B32D1AB6883BBEA
:1092F0000123002023716071A37138BD0023237105
:109300002A78122A08BFAB68A26808BF5B7802F00F
:10931000600108BFC3F300132029637101D0402905
:1093200001D1012310E002F01F02102AF9D8012117
:1093300001FA02F20B490A42F3D02BB90A4AE36858
:10934000126C9A1A53425341A371002038BD8568AC
:10935000C7E7294604F10800044B98470028CDDAF6
:1093600038BD00BF0201010098310020D517020866
:109370002DE9FF410D469046044690B10678D8F895
:1093800000000023CAB243F00103D8F80410CDE96D
:109390000023B54202AB03C30AD01B2D13D1122EFA
:1093A00003D0002004B0BDE8F081A368002BF8D101
:1093B0002346012003F8085BD8F80020A260D8F803
:1093C00004205A60EEE7122D05D1029B002BE8D154
:1093D0001B2EE6D1ECE718230A4F7343FB589B037F
:1093E00002D40120084B9847182303FB06725279D8
:1093F000042AD6D103FB05756B79032BD1D83546EA
:10940000D6E700BF30550308154C000830B50C4BAB
:1094100089B0D3F8B041029412220123CDE9002390
:1094200005460246694604A8064B98470028A3BF94
:10943000607D05FB00401830002009B030BD00BF42
:10944000002E0020254F02080378122B0AD18068D5
:1094500048B10378142B05D1407880F01000C0F398
:10946000001070470020704738B50748074B084C7C
:10947000084D984723689A0005D423689B0302D4BB
:109480002046A847F6E738BD3C140308754A010892
:10949000002E0020B1DC00082DE9FF471E4D1F4CB7
:1094A000DFF89490A8471AA7D7E900670023361879
:1094B0004F410293A046D9F80030186840B142F2FB
:1094C00001030093082202AB0021DFF870A0D0470F
:1094D0002368002B0FDB124B984760B1114B0F48EC
:1094E000984704B0BDE8F087A847864277EB0103B0
:1094F000E1DA0D4807E00D4B20469847D8F80030D8
:109500005B00F1D50A480B4B9847E7E7AFF30080C3
:1095100080F0FA02000000008D100208002E0020EA
:1095200089F90108EDDC00082D140308B1DC0008FE
:109530001B140308754A0108D02B00208579010807
:109540001FB5074B02901B680193064B0093064B17
:10955000064A1B680068064CA047002004B010BDF6
:109560009C1403089414030868160308A014030845
:10957000A976010838B5134B134D144C1C60B0226A
:109580000021134B28469847124B104859699B6994
:10959000994209BF104B25601B6823600F4B984709
:1095A00000280DDB0E4B0F4C98472146836841F88D
:1095B000040B98474FF47A73A3600B4B9847002035
:1095C00038BD00BFD02B00201C33002014330020F6
:1095D000190203083C0A0020E434002041950008E9
:1095E00079610008D0330020617C01080068014BDC
:1095F000184700BF9577010808B5034B1868034B5F
:109600009847002008BD00BFD02B0020ED95000832
:109610000068014B30301847454702080068014B8D
:10962000184700BF41780108064BD3F8D40083687F
:109630002BB1026A8A4200D170471846F7E71846F4
:10964000704700BF002E002010B50B4AD2F85831E9
:10965000996821B1DC69844208D00B46F8E7D2F85A
:1096600064319A6832B1D969884201D1184610BD77
:109670001346F6E71346F9E7002E0020F8B5154823
:10968000154D0E461746A84704461448A8470444FB
:10969000601C800038600121114B98473060A0B1F8
:1096A000104B40F8044BD3F85821916821B1D2698E
:1096B00040F8042B0A46F8E7D3F8642193683BB1DD
:1096C000D26940F8042B1A46F8E74FF07A40F8BD0B
:1096D0001846F8BD582F0020E94C0208642F0020DE
:1096E000F54B0008002E00202DE9F74F9B46084659
:1096F000354B01929847054600285BD00026D5F8E7
:1097000058310024D3F808E0BEF1000F3AD0012E02
:10971000D86C04F1010C2DD1002831D0019A1168C8
:10972000026901EB0411E146CA60C269076AD21BF3
:109730000A615A6D126A4A619A6A8A61019AD96A03
:109740001268DF6B4FEA091902EB090ACAF80C101C
:10975000196AC91BCAF8101019B1D5F86071BB425B
:109760002ED102EB09085A6D9B6A126AC8F81420C0
:10977000C8F81830002818BF644601347346C1E7A2
:10978000A146DBE77EB920010C30104BCBF800007E
:109790004FF400619847019B186070B12B6A4360D9
:1097A0006B6A046083600136022EA8D1002003B0EA
:1097B000BDE8F08F4FF02140F9E74FF07A40F6E72F
:1097C0000139CAF81010CCE749960008F54B00089B
:1097D0007FB51C4D446A2B6843F080432B60C369FE
:1097E00013F002030E4623D104B3646804F00104AD
:1097F00002932B6813F4006F14BF04230023039318
:10980000082301936B4400930146002330680E4EF9
:109810000122B0472B6813F4406F04D12B686CB160
:1098200043F000432B60012004B070BD1C46DFE70D
:10983000002CEFD0646804F00104EBE723F0004350
:10984000F0E700BF002E0020A17901082DE9F041CA
:10985000C26912F0020286B006460F4645D106AB39
:109860000392049243F8042D214A106803A9046A64
:1098700004AAA047044678B9059B6BB10C20584355
:109880001C4B9847054658B9019500952B46012277
:1098900031463868184CA047002006B0BDE8F0817A
:1098A000DDF81480DDF80CC004992B4620465022C8
:1098B000404503F10C030BD05CF8204043F80C4CFE
:1098C00051F8204043F8084C43F8042C0130EFE7EE
:1098D0000C2358430190009500233868064C012260
:1098E0003146A0472846054B98470120D5E700BFE1
:1098F000D0330020E94B0008A1790108854B00080E
:10990000F0B51646164A85B0106804AB00240D4623
:109910000194029443F8044D076A02AA01A9B847CA
:1099200088B9039B7BB1019A1168029A02EB830309
:10993000934203D052F8044B2044F9E7002E0DD097
:1099400001DB032E01DD002006E0A942FBD808441C
:1099500085422CBF0020012005B0F0BD0120FBE7AF
:10996000D033002070B500249C420AD051F8245016
:10997000854204D852F824603544A84204D3013407
:10998000F2E74FF0FF3070BD204670BD2DE9F04F7B
:109990008BB09246149C01932246624B05900D4673
:1099A00098478146002800F0A280032C02D15E482F
:1099B0005E4B98475E4F0AAB3868002207920892C8
:1099C00043F8042D066A08AA07A9B047002840F00A
:1099D0008B80099B0493002B00F08680CDF80CA0AF
:1099E000019E029012E03B79002B33D0424629467B
:1099F0003046504B9847039BA3EB0803002B03937F
:109A000049DD029B0133464445440293049B029A7C
:109A1000934240DD00238DF81B30089B059853F8D6
:109A20002230039A9A4228BF1A4690462946224677
:109A30003C4B9847002857D0032CDCD801A353F89F
:109A400024F000BFE7990008E7990008A99A0008E8
:109A5000BB9A000834B901215046374B9847064657
:109A6000002841D03B79D3B938683346D0F810B0DC
:109A700042462946D847834654B9019B41461A6855
:109A80002E4B30469847019B186030462C4B984728
:109A9000BBF1000FAFD048460BB0BDE8F08F2E46AB
:109AA000002CA8D1A346E8E738683346D0F814B0B4
:109AB00042462946D8478346EAE707A90EC9DFF898
:109AC00088B02846D847834638680DF11B02C36921
:109AD0005946984740B99DF81B30002B8BD1386808
:109AE000594683699847E6E74FF00009D3E7022C0F
:109AF0000BD0032C0DD0012C04D1019852462946DD
:109B00000C4B98474FF00109C5E75246019928468A
:109B1000F6E7BAF1000FF5D05246FF212846094B6F
:109B2000EFE700BF01990008002E0020ADDE00081D
:109B3000D0330020CF0103088D4B00086D8602084A
:109B4000594B000819020308659900082DE9F043F4
:109B50000E46416A124B4D6807461868B5F5806F8E
:109B6000ADF20C4D28BF4FF48065A0B101240DF17A
:109B7000080800942A4643460968DFF82C903046CE
:109B8000C84701953068CDF8008000232246394649
:109B9000044DA84720460DF20C4DBDE8F08300BFF0
:109BA000D0330020A17901088D9900080C4B73B5C2
:109BB0001C6806460D467CB1416A0A4C022300939C
:109BC000284601F1080306C9A047002304460246BF
:109BD00031462868044DA847204602B070BD00BF3A
:109BE000D03300208D990008457B01082DE9FF4105
:109BF0000C460026416A009603AF05463B4606C95F
:109C00002046DFF82480C047042301930097206892
:109C1000044C334601222946A047012004B0BDE888
:109C2000F08100BFA17901088D9900080B4B73B535
:109C30001C6806460D4674B1416A094C0323009323
:109C400006C900232846A0470023044602463146A1
:109C50002868044DA847204602B070BDD0330020CC
:109C60008D990008457B010838B50D46446A0146C8
:109C700001222868034D0023A84723689847012044
:109C800038BD00BF457B0108F8B5476A0F4C054653
:109C90000E464FB10E4B984730B13B689A070FD52F
:109CA000A36843F00103A3602368306843F00053C6
:109CB0002360012200232946064CA0470120F8BD5D
:109CC0005B07F1D5A36843F00503ECE7002E002005
:109CD00089F90108457B0108012070470120704780
:109CE0001FB504AB074A43F8042D0C460422019229
:109CF0000093014600232068034C0122A047012065
:109D000004B010BD002E0020A179010830B5104A22
:109D10000C46416A13680D6849682B431360136849
:109D200023EA01031360C36913F0010385B00BD16B
:109D3000116804AA42F8041D042101910092014611
:109D400001222068034CA047012005B030BD00BFB0
:109D5000002E0020A179010870B4049CBDF80C60AD
:109D600083800023059D01804280C68003725CB120
:109D700055B12246054C372D2B46A44628BF372324
:109D80003821083070BC604770BC7047895B0008A0
:109D900070B5466A3E4BA2B004460D4674220021BF
:109DA00005A898473368013B062B2AD8DFE803F063
:109DB000080415292437640001200C2205AB23E098
:109DC00040F21F430593334B984700285BD0059B17
:109DD00043F0200305930422F0E706230A932E485C
:109DE0002E4B2F4E9847142103462B4A0DEB0100B2
:109DF000B04701201822E1E705A82A4B984701281F
:109E000043D00020024603460192009302462146B9
:109E10002868254C0023A047012022B070BD234EA6
:109E20001E4B304698470023029001960093194636
:109E3000052205A81E4EB0471E4BD3F8043183B14E
:109E40009B6973B1D88B198C5A8C9B8BADF85430AD
:109E5000ADF85600ADF85810ADF85A200120482250
:109E6000ACE700230120ADF85400ADF85630ADF852
:109E70005830ADF85A30F2E705A80F4B9847002844
:109E8000BFD040229AE70120A5E7742296E700BFE1
:109E90001902030889F901088A100308B55B000854
:109EA000895B000845860208A17901085C14030853
:109EB000599D000880300020714C000830B5436A7D
:109EC00085B004460D461868094B4FF40061984769
:109ED000039050B10423019303AB009321462868FB
:109EE000044C00230122A047012005B030BD00BF73
:109EF0008D4B0008A17901080020704701207047B0
:109F000001207047012070470120704701207047F1
:109F100001207047F0B5ADF5357D06461046BA9A7A
:109F200000920F4C0F4604AD042203A90395A047ED
:109F3000044668B1039B00955B1B0193012200233B
:109F400039463068074DA84720460DF5357DF0BDF0
:109F50000346024639463068034DA847F4E700BF80
:109F6000B5910008A1790108457B0108436A70B5E5
:109F70000D4606461968094B28469847044618B10D
:109F80000146074B074898470023E21A2868064C09
:109F900018BF01223146A047012070BD2996000854
:109FA00011D80008002E0020457B010838B5026A50
:109FB0000D46416A0446242304310748043AB2FBA3
:109FC000F3F2064B984721462868054C00230122EE
:109FD000A047012038BD00BF002E002041D300085B
:109FE000457B010870B58CB003AC06460D460B48A6
:109FF0000B4B21469847014618B924222046094BAD
:10A0000098472423019300942868074C00230122D9
:10A010003146A04701200CB070BD00BF002E0020CB
:10A020006DD0000819020308A1790108084A30B56B
:10A03000D2F8004100239C4207D052F8230010B10F
:10A0400005698D4202D00133F5E7002030BD00BF25
:10A050008030002070B50C68084B0D46210C164668
:10A06000984748B1436BA4B29C4205DA2946304672
:10A07000034BBDE870401847002070BD2DA00008BC
:10A080009513020870B50C68084B0D46210C164656
:10A09000984748B1836BA4B29C4205DA2946304602
:10A0A000034BBDE870401847002070BD2DA000088C
:10A0B0006515020870B50C68084B0D46210C164654
:10A0C000984748B1C36BA4B29C4205DA2946304692
:10A0D000034BBDE870401847002070BD2DA000085C
:10A0E0001916020838B508461D460D4B1446984708
:10A0F00000232B7090B1D0F8580182686AB1C36C0C
:10A1000033B1611E2CB901232B7038BD1046F4E722
:10A1100021464C1E0029F9D138BD104638BD00BF7C
:10A12000499600082DE9F04F476A9FB0012312229B
:10A13000BC68CDE90623002381468A46089306A918
:10A140000AA84C4B98471CB120464B4B98470446F5
:10A1500000252A46394606A8484B05959847B0F190
:10A16000000B0DF1600848DB4FF0FF3301950093C1
:10A17000089A4348434D042305A9A847B0F1000BB2
:10A180003BDB059B0CB1C3F87841D3F860516A6B97
:10A19000547A002C68D0296B3B4B12A89847169B29
:10A1A000AD699B0608D501231222C5E90023013CB5
:10A1B0000023AB60E4B210350EA912A8334EB047AD
:10A1C000B0F1000B19DB0DF1480CBCE80F00C646DE
:10A1D000AEE80F009CE803008EE803001D9B002BF7
:10A1E00012DD0EA94046B047B0F1000B05DB9DF82B
:10A1F0003830002BF2D04FF0224B0598C8B1244BD9
:10A2000098470023059314E01D4B0026F2B2A242AA
:10A2100005EB06110BDA1846039312AA1D4B98475B
:10A22000B0F1000B06F10106039BEFDAE5E74FF012
:10A23000000B0AA8184B9847BBF1000F16D1059BDD
:10A240007A68C3F87021DB69189304230193DAF864
:10A250000000CDF800800023012249460F4CA047A2
:10A2600001201FB0BDE8F08FA346E2E74FF0FF33B7
:10A27000EAE700BFC5DF000849960008ED6702085D
:10A28000002E0020B1BC0008A11202083D300208D7
:10A29000ADFE01085DC3000809E00008A1790108CE
:10A2A0007FB504AA00240D46064642F8044D02A9D3
:10A2B00028460E4B02949847A0420BDA23462246CA
:10A2C000314628680A4CA04702980A4B984701205B
:10A2D00004B070BD039B0193029B009301222346AF
:10A2E00031462868044CA047EEE700BF7D96000881
:10A2F000457B0108594B0008A1790108F0B585B0EC
:10A300000D4604AB416A114F09680024064643F824
:10A31000044D02AA28460294B847A0420BDA23460D
:10A320002246314628680A4CA0470298094B9847B4
:10A33000012005B0F0BD039B0193029B0093012215
:10A34000234631462868044CA047EEE7E99600080A
:10A35000457B0108594B0008A179010830B5436AD3
:10A3600085B0044618680B4B0D469847034610B15C
:10A37000094B9847012303930423019303AB0093F4
:10A3800021462868054C00230122A047012005B082
:10A3900030BD00BF49960008ADFE0108A179010853
:10A3A000436A70B504461868084B0D469847064640
:10A3B00008B1074B98470023F21A21462868054C3C
:10A3C00018BF0122A047012070BD00BF49960008B8
:10A3D0005DFE0108457B0108436A70B504461868B4
:10A3E000084B0D469847064608B1074B984700238F
:10A3F000F21A21462868054C18BF0122A047012007
:10A4000070BD00BF4996000885FE0108457B010824
:10A41000436A2DE9F74F07461868254B8846984749
:10A42000002841D0D0F87861DFF8A8A03369DFF8C0
:10A430009C909D68C5B15C690CB90120D04704F1BE
:10A4400040001C4B984778B1D0F810B01A4B4846E2
:10A45000984783452B46ECD100232246009339468A
:10A460004046164CA04720E0154B10209847154A4F
:10A47000154B0146044615489847002814DBD6F8CA
:10A480006C31A568DB69AB62304605F130022946C4
:10A490000F4EB047002807DB074B0C48984705F1E3
:10A4A00040022946B047D7E7002003B0BDE8F08F4F
:10A4B00049960008718202081DD80008159F0008FF
:10A4C000E94B0008C8320020E1C50008002E00203A
:10A4D00019820208154C0008436A37B5044618680B
:10A4E000084B0D469847002348B100F1380200930D
:10A4F000214600232846044CA04703B030BD1A462D
:10A50000F5E700BF49960008159F00082DE9F341C3
:10A510000C4602AB416A002203F8012D204606C911
:10A520001E4CA0478046A0B30569D5F8203113B969
:10A5300001201B4B9847D5F820412423013C03FB05
:10A5400004F202F148072A442F44D16C2A6C91424C
:10A550001E4602D00120124B984706FB045393F984
:10A560006830002B02DB01200D4B9847242303FBAE
:10A57000045494F86830C4F8648043F0400384F8CD
:10A58000683097F8203023F0070343F0040387F87E
:10A590002030012002B0BDE8F08100BFE5A0000836
:10A5A000154C000870B588B008AB0C46416A204EC7
:10A5B000002203F8152D054606C92046B04703467C
:10A5C00000282ED09DF80B204069E2B1DA6C1369A7
:10A5D0000393D169136AC91A93690491597A059151
:10A5E0009B7A06939368C31A1B1107931423019354
:10A5F00003AB009320680F4C002301222946A0479B
:10A60000012008B070BDDA6AD96B03921A6A521A37
:10A6100004925A6B1B6C517A0591927A06921B1A1E
:10A62000E2E7024629462068034CA047E8E700BF5E
:10A63000E5A00008A1790108457B0108F7B5446A47
:10A64000134F02AB0D46002203F8012D064694E895
:10A6500006002846B8470F4F10B19DF807303BB1B0
:10A6600000231A4628683146B847012003B0F0BDE0
:10A67000A168C26B0A440262E168426902EB0112FE
:10A680000264826A22F0005282620122EAE700BF7D
:10A69000E5A00008457B01082DE9FF41436A0E460D
:10A6A0001968044661B9154BC3F8B011012221465F
:10A6B0003068134C0023A047002004B0BDE8F081AF
:10A6C000104A114B68469847002815DB0B4FDDF800
:10A6D0000880D7F8B03163B11A69D8F810509542A4
:10A6E00003F1180108F1180034BF2A011201074BC9
:10A6F0009847C7F8B081D9E70022D8E7002E00209C
:10A70000457B0108E031002059610208CF010308B0
:10A710002DE9F0439BB0456A574C1AAB0F46002217
:10A72000064603F85D2D384695E80600A047002848
:10A7300000F08D809DF80B2052B1C36C03F110081E
:10A74000A968012907D01CD3022923D000207EE06C
:10A7500000F12C08F4E792B1C36C5C68D8F80830BB
:10A760005B7AEA689342F1D9022904EB021459D0CA
:10A770002046424B9847002856D1814646E08469DE
:10A78000ECE72AB1C36C1C68D8F808309B7AE8E77C
:10A79000C469F9E7436922B1C26C94681B1B1B11A1
:10A7A000DFE71C46036CF9E7D8F80820D8F8041056
:10A7B000334B0EA89847334D0AA90EA8A84709F1B4
:10A7C000FF33B9F1000F2BD12F492278182000FB5D
:10A7D00002125379042B06D19DF8303000FB03138D
:10A7E0005B79032B36D90DA9284B14A89847179BE2
:10A7F000DB8A03F03003302B01BF15AB93E8070071
:10A8000003AD85E8070014BF0020284600902246CB
:10A810004B46314638461E4CA04718E08146CAE7F1
:10A820009946C9E70020A8E7AB68D5F80C90012B42
:10A83000BAD10EA8174BD8F80820D8F804109847BA
:10A84000129B9B0609F10100E8D50028B3D11BB08B
:10A85000BDE8F0836368012B02D001200E4B9847BE
:10A8600094E80F0006AD85E80F009DF830308DF8B4
:10A870001830A1462C46B6E7E5A000087D910008F7
:10A88000B91202083D3002083055030825170208A6
:10A89000159F0008A1120208154C00082DE9F0438D
:10A8A000456A95B00E4629680391074651B36B6817
:10A8B00043B30EA8444B9847002803DA002015B094
:10A8C000BDE8F0830FAB93E8070004AC84E8070011
:10A8D0006A68DFF8109102F1FF380599049BCA6F8E
:10A8E00006981FFA83FE02EBCE02417D5288521A6F
:10A8F000904524D3418AA8EB02021B0C0A441B0496
:10A900001343AB6005F1080807AA414630462F4BB8
:10A9100098470028D2D0039CB4B940462C4B9847A6
:10A92000039003982B4B984700283ED100230093B7
:10A93000039A234639463046274CA047BFE72046B6
:10A94000C8470028C9D1B9E76B683BB9089BBDF877
:10A950001C20D3F8803033F812306B606B68002B0A
:10A96000ACD02378133B012B05D903A920461B4B00
:10A9700098470028A2DB039C2278102A0FD80123D5
:10A98000934013F4C63F0AD0E368A2680D930C20ED
:10A9900001210AABCDE90A010C920393C1E76B6870
:10A9A00004EB031403940024BBE707A90EA80C4B87
:10A9B00098470028BADB119BDB8A03F03003302B69
:10A9C000B4D10FABB3E700BFD517020885A00008CC
:10A9D00079C100087D910008159F0008155F0208E5
:10A9E00025320208FD1402082DE9F043D0F8248036
:10A9F0008FB006460F4612200121D8F80030089388
:10AA0000CDE90601204BD8F8042006A90AA89847EA
:10AA1000002832DB0C9DAC7D2CB3D8F804206C7D73
:10AA200002FB045418344FF000082046174B984797
:10AA300078B10DF10C0905F10C014846144B98470B
:10AA400038B1059BDB8A03F03003302B0CBF48463E
:10AA50000020009022464346314638460D4CA04720
:10AA60000FB0BDE8F0830AA906A80B4B9847002851
:10AA700007DB4FF0FF3806ACD7E7002080460446DE
:10AA8000E7E72046ECE700BF254F02087D9100086C
:10AA900095130208159F0008C14F020813B5426ABA
:10AAA00000230C460093014612682046014CA04743
:10AAB00002B010BD159F0008436A37B504461868F8
:10AAC000054B0D4698470023024621460093284631
:10AAD000024CA04703B030BD0D940008159F00083C
:10AAE00038B5436A0D681979044603F108021868FD
:10AAF000044B98472146024600232846024CA047B3
:10AB0000012038BD71930008457B0108F0B5446A07
:10AB100089B02268029205460F4612200121CDE934
:10AB2000000102B3967D36B96268134B694604A8EA
:10AB30009847002801DA002215E004A968460F4B67
:10AB400098470028F7DB04F108029DF800100C4B31
:10AB5000684698470028EED0324604A96846094B5B
:10AB60009847C243D20F3868074C00232946A047B4
:10AB7000012009B0F0BD00BF254F0208C14F0208F7
:10AB800071930008F9520208457B0108F7B5466A3F
:10AB90000C4B054630680F469847044648B90024D8
:10ABA00000232246009329463846074CA04703B0AD
:10ABB000F0BD0146321D0548054B98470028EFDAE5
:10ABC000EDE700BF0D940008159F0008002E00203F
:10ABD000E1C500082DE9F341446A114B05462068A0
:10ABE0000F469847064650B9002600230093324688
:10ABF000294638460B4CA04702B0BDE8F081616899
:10AC0000094B98470028EFD083686268DFF81C8002
:10AC100020211846C047626800218154E5E700BF43
:10AC20000D940008159F0008E17502081902030839
:10AC3000F0B5446A0F4B85B0064620680F4698472A
:10AC4000054670B10223ADF80830A368ADF80A30AC
:10AC50006368039302AAE168074B98470028B8BFCE
:10AC60000025002300932A4631463846034CA0476E
:10AC700005B0F0BD0D940008B5600208159F0008EE
:10AC80002DE9F04F436A5C68A3B00746894654B982
:10AC9000002400232246009339464846384CA047FA
:10ACA00023B0BDE8F08FD3F80080DFF8FCB01222AB
:10ACB000012302ADCDE90223294606A8314B4FF00E
:10ACC000000ACDF810A098470AA92046D847061ECA
:10ACD0002EDB16A94046D847061E29DB9DF85C30BE
:10ACE0005BB19DF82E30002B47D0524621462846B6
:10ACF000254B984700EAE0761AE041462846234B68
:10AD00009847061E14DB9DF82C30DBB19DF85E30B1
:10AD100043B1039B012B11D195E80F00002684E875
:10AD20000F0005E019A92846194B9847061EF0DACE
:10AD300006A8184B9847002EABD0A9E70120164B68
:10AD40009847E9E72846154EB04770B12046B0470E
:10AD500020B129462046124B9847CBE70C4B19A946
:10AD600028469847061EF4DAE2E72046B047002856
:10AD7000EFD019A928460B4BF3E74FF02246D7E74F
:10AD8000159F0008C5DF0008F9520208C14F0208EC
:10AD90000551020809E00008154C00084994000814
:10ADA0001154020825520208D5920008F0B50D464C
:10ADB0000F49C3B00022D1F80061134602AF96429A
:10ADC00009D051F8224024B12469240447F82340D3
:10ADD00001330132F3E79B00019302AB009301467C
:10ADE00000232868034C0122A047012043B0F0BD96
:10ADF00080300020A179010830B50F4BADF20C4D29
:10AE00000D46D3F8D42002A9002394683CB1126AFD
:10AE100041F823200133B3F5807F2246F5D19B0012
:10AE20008DE80A000122014600232868034CA04750
:10AE300001200DF20C4D30BD002E0020A17901083B
:10AE40002DE9F043436A0D46ADF5457D1968224B67
:10AE50000646284698470446002835D002AF037FAF
:10AE60003B60436BDFF87C90D3F808804046C847CE
:10AE70000130B0F5FF7F16D84046C847431C424614
:10AE80004FF4007103A8DFF86080C047616A83A8AF
:10AE900000228B6853B189690969090440F8041BD1
:10AEA00001321946F5E740F2FF13E8E781329200DC
:10AEB00001920097012231462868084CA0470120E2
:10AEC0000DF5457DBDE8F08303460246314628680E
:10AED000034CA047F3E700BF29960008A1790108B9
:10AEE000457B0108B55B0008895B00082DE9F0414E
:10AEF000436A0D46ADF5067D5988174B0646284630
:10AF00009847044608B3C269DFF8588003AF40F29F
:10AF1000FF134FF4007106A8C04763693B60A36943
:10AF20000E4C1C3393E8030004AA4FF4037382E829
:10AF30000300019300970023012231462868A047AF
:10AF400001200DF5067DBDE8F0810346024631463D
:10AF50002868034CA047F3E72DA00008A179010859
:10AF6000457B0108895B0008F0B50C46ADF5097D0D
:10AF70000546416A134B05AA20469847D0B140F2D6
:10AF8000FF13049308AE04AB03AA05A90E480F4FA4
:10AF90000396B84700280DDB4FF400730193009629
:10AFA00020680B4C002301222946A04701200DF503
:10AFB000097DF0BD00232068064C1A462946A047AB
:10AFC000F4E700BF55A0000880300020F13A0208E5
:10AFD000A1790108457B0108F0B50C46ADF50D7D62
:10AFE0000546416A1B4B04AA20469847002829D0F1
:10AFF0000CAB029340F2FF13039302AA03AB04A924
:10B000001548164FB84700280AAE1BDB04A9144B9D
:10B0100007A89847079B3360059BBDF81020D3F81D
:10B02000803033F8123073604FF40273019300964E
:10B0300020680C4C002301222946A04701200DF571
:10B040000D7DF0BD00232068074C1A462946A04715
:10B05000F4E700BF85A000088030002049400208C6
:10B0600011140208A1790108457B0108F0B50C46CE
:10B07000ADF50D7D0546416A184B05AA2046984757
:10B0800020B105A908A8164B984748B900232068A5
:10B09000144C1A462946A04701200DF50D7DF0BD40
:10B0A0000CAB039340F2FF130493089B0B93079B95
:10B0B000069819880C4B0D4F984704A903460C4A73
:10B0C00003A8B8470BAE4FF40173019300962068B4
:10B0D000084C002301222946A047DDE7B5A000085F
:10B0E000C9130208457B0108ADFA0108154901089A
:10B0F0001C100308A179010870B5456A86B00023C9
:10B10000039304460E4668680D4B04A9984700282F
:10B1100008DB2A4605AB04A90A480B4DA84708B12D
:10B12000059B03930423019303AB009321463068EE
:10B13000064C00230122A047012006B070BD00BFCD
:10B14000651902080C2C00200D4C0208A179010899
:10B150002DE9F04FA84BD0F824908FB09846089076
:10B160001868099118B30EAB00240B940C9443F8A3
:10B17000044D056A0CAA0BA9A847002840F02381BA
:10B180000D9D002D00F01F810B9C0C9B27681A461B
:10B1900003EB85010646914203D052F8040B0644A6
:10B1A000F9E7D9F8001001290CD002294AD000246F
:10B1B00009980194009423462246089900688F4D0F
:10B1C000A84700E12B1DDB00049318468C4B9847E1
:10B1D0000446002800F0F780049A8A4B0021984723
:10B1E000894A0C98D2F80C21A66084E884004FF0BC
:10B1F000FF3204F120032261D8F808206261A261C5
:10B20000E3610022AA4203F1080308DA50F8221091
:10B2100043F8041C43F8087C01320F44F2E7002392
:10B22000E360049B002BC2D0099801930094002393
:10B23000012208990068714DA8472046734B984732
:10B240000120C1E0D9F804200392D9F80820059222
:10B2500000220292029A029954F8222053F82110F7
:10B260000A4403999142029A01D30132F1E74FEA6D
:10B27000820800224344924605998A4205DA53F82F
:10B280002A100AF1010A0A44F6E70AF10403DB0076
:10B290000493184601215A4B98470446002800F0B1
:10B2A0009280584B049A0021984704F12003E361EF
:10B2B000554BD3F80C31A66084E888004E4F029EAF
:10B2C0004FF0FF3323610DF1380BBB686361A3615D
:10B2D00001230BF80D3D029B53440693059BC14689
:10B2E0001D46069B9E429DF82B3010D08BB1002D41
:10B2F0000DDD38683146C3695A4698470C9B53F8B0
:10B300000930EB1A1D46013609F10409E9E7002B63
:10B3100040D10027DFF8E0900697B846BA4568D0DC
:10B32000029B0C9A0399FB1852F82360E36903EB24
:10B33000C70243F8371099F804305660002B3BD011
:10B340000023DDF80CB00793079BB34241DA059B5D
:10B35000002B3EDD99F80430002B38D1D9F80000DD
:10B36000036932461D4659464346A8474046284B86
:10B37000069A31469847079B069033440793059BEE
:10B380009B1B059399F80430002BB34418BF4FF072
:10B390000008D9E70C9B984400239A4527D0E1691F
:10B3A00058F82320039D41F8335001EBC3000133CB
:10B3B0004260AA180392F0E701213046104B9847EB
:10B3C00080460028BCD100200FB0BDE8F08FD846E1
:10B3D000CCE799F8043013B940460C4B9847039BCF
:10B3E00033440393059B002B03DD013796E70023CD
:10B3F0000693069B14E700BFD0330020A179010813
:10B400008D4B00081902030880300020594B0008BA
:10B410006D8602081FB514460E4B01AA984780B1ED
:10B42000039B5A884FF6FF739A4210D0029BBDF8D7
:10B430000420D3F888108B5C2CB143F001038B54AB
:10B44000204604B010BD23F001038B54F9E700201F
:10B45000F7E700BFB5A000082DE9F04F87B092468E
:10B46000134B03AA81468B4698470746D8B1059EE1
:10B47000DFF84480737B347B1C44B37B1C440D4B4E
:10B480000025A5420FD0DBF80020718901932944E3
:10B4900002EA08020A43029202A952464846984725
:10B4A0000135019BEDE7384607B0BDE8F08F00BFDE
:10B4B00055A0000815B400080000FFFF2DE9F34770
:10B4C000456A2E686B68003618BF0126022B0F46AE
:10B4D0001FD0052B26D0012B2AD16989164B38465F
:10B4E0009847044620B3DFF85CA0DFF850904FF097
:10B4F0000008636B98451DDAAB6803EA0A0343EA68
:10B500000803324601A93846019308F10108C847EB
:10B51000EFE70A4B324605F108013846984702B07A
:10B52000BDE8F087324605F108013846044BF5E7DF
:10B530000020F4E70120F2E72DA0000859B400082C
:10B5400015B400080000FFFF0123037070470000DE
:10B5500073B50646074B68460C4698473568064B58
:10B5600025421CBF25EA04043460684698472846F3
:10B5700002B070BD097501084175010813B5084B8B
:10B5800000241C605C606846064B9847064B684682
:10B590001A681C60054B9847012002B010BD00BF1F
:10B5A000E833002009750108DC33002041750108EB
:10B5B00008B50248024B9847012008BDE833002037
:10B5C0007D8E000813B50A4B044668469847094B20
:10B5D0001A68144204BF14431C606846064B98471F
:10B5E000064B1B6813B1064A1068984702B010BD9D
:10B5F00009750108DC33002041750108E0330020A3
:10B60000E433002010B5C1430446024B024898477A
:10B61000204010BD51B50008DC3300202DE9F04F6B
:10B62000224B234DDFF8ACB085B0824688461046E9
:10B63000002198471F4B064602A80F469847A84787
:10B6400036184F414FF00109DBF8004018EA0404B6
:10B6500024D1A847B94208BFB0421FD2B9F1000FA8
:10B660000DD00220144B984748B902A8134B9847B5
:10B67000134B9847134A814602A89047E4E70023FA
:10B6800001935246304639460F4BCDF8008098471B
:10B6900002A80E4B98474FF00109D5E702A80C4BC2
:10B6A0009847204605B0BDE8F08F00BF490E02085C
:10B6B0008D0E020809750108795E00088974010879
:10B6C000F590000825750108118F0008A574010880
:10B6D00041750108DC33002070B50B4C0B4B05465F
:10B6E00020460E46984775B10123237620462A4608
:10B6F0000749084B98474FF47A7171432046064B2F
:10B70000BDE87040184770BDE83300207D8E00080A
:10B7100049B50008E9900008558E00080A46014B1B
:10B720000021184719020308C268836802B19360B8
:10B7300003B1DA607047000038B50C46054650B1D9
:10B7400049B1884207D0044B08469847EB68E3604C
:10B75000A560EC609C6038BD29B70008C2688368AA
:10B7600002B1936003B1DA600023C3608360704765
:10B770002DE9F04F2E4B00255C68D3F800A0002D7A
:10B7800008BF292C85B083464ED301220023CDE982
:10B790000223002600270F23AB426FF0100208BFE0
:10B7A000A2424FF0C86227BFA046A9466FF00F081B
:10B7B0004FF00F090023B242BB412FDB4FF42002B0
:10B7C0000023B242BB412CDB4FF480120023B24273
:10B7D000BB4104DA4FF480620023CDE90223DDE9A6
:10B7E00002235046CDE90023124942464B46884782
:10B7F00051460BF59270104B9847B4EB080465EB7B
:10B80000090516EB080647EB0907002D08BF292C90
:10B81000C244C0D2002005B0BDE8F08F4FF0FF3227
:10B82000DAE74FF42052D7E74FF07A40F3E700BF52
:10B83000042A00207580020839B700080148024B2D
:10B84000184700BFD42B00209544010870B50E4C5A
:10B850000E4B0F4D06460121002098472046A84771
:10B8600000232046A365E365A8471EB1094BBDE848
:10B8700070401847084B9A6842F001029A601A68B3
:10B8800042F000521A6070BD083000209D6D000823
:10B89000CD4601085DF90108002E002010B5054CC9
:10B8A00023685A1C22601BB9034B9847C4E9020164
:10B8B00010BD00BF083400208D0E020870B50A4E7E
:10B8C00033687BB1013B336063B9084B9847D6E9D5
:10B8D0000423D6E90245121B63EB050312184B4102
:10B8E000C6E9042370BD00BF083400208D0E020895
:10B8F00070B5084D2C6814F00064064608D1064B5C
:10B90000064898476B68C6F8344123F002036B6021
:10B9100070BD00BF002E0020EDE90008C02F002000
:10B9200070B50446074D00F5D870A84704F5D270ED
:10B93000A84704F59E70044B98470448044BBDE8A3
:10B940007040184779EA0008F94C020808300020D6
:10B95000CB4601080B680020996869B15A6A120742
:10B9600008D5D3F858319A6822B15B6D83F840004E
:10B970001346F8E70B46EFE7704700002DE9F04764
:10B980000C68DFF83490DFF834A0074690460026B4
:10B99000A56875B1A069C84748B9B8F1000F03D0D0
:10B9A000214607F5C670D047A36983F840602C464E
:10B9B000EEE7BDE8F08700BFB925020839B70008F7
:10B9C0002DE9F0411D46D0F8A0318AB006468846E0
:10B9D000144613B901201E4B98472B68019314B9E4
:10B9E00001201B4B984701A9A0691A4B98470546AF
:10B9F00038B3122201230027CDE9022302A906A8A9
:10BA0000154B049798473A4601A902A8134B98474B
:10BA1000B842134F13DB0499D6F8A001C1F828806F
:10BA2000104B984700280ADBD6F8A0310E4AC3F81D
:10BA3000242106A8B84728460AB0BDE8F08106A828
:10BA4000B847236943F0010323610025F3E700BFF2
:10BA5000154C0008F52B0208C5DF0008ED67020849
:10BA600009E00008F9FB010859BE00082DE9F04182
:10BA700006460B4D086890460127846874B1836AB6
:10BA8000D6F8B81143448362D0F86C31DA69C2F158
:10BA9000050207FA02F2A8472046EEE7BDE8F0816A
:10BAA000D1FB0108D0F8B831013B8B627047000030
:10BAB00038B50868064D0C4683683BB1426A920768
:10BAC00002D4A8472068F7E71846F5E738BD00BF5D
:10BAD00041FF0108F8B5064E064D0F463C68A368C5
:10BAE00023B12046B0472046A847F7E7F8BD00BF7E
:10BAF0005DB70008550002082DE9F041012300253B
:10BB000080F8B431C0F8B05105611E4B1E4EDFF80D
:10BB1000A480044698471D4B98471D4B984704F551
:10BB2000C270B04704F5C870B04704F5AC76314632
:10BB3000204604F5B277C4F89C51C4F8A051C4F86B
:10BB4000AC51C04739462046C04731462046114EC9
:10BB5000B04739462046B04704F5B8712046B04793
:10BB60000D480E4B98470E4B0E4898470E4B984782
:10BB70000E4B9847C4F8A85104F594700C4BBDE8DF
:10BB8000F0411847F9950008A54C0208C177010853
:10BB90008D450108D5BA000880300020012D02082B
:10BBA000514A02080C2C0020A5FA0108F96C020881
:10BBB000934C0208B1BA000808B50248024B9847F6
:10BBC000002008BD002E0020F9BA000870B510460C
:10BBD0000C46184B15469847214651F804498C42AB
:10BBE0000DD0D5F86C31DA69AB6A1A44A16831B16D
:10BBF000D4F86C31A06ADB6903449A4218DD6FF017
:10BC00000041002605F598734FF0FF30C5F82C6110
:10BC1000C3E90001D5F8501121B10748074B9847F7
:10BC2000C5F8506129462046054BBDE870401847CD
:10BC30000C46DBE75DB700080C2C0020A54A020883
:10BC400039B700080B6A70B50C46032B26D8DFE81D
:10BC500003F0020C13184B6ADB0706D40A46104B9C
:10BC600000F5AC71BDE870401847214600F5B07092
:10BC70000C4BBDE87040184708460B4BBDE87040C0
:10BC8000184710F5B47509D0A94207D0074B0846EC
:10BC90009847AB68A360E560DC60AC6070BD00BF36
:10BCA000CDBB000839B70008ADFF010829B700086F
:10BCB00073B505460698114E0C4611461A46431CAC
:10BCC00008BFD5F87C01079B009304BF0130C5F87D
:10BCD0007C012346B047061E07DB2168084B284637
:10BCE00098470026304602B070BD20680028F9D081
:10BCF000044B984700232360F4E700BFC9FD010807
:10BD000045BC00085500020813460A6813B52AB15D
:10BD1000084B104602B0BDE8104018474FF0040E23
:10BD20004FF0FF348DE81040034CA047C043C00FD4
:10BD300002B010BDDFFB0108B1BC000870B5D0F83F
:10BD400048510446AB68BBB1EA69D20612D502225B
:10BD500004F5D6712046094B984768B1D4F8AC1168
:10BD6000074B28469847294604F5A270054BBDE8C5
:10BD7000704018471D46E5E770BD00BF09BD0008CB
:10BD80003178020839B700082DE9F043052285B063
:10BD90002A4B06460D469847002843D02B681C6B5B
:10BDA0003CB36369009313B90120254B984769465A
:10BDB00001A8244B984710B90120214B98470299BC
:10BDC000A06A214B9847074610B901201C4B9847A1
:10BDD000BA69029B9A4202D00120194B9847009BF6
:10BDE000A16A1A4C013300933A466B463046A0478D
:10BDF000C0B9174BDFF85490D3F8D440A768C7B147
:10BE0000626AD2F80880B8F1000F0ED01369DB0720
:10BE10000DD493691B691B040193214601AB304685
:10BE2000C84720B105B0BDE8F0833C46E6E742468E
:10BE3000E7E72868074B9847F4E700BF09BD00080B
:10BE4000154C0008191602089D210208C1B9000806
:10BE5000002E0020550002080249034BA1F5D070C6
:10BE6000184700BFA02F002089BD00082DE9F04130
:10BE7000D0F89051AB6888B00446002B34D06946A6
:10BE800004A81B4B122601274FF00008CDE90067DC
:10BE9000CDF808809847AB69C4F8E030012204F57A
:10BEA000CE712046134B9847D8B1424605F1140194
:10BEB0006846114B9847404513DB02992B690B628A
:10BEC000C1E906670D4BD4F89C019847404508DB53
:10BED0000B4B0C4829469847D4F89C310A4AC3F8C2
:10BEE000242104A8094B984708B0BDE8F08100BFA1
:10BEF000C5DF000809BD0008ED670208F9FB01086D
:10BF0000A54A02080C2C002059BF000809E00008CF
:10BF100038B501230446C0F838310B4B0B4898471D
:10BF20000023C4F83831C4F8343194F8D1300546D0
:10BF300023B1074A536843F0020353600448054B9A
:10BF40009847284638BD00BFE1E50008C02F002013
:10BF5000002E00206DBE00080148024B184700BFAC
:10BF6000002E00206DBE0008D0F87C310133C0F8EF
:10BF70007C311846704700002DE9F74F1C46D0F879
:10BF800038310C9D012B06468B46914602D114F4A4
:10BF9000806715D0DFF8C0A04FF00008630714D504
:10BFA000DBF808E0DEF80C704FB370462B462246F3
:10BFB0004946D047BE460028F4D003B0BDE8F08F14
:10BFC0001F48204B98473846F7E7D6F8340168B940
:10BFD000DBF80070BB6801938BB12B4622464946C3
:10BFE0003846D04748B1C6F83471E6E72B462246BA
:10BFF0004946D0470028EBD0DFE7019FEAE700235E
:10C0000014F4C067C6F8343101D00020D5E7B8F188
:10C01000000F05D130460C4B98474FF00108BDE7A3
:10C020002C01084B0948224629469847084B9B6932
:10C030009C42EAD8074A536843F002035360C2E7C0
:10C0400070160308754A010811BF0008B9160308E5
:10C05000C02F0020002E0020457F02082DE9F34765
:10C0600099468B68144DDF7BDFF850A018247C4381
:10C070002E1990467379534327331B0900931522D9
:10C08000002300F59471D047034680B100F1080207
:10C0900099E8030082E80300C3F810801F757279E5
:10C0A0005A752A5982F40032C2F340429A751846F2
:10C0B00002B0BDE8F08700BF3055030879BF000823
:10C0C000F7B51E46A1F11303012B04460D46174692
:10C0D00002D90120094B9847089B009304F59471FD
:10C0E000204647F48073064C2A46A047044610B108
:10C0F0003146044B9847204603B0F0BD154C00086C
:10C1000079BF0008FD4E0208F7B51F46A1F11303E1
:10C11000022B04460D46164602D80120064B9847CE
:10C1200004F59471009726F001032A462046034C3B
:10C13000A04703B0F0BD00BF154C000879BF000850
:10C1400010B4034C0F33A4461B095DF8044B604741
:10C1500009C1000813B5074C009342F005030A46D5
:10C1600000F59471A04710B100238360C36002B052
:10C1700010BD00BF79BF00081FB501460F4B01A8D5
:10C18000984718B9002005B05DF804FB039BDB88D5
:10C19000DB06F7D50A4B0299D3F8E000094B984724
:10C1A0000028EFD0029BBDF80420D3F88030C0698E
:10C1B00033F8123000EB0310E5E700BF6515020805
:10C1C000002E00209D2102082DE9F04F0123144686
:10C1D0001222C1E90023584D00238B608346D5F815
:10C1E000A4302068A26898420E4689B0D17B00F046
:10C1F0009D8018234B435148C05810F4803008D11B
:10C200000023CAB243F00103C6E9002309B0BDE828
:10C21000F08FA1F11103092B00F28880DFE803F011
:10C220001D861F1F86868686860505A8444B98476F
:10C230000028EBDB2268D5F8D0309A42059B08BF76
:10C240005A694FF0120008BF42F000424FF001015E
:10C2500008BF5A61C6E90001B3600020D6E76368F1
:10C2600092F81590DB6F2288364F03EBC2035846D5
:10C27000B3F8028008F10105009523460022B84773
:10C280000746002855D012220123C6E90023B060DA
:10C2900094E8070005AB83E80700214638462A4B9F
:10C2A00098470028B2DB07EB05134FF0000A039311
:10C2B0005546B8F1000F2AD0B9F1000F09D105A8F1
:10C2C000224B984700282ED0079B002593F8159005
:10C2D000F2E75DB9DDF818A0079BDAF818505B8A21
:10C2E000EA6B4B449BB202EBC3031D44039B184F04
:10C2F000103B0393083D53462A4603995846B847D6
:10C30000002809F1FF3908F1FF38D2DA7EE720462C
:10C31000104B98470028A0D02146B0680E4B984794
:10C3200000EAE07072E74FF07F406FE74FF0224085
:10C330006CE74FF07A4069E79831002030550308E8
:10C3400005470108C1C00008FD4E0208FD1402089F
:10C35000E1C3000849150208C96A020830B589B06E
:10C3600005460C46104604A9194B9847002822DBC5
:10C37000059B002B2ADC9DF81820142A1DD1154B93
:10C3800007A901A89847039AD38A03F03003302BFA
:10C390000CD1D27BD2B20023002042F4807243F051
:10C3A0000103C4E90023A060E06004E001AA214683
:10C3B0002846094B984709B030BD18235343074915
:10C3C000CB5813F4803F18BF1222E3E71222E1E7B3
:10C3D0003D30020895130208C9C100083055030812
:10C3E00030B587B004460D4668461946044B984759
:10C3F0006A4629462046034B984707B030BD00BF28
:10C40000691202085DC300082DE9F04F91B0904613
:10C41000029191699A899B7A03900193886D99465C
:10C42000029B024403F1100500230A440093A5F186
:10C43000100AB9F1000F00F0C5804FF0000B5F4605
:10C44000164616F8014B162C0DD8152C10D2132CAD
:10C4500010D25D4A182303FB04239B68002B00F0D5
:10C46000AC801B6820E0452CF3D1A3463246E7E7B9
:10C470000137FBE73378190618D4961C03F0030242
:10C4800052498A5CC3F3970343EA0263190E0429F5
:10C4900023F07F424DD008291FD0012940F08D8024
:10C4A000D8F8703053F8223005932BE003F0C00128
:10C4B0008029707805D11B0203F47C530343D61CFA
:10C4C000DCE71B0603F0F851B3781B0243EA004394
:10C4D000F07803430B43561DD0E7D8F81820916C31
:10C4E0009BB201EB83031A4441460AA8384B984794
:10C4F00006A90AA8374B9847002860DB099B0593DB
:10C50000079B1F44DFB10123122245E90423BBF13D
:10C51000450F4FF0000345F8083C05D115F80F3CD6
:10C5200043F0080305F80F3C09F1FF391035324696
:10C530007DE7D8F8103042EA03420592E2E7142C76
:10C5400031D1254B05A90AA898470C9BDA7B142A00
:10C550000CD0D2B2002342F4807243F0010345E9CB
:10C56000042345F8087C45F8047CDDE7009B4BB1CB
:10C570000AAA51460398194B984700281FDB01234C
:10C580000093D1E7BDF80410029A102313FB013386
:10C590005B1B13445344524607200121E2E8040187
:10C5A0009342FBD8E4E718236343074AD35813F4B4
:10C5B000803F18BF1224E2B2CCE74FF0224011B006
:10C5C000BDE8F08F4846FAE7305503086C160308BB
:10C5D0001D1202083D30020895130208C9C1000867
:10C5E00030B585B004460D4601A81146064B984764
:10C5F00030B101AA29462046044B984705B030BD0A
:10C600004FF02240FAE700BF95130208C9C10008A5
:10C61000F0B5914285B00C46154623D002F10801D1
:10C62000A36892689A421FD1114B124F01A89847F4
:10C63000029BBDF80420DB6F03EBC2035E886B78BE
:10C64000DB0642BF637843F01003637056B11035C8
:10C65000103429462046B847002806F1FF36F5DA9F
:10C6600005B0F0BD0020FBE74FF02240F8E700BF27
:10C6700095130208115402082DE9F041804688B054
:10C680000E461446207800F0FB03122B05D1A46857
:10C69000002CF7D14FF0214522E0A0F11303012B2C
:10C6A00022D812220123CDE90023694604A8154BA4
:10C6B0000294984704F1080231464046124B134F4A
:10C6C0009847051E0ADB2246B168114B4046984741
:10C6D000051E03DB04A8B847002501E004A8B847FD
:10C6E000284608B0BDE8F081182343430949CB58D8
:10C6F0009B0204D511463046074B9847ECE74FF0B4
:10C700007745EDE7C5DF0008E1C5000809E000084E
:10C7100011C6000830550308457800082DE9F84394
:10C720000D680E4F81469046AB68ABB1D5F84041DD
:10C730001D46A668002EF7D0D9F8E020A36A9A42D9
:10C7400008D10122414604F11800B84710B1204633
:10C75000BDE8F8833446ECE71C46F8E79D5602082E
:10C7600070B50B78122B04460D4607D18B682BB1A0
:10C770001A78133A012A01D8D86870BD2A4604F500
:10C78000AC712046054EB04738B92A4604F5B2715F
:10C7900020463346BDE87040184770BD1DC70008ED
:10C7A0002DE9F84F8A46DFF84C90196893468D685A
:10C7B000D5B1D1F84021DFF8408096682946002E97
:10C7C000F5D0916B8F683246002FF6D00C695C452E
:10C7D00002D02269524509D14046C8474FF0FF3187
:10C7E0002046034B984708B1BDE8F88F3946E9E782
:10C7F00015FF0108A54A02080C2C00202DE9F04184
:10C80000044616460D4611B1D1F84C3113B98EB11C
:10C81000B3697BB1084F04F5AC7332462946204614
:10C82000B84704F5B273324629462046BC46BDE8F7
:10C83000F0416047BDE8F081A1C7000810B5034B87
:10C8400098470348034BBDE810401847B7FA010862
:10C85000D42B0020A5450108024B002283F81821A3
:10C86000704700BF002E002030B5A3B1D0E93E458F
:10C87000D1E90001844275EB01030FDA001B61EB83
:10C880000501D2E90045A04271EB050301DAC2E9D6
:10C890000001002030BDD0E93C45E9E7012030BD72
:10C8A0002DE9F04F85B00023D0F84841DFF85C80D7
:10C8B000019305468946A768CFB1E369002B14DAD6
:10C8C000D4E908AB04A961E902ABC3F340734A465B
:10C8D00028460B4EB047824638B10A4B1A685301BE
:10C8E00003D42046C047CDF804A03C46E3E7019BB3
:10C8F00013B12846044B984705B0BDE8F08F00BF40
:10C9000069C80008002E00203DBD00081978020803
:10C910002DE9F04F1468DFF888A187B006468B46F2
:10C92000A3680193002B00F0A180656A15F0010552
:10C9300040F09A8004F59877D7E9002306A961E9C9
:10C94000042330462B465A46D04748B16FF0004387
:10C950004FF0FF32C7E9002329462046484B98474D
:10C96000D4F8501169B100235A4610313046D047EF
:10C9700038B14FF48173C4F8543101212046404B43
:10C980009847D4F840319F68CFB19D6BDFF8149180
:10C99000D5F808803B46B8F1000FF4D000235A4682
:10C9A00005F118013046D04738B14FF0FF31286902
:10C9B000344B984729463448C8474546E8E7D4F8F9
:10C9C0006C51EF68002F4FD0D5E908896FF0004314
:10C9D0004FF0FF32994508BF904537D02B4BD3E934
:10C9E00004012B4B984710EB080041EB09010DF1B6
:10C9F000180E6EE9020100235A4671463046D047B0
:10CA000020B3D4F860312349DFF89C80002204F180
:10CA10003800C047AB6A13F0010119D143F001039C
:10CA2000AB620FF25409D9E90089D5E9082318EB64
:10CA3000020849EB03094B464246C5E90823164B59
:10CA400083F81811012120460D4B98473D46B8E761
:10CA50000222124B2946204698474FF0FF326FF0D2
:10CA60000043C5E90823EDE7019C59E707B0BDE89D
:10CA7000F08F00BFAFF30080404B4C00000000007F
:10CA8000E1FE010815FF01080C2C002008340020ED
:10CA90002D0E02082C320020002E002059FB010828
:10CAA00069C80008A54A0208D598010873B5274B44
:10CAB00004469847D4E93A23CDE90023244B1B6868
:10CAC000002B11DAD4F8642104F5B0739A420BD12B
:10CAD000204B5B6BDB0603D4D4E93A23CDE900237A
:10CAE000DDE9000102B070BD94F8183104F59075CD
:10CAF00063B1D5E90023D4E93C01904271EB030610
:10CB000004DA121A63EB0103CDE90023124B134E32
:10CB100069462046984704F5AC7269462046B047FE
:10CB200004F5B27269462046B047D4E93C01DDE91C
:10CB3000002312184B419042C5E9002371EB030317
:10CB4000B4BF0123002384F81831C1E73DC80008B1
:10CB5000002E0020D42B0020A1C8000811C9000815
:10CB600073B51E460B4B0D4614469847019040B1D5
:10CB700021469DF818300198074C3246A04702B074
:10CB800070BD2A462169054B01A898470028EFDAB5
:10CB9000F5E700BF61C7000819700208716F02084D
:10CBA00010B5044B144698472146034BBDE810408E
:10CBB000184700BF61C700089D71020830B5D2E96F
:10CBC000004501F59873C3E90045044B002283F842
:10CBD000182101230B624FF0424030BD002E00208F
:10CBE000F8B50E46D0F854111D4611EA0504174653
:10CBF000069B07D021EA05010122C0F854111A70E2
:10CC00000020F8BD1C700A4B9847D7E900239042DA
:10CC10009941F5DA06F59871C6F82C51C1E900235F
:10CC2000044B83F81841012333624FF04240F8BDB2
:10CC30008D100208002E0020D0F854312DE9F04765
:10CC400013430C68DFF840A0DFF84090C0F854317F
:10CC50000F46904600F5B275A66896B1D4F82C310F
:10CC600018EA030F0BD0AF4201D00120C847236A56
:10CC7000012B01D00120C84701212046D04734466E
:10CC8000EAE7BDE8F08700BFE1FE0108154C0008A7
:10CC900070B5074D04460E460A4600F5AC71A8472C
:10CCA000324604F5B27120462B46BDE87040184765
:10CCB00039CC00082DE9F041304E0D468AB00446CB
:10CCC0000021628A6B8A42B13BB121462046B047BF
:10CCD00029462846B0470121F3E7934203DD0020AF
:10CCE0000AB0BDE8F08119DA93B9254A6368D2F831
:10CCF000A400834201D10120F2E7906C8342FAD074
:10CD0000D2F8B0008342F6D0D2F8AC209342F2D0F1
:10CD1000E268EB68D27BDB7B9A42E0D1EB68DE8A8B
:10CD200006F0300629B1E368DB8A03F03003B34232
:10CD3000D5D1144FDFF8548062686B689A42DAD01C
:10CD4000202E15D1E26811894FF6FF7399420FD05A
:10CD5000A16804A8B847099B002B09DD694604A80F
:10CD6000C047002804DB6B68039A9A42F3D1C2E7FC
:10CD7000201D054B98470028DED1B0E70D190208A9
:10CD80009831002039120208FD1402083D300208D3
:10CD900030B58DB00D46094C01466846A0470028C5
:10CDA00002DA00200DB030BD294606A8A0470028B1
:10CDB000F7DB06A96846024B9847F3E725170208F8
:10CDC000B5CC000810B58CB00C460A4B014668463D
:10CDD0009847002802DA00200CB010BD214606A8B2
:10CDE000054B98470028F6DB06A96846034B984791
:10CDF000F2E700BFD517020825170208B5CC0008D6
:10CE000030B593B00D46154B014606A81446984719
:10CE1000002802DA002013B030BD2A4621466846B9
:10CE20000F4B984770B1009B079A9A42F3D00D4B75
:10CE300069460CA898470028ECDB0CA906A80A4B09
:10CE40009847E8E72A46214603A8084B9847002858
:10CE5000E0D003A90CA8064BECE700BFD5170208E9
:10CE60009514020825170208B5CC000859130208CA
:10CE7000E931020870B504461E462378122B084695
:10CE8000114606D1A36823B9002070BD4FF024409D
:10CE900070BD0246064D2046A8470028F4D1002E5A
:10CEA000F4D012220123C4E90023A06070BD00BFAA
:10CEB00001CE000870B5D2E90045002C75F10003E1
:10CEC0000E460CDA013508BFB4F1FF3F0ED14FF02A
:10CED000FF326FF00043C1E90023002070BD054B15
:10CEE000984700196941C6E90001F6E74FF025406F
:10CEF00070BD00BF8D100208002A10B50C4609DA7B
:10CF0000013216D14FF0FF326FF00043C1E9002328
:10CF1000002010BD42F2107382FB0323C1E90023FD
:10CF2000054B9847D4E9002380185941C4E9000112
:10CF3000EEE74FF0254010BD8D1002082DE9FF41AE
:10CF4000DFF8488005460E46002424272B699C42C2
:10CF500018D2696907FB04114B881B070DD51431E2
:10CF600001A8C04748B1029BBDF80420D3F888103F
:10CF70008B5C26B143F002038B540134E6E723F0C7
:10CF80000203F9E704B0BDE8F08100BF19160208FA
:10CF9000DFF894C0DCF80030DB042DE9F3410646ED
:10CFA000964630D4D0F8CC30042B2FD85F1C4FF0ED
:10CFB00024080C46C0F8CC7008FB03080FCC08F11D
:10CFC00018050FC50FCC0FC523682B60DCF80030A7
:10CFD00043F00043CCF80030BEF1000F06D0DEF87D
:10CFE0001C30C8F81C3001238EF82C30012F0AD1D8
:10CFF000094B1B68186830B1009706F1180324220A
:10D000000649074CA04702B0BDE8F081054B01205E
:10D0100002B0BDE8F0411847D02B00200600020006
:10D0200085790108154C0008002E002070B50646D1
:10D030000D46144603B9136A226DAA60E26A6A615A
:10D04000E26B991AA961013104D0934202D2012006
:10D05000044B98472269044B29463046BDE870408E
:10D06000184700BF154C000891CF0008F8B5D0F85C
:10D07000CC6007468E46E6B100F118050C460FCD90
:10D080000FC40FCD0FC4013E2B68236007F11800B9
:10D09000C7F8CC602EB9BEF8023043F48063AEF816
:10D0A00002302422724307F13C01034B98470120D0
:10D0B000F8BD3046F8BD00BFE50103082DE9F74F84
:10D0C0000C9D1C4607468846914600230093009A13
:10D0D0003B699A4233D2242303FB02FA7A6902EBBA
:10D0E0000A0B4DB13CB12869844204D00120154B94
:10D0F00001929847019A2C6934B1DBF80430E06959
:10D10000834201D0013311D1BBF8021019EA010F9B
:10D110000CD032F80A30A8F80030A8F8029045B1D7
:10D120000D9B094E2A4641463846B047009B0133C5
:10D13000CCE7224641463846044B9847F6E703B011
:10D14000BDE8F08F154C00082DD0000891CF0008E5
:10D1500010B504468CB024210E4B03A89847D4F890
:10D16000CC2000232421934206D001FB0340408BB6
:10D1700080050CD40133F6E7002301930093D4F823
:10D18000803120464FF4007203A9034CA0470CB035
:10D1900010BD00BF1DB70008BDD00008D0F8D430C6
:10D1A0002DE9F047012204469D681DB183F8402017
:10D1B0002B46F9E7204EDFF894A0012204F5C27156
:10D1C0002046B0472A4604F5C8712046B0471B4E9A
:10D1D00004F5AC712046B047204604F5B271B04763
:10D1E000174BD4F8D4005A6822F004022E465A6035
:10D1F0001D464FF00209876897B1037F012B08D1C4
:10D2000090F84080B8F1000F05D080F81C90D0470E
:10D2100046463846EFE76B6843F004036B60F8E777
:10D220003EB12046074B4FF0007198472046064B11
:10D2300098473046BDE8F0877DB9000855B9000829
:10D24000002E002091CC000851D10008E5250208ED
:10D2500009682DE9F04F4FF0010C4FF000094FF035
:10D26000240B8F68002F69D0026981F87491002423
:10D2700094420CD043690BFB04335D882E0531D5F5
:10D280005D68CB699D422DD181F874C11446D1F8F7
:10D290005831D3F808E0BEF1000F21D09A6A1D6B17
:10D2A000B3F82C80D5F8885022F000429A6215F825
:10D2B000088018F0020817D042F000429A62DA6C37
:10D2C00062B15569128AD5F8885015F8028018F0B5
:10D2D00002081FD09A6A42F000429A627346D8E769
:10D2E0003946BEE70134C3E7A045E8D045690BFBEA
:10D2F0000855B5F802A01AF0070F08D06E68B246BC
:10D30000CE69B24503D1AD681E6DB542D4D008F1E7
:10D310000108E9E7A045E1D042690BFB08225588E6
:10D320006D0708D0CD695668AE4204D11D6D926874
:10D33000013DAA42CED008F10108EBE7BDE8F08F2D
:10D340002DE9F04104468846144D00211746A847B0
:10D35000606920B1124B98470023636123616FB16C
:10D3600024267E434FF4006130460E4B984760619F
:10D3700020B1324641460C4B984727612046012197
:10D38000A8470A4D04F5AC712046A84704F5B271D0
:10D3900020462B46BDE8F041184700BF3DCF0008AE
:10D3A000594B00088D4B0008CF01030851D20008EB
:10D3B00030B58DB00C460546242103A80B4B984789
:10D3C0004FF0FF330593D4F87031002B4FF000037A
:10D3D00001930093B8BF80222346A8BF4FF40252A6
:10D3E00003A92846024CA0470DB030BD1DB7000868
:10D3F000BDD0000830B58DB004460D4603A82421E9
:10D40000064B984700220192009220462B464FF48B
:10D41000807203A9024CA0470DB030BD1DB70008B3
:10D42000BDD000082DE9F04F0B69CD68DB69D1F85C
:10D4300050808DB006460193EB6817465BB300231E
:10D44000002F14BF8B46AB4600934FF024094FF0DA
:10D45000040A3369009A9A421FD2736909FB023E9B
:10D46000BEF802305A0712D5DEF8042001998A422C
:10D470000DD113F4006FDEF8083011D0984506D8AE
:10D480002A6BAB8DD2F88820D35CDB070AD4009BD3
:10D4900001330093DDE7002AD1D10DB0BDE8F08F54
:10D4A0009845F4D8BEE80F000DF10C0CACE80F0065
:10D4B000BEE80F00ACE80F00DEF80030CCF800301A
:10D4C000ADF80EA047B150230B935A46002303A991
:10D4D0003046024CA047DAE72023F5E72DD00008BC
:10D4E0002DE9F04FCB688BB080460C46174603B150
:10D4F00012B90BB0BDE8F08FCE6BDFF87890961BB9
:10D5000000254FF0240B4FF0080AD8F81030AB423A
:10D51000EFD9D8F814300BFB053EBEF802301B07DC
:10D5200025D52269DEF80430D269934201D0013357
:10D530001DD1DEF81420E36A9A4218D1DEF81830C3
:10D540009E4214D1BEE80F000DF1040CACE80F00B0
:10D55000BEE80F00ACE80F00DEF80030CCF8003079
:10D5600022463B4601A94046ADF806A0C847013512
:10D57000CBE700BF2DD000082DE9F04F0F698FB029
:10D58000FB6902938B6A03921B0306460C4647D441
:10D590000D6D6B1E019398464FF0010900274FF067
:10D5A000240A4FF0010B33699F425FD273690AFB73
:10D5B000073EBEF8022019EA020F2FD0DEF8043031
:10D5C00002998B422AD112F40063DEF8081045D08C
:10D5D000236BA08DD3F888301B5C03F001038845D2
:10D5E00003D102F00702042A18D0BBB1BEE80F0035
:10D5F0000DF1140CACE80F00BEE80F00ACE80F0012
:10D60000DEF80030CCF80030039B0D932246002357
:10D6100005A93046194DADF816B0A8470137C2E745
:10D62000D7F8203113B90120154B9847D7F820516E
:10D630002423013D03FB05729846926C944202D06C
:10D6400001200F4B984708FB05754FF007096B6EDB
:10D65000D3F850804FF0FF3301939FE78845BED841
:10D66000019B8B4234BF00230123B8E7226A054B9C
:10D670002146304698470FB0BDE8F08F2DD0000806
:10D68000154C0008E1D400082DE9F04F0B69CF6B71
:10D69000DB69DFF8A8B08DB0054600930B6D0193F0
:10D6A0000C469046D71B00264FF024094FF0020A83
:10D6B0002B699E4238D26B6909FB063EBEF80230E8
:10D6C00099072FD5DEF8042000998A422AD1DEF886
:10D6D00008200199914225D1DEF80C20974203D30E
:10D6E000DEF8102097421DD31A0506D5226BA38DB4
:10D6F000D2F88820D35CDB0714D5BEE80F000DF10B
:10D700000C0CACE80F00BEE80F00ACE80F00DEF830
:10D710000030CCF800302246434603A92846ADF835
:10D720000EA0D8470136C3E7424621462846024BA1
:10D7300098470DB0BDE8F08FE1D400082DD0000867
:10D7400030B58DB004460D4603A82421064B9847FA
:10D7500000232046019300954FF4805203A9034C07
:10D76000A0470DB030BD00BF1DB70008BDD00008F8
:10D77000F0B58DB004460D461E4603A82421074B84
:10D780001746984720468DE860000023102203A921
:10D79000034C0B97A0470DB0F0BD00BF1DB70008AC
:10D7A000BDD0000830B58DB004460D4603A8242135
:10D7B000084B98474FF0FF3205920B9200220192DE
:10D7C000009220462B46102203A9034CA0470DB01F
:10D7D00030BD00BF1DB70008BDD0000830B50C46F5
:10D7E0008DB00546242103A8074B9847236D0B9362
:10D7F00000230094019344F2200203A92846034C1D
:10D80000A0470DB030BD00BF1DB70008BDD0000857
:10D810000346D0F8E000C3F8E0107047D0F8E0000D
:10D82000704700001068F8B50D4686681EB30022E8
:10D83000D0F8583111469F68C7B171B95C6DAC42E0
:10D8400009D19A6A42F000629A62436A012243F067
:10D850000803436211463B46EDE79C6A14F0006FF3
:10D86000F9D024F000649C620022F4E70AB1024B74
:10D8700098473046D9E7F8BD41FF01082DE9F0414E
:10D88000D2F85871DFF8508006460D46BC6854B196
:10D89000786DC04718B17B6DAB422746F6D14FF08B
:10D8A0007D40BDE8F08106F5AC7229463046084F50
:10D8B000B84706F5B27230462946B847054A0123F3
:10D8C0002B77536843F0040353602046BDE8F08192
:10D8D00025D80008002E0020B925020830B5144BC9
:10D8E00085B004469847134BC4E93C019847124B56
:10D8F000C4E93E019847D4F80831984215D0C4F8DD
:10D9000008016A46D4E93E010C4B0D4D9847D4F806
:10D91000480184684CB1C369002B04DA1B0702D0AC
:10D9200000226946A8472046F3E705B030BD00BF96
:10D930008D1002085D1002086D1002089D1002088B
:10D94000A179020800000000F8B545A3D3E900233F
:10D95000C0E93A23324B334E04469847002504F57C
:10D960009477C4F8080184F818513846B04704F594
:10D970009E70C4F83851B04704F5A470B04704F560
:10D98000AC70C4F85451B04704F5B270B04704F518
:10D99000B870B04704F5C270B04704F5C870B0471E
:10D9A000214BC4F8A4519847204B984704F1D40068
:10D9B000C4F8A851C4F8B051B0470123C4F8E4300A
:10D9C000C4F8E050C4F88051C4F8B85184F8B45198
:10D9D0002046174B9847002821DB1648164B9847DE
:10D9E0001648174B9847174B9847002817DB164BDC
:10D9F0009847002813DB04F1E0011448144B9847C2
:10DA000000280CDB2046134B9847134B984704F52E
:10DA10008074C4E90001114B384698472846F8BD88
:10DA20006D100208934C0208A1FA0108FD6B020870
:10DA300071B7000880300020D52C02080C2C002083
:10DA4000DD4902087D44010851770108E716030803
:10DA50000D200208DDD800083110020859480108DD
:10DA60000046C3230000000010B5064C064B4FF4DF
:10DA7000E071204698472046044B984700EAE07042
:10DA800010BD00BF002E00201DB7000849D90008B6
:10DA90002DE9F84FD0F8B831484EB3F1104F044695
:10DAA0000F46D6F8E09015DA03F1C043C0F8B8315C
:10DAB00000F5AC714FF0C042414DA8474FF0C04255
:10DAC00004F5B2712046A8474FF0C04204F5B87182
:10DAD0002046A847DFF8E4A0DFF80481002F6ADDC4
:10DAE0003368002B3EDBD4F8A051002D35D1D4F89B
:10DAF0005851AB683BB9334B504698473368D4F81C
:10DB00005851002B2EDBAB68002B3CD0D5F86C3184
:10DB1000D4F8B811DA692C4BC2F105024FF0010BB1
:10DB20000BFA02FB5A4628469847AA6AD4F8B8313D
:10DB3000A2EB0B029A42AA6201DAC4F8B821C047EC
:10DB40002846224B9847002828DAB0F1424F23D0CC
:10DB5000B0F1784F22D002231FE02B6A13B96B6A11
:10DB6000DA07C6D54FF0407573685B0706D52046C7
:10DB7000174B9847002818BF4FF00075C6F8E09083
:10DB80002846BDE8F88FD4F8642104F5B0739A42B2
:10DB9000E8D14FF08065E7E701232B62C0472946B3
:10DBA00020460C4B984720460B4B984720460B4B82
:10DBB0009847013F92E74FF00075D5E7002E00200F
:10DBC0006DBA00086DBE0008D1FB01082958010894
:10DBD0009DD1000845BC0008DDD80008ADCA00088A
:10DBE000B7FA0108F8B50446174B9847174B20467B
:10DBF0009847D4F8582104F5AA739A4206460F466E
:10DC000001D00020F8BD012871F10003F9DBD4F840
:10DC100064018268002AF4D0D0F82C114B0011D591
:10DC200000F59C71D1E90045B44275EB070309DAB0
:10DC300000240025C1E90045054B012198474FF01C
:10DC4000FF30F8BD1046E4E7DDD80008ADCA000893
:10DC5000E1FE01082DE9F04100F588750E461746F2
:10DC6000D0E93C01DDE906238018594142F21074E5
:10DC700092FBF4F4002C08BF0124C5E90001DFF891
:10DC80002C8001210020C04722463946064B3046F1
:10DC90009847012104460846C04700220023C5E9F1
:10DCA00000232046BDE8F0811DB600089D6D0008E8
:10DCB00013B5094B044698472046084B9847084A35
:10DCC0000023CDE90023074B00215A6B064B204669
:10DCD000984702B010BD00BF3DC80008DDD800085D
:10DCE00040420F00D42B002055DC000870B5084CD2
:10DCF000084D06462368002B08DA23689A0005D4ED
:10DD000023689B0302D43046A847F3E7002070BD88
:10DD1000002E0020B1DC00082DE9F04FDFF87CA1D7
:10DD20008DB0DAF80C314FF0000806469146CDF878
:10DD30000C805BB94848494B98474FF050444848DD
:10DD4000484B984720460DB0BDE8F08F464FB84786
:10DD5000041EF4DB454D2B6823F440632B602B68D5
:10DD600043F480632B6042460AF5867104A8404B59
:10DD70009847041EE3DB04A908A83E4B3E4C984795
:10DD80004FF0FF330093CDF804800223069A03A9D5
:10DD90003046A047041E394B08A825DB9847039B53
:10DDA000D3F860315A6B527A02BB3046B847041E32
:10DDB000C5DB06F5D0713046314BDFF8E480DFF883
:10DDC000E4A0DFF8E4B0984749463046C047041E57
:10DDD000B5DB2B689A0005D42B689B0302D4AB6893
:10DDE000D80719D50124AAE79847A8E79869254AD2
:10DDF000254B41469847041ED7DAA0E7B4F1007FCF
:10DE000008D196F8D030002BDED030461F4B1DE0F5
:10DE1000044694E7002492E72B68002B05DAD047EC
:10DE20003046B8470028F3DBD8476B68990708D518
:10DE3000174B304698472B681A0102D46B689B0732
:10DE400006D4B4F1407FD9D1124B30469847BBE796
:10DE50000120114B9847F4E7EF160308754A0108B3
:10DE600008300020CD460108EDDC0008002E00201F
:10DE7000ED670208C5DF0008B1BC000809E0000832
:10DE800089BD0008D83100205961020811BF00087F
:10DE9000F1B80008E5DB0008154C000880300020D0
:10DEA00091DA00089DB80008BDB8000870B50546B5
:10DEB000094C00F5C270A04705F5C870A04705F5EC
:10DEC000AC70A04705F5B270A04705F5B8702346C1
:10DED000BDE87040184700BFA54C02080B4619B1B9
:10DEE00002680121184610470120704710B40B4604
:10DEF00031B104681146184623465DF8044B1847B3
:10DF000001205DF8044B70472DE9F041204BD3F818
:10DF10004441ADF5087DE368002B32D0E26A002A67
:10DF200033D0A76A002F30D140F2FF1308AE194852
:10DF3000194D02930196A847E169184B03A8984729
:10DF40003A4603A905A8164B984760B101AA05A94E
:10DF500002AB1448DFF86880C04786F8FF71226A78
:10DF600011483146A847E36AA06A1049104A0028C0
:10DF700018BF0A4619690F48A84721460E480F4B9B
:10DF800098470DF5087DBDE8F0811C46C3E700BF4A
:10DF9000002E002014170308754A01081112020808
:10DFA000912F020880300020251703080D17030861
:10DFB000BA5E03082C17030808300020C946010880
:10DFC000F13A0208094B41601A68026018600023A8
:10DFD00083604B789B075DBF0623C3604B780223A9
:10DFE00056BF43F00203C3604B70704720340020DB
:10DFF00010B5044B41601C68046018600123826006
:10E00000C36010BD20340020054B02681A60C3684D
:10E010005B0741BF4268537823F002035370704797
:10E0200020340020836841680BB10868184719B193
:10E0300001220248024B1847704700BF0030002001
:10E04000EDDE000838B5044B044D1C681CB12046B9
:10E05000A8472468FAE738BD2034002025E00008EE
:10E060002DE9F843124F064696F84430F3B10023E9
:10E0700086F844300F4BD3F8285106F14008AB68BE
:10E08000002BF1D0EC69D5F820904C4508D263788C
:10E09000DA0701D55B0705D5636804EB0314F4E7E1
:10E0A000AD68ECE721464046B847F5E7BDE8F883A0
:10E0B000DDDE0008002E0020214B2DE9F041D3F8D1
:10E0C0003C41204FDFF880800026A568002D35D028
:10E0D0006269510005D5E36A1BB1637843F001031F
:10E0E00063706378DB0715D5002A04DAE26A12B19F
:10E0F0005378D8071AD5A36A43B15B7813F00103AC
:10E1000006D0E26A12B15378D90713D52C46DCE762
:10E11000A362FBE721463846C047E268A36802B124
:10E12000936003B1DA60E660A660EFE743F00103B5
:10E130005370E0E743F001035370E7E7BDE8F08177
:10E14000002E002008300020C94601088369B3F57D
:10E15000803F2DE9F041044603D90023E361BDE887
:10E16000F081114B114F124ED3F844110023CD68AA
:10E170004DB14A69520004D5CA6A12B13846B04757
:10E1800001232946F3E7002BE7D1A369B3F5404FFC
:10E19000E3D8E36901330A2BE36103D9054BBDE8FA
:10E1A000F0411847BDE8F081002E00200830002023
:10E1B000C946010809DF0008134B2DE9F047D3F8E1
:10E1C000D440DFF84CA0114E8146A768CFB1636AF6
:10E1D00009F14005D3F80880B8F1000F06D09A691C
:10E1E000D969526E2846D0474346F3E7216B28464B
:10E1F000B047616B2846B047A16B2846B0473C4604
:10E20000E3E7BDE8F08700BF002E0020DDDE000858
:10E21000EDDE0008F8B5084DD5F80061074600248A
:10E22000A64207D055F8240010B1FB6B6830984720
:10E230000134F5E7F8BD00BF803000202DE9F0473C
:10E240000446C36B2D4F0E4601F130004034984711
:10E2500006F138012046B847B84600252427D6F8ED
:10E2600020319D4206DA07FB05632046D96CC04782
:10E270000135F4E7D6F85851214FD5F80890B9F197
:10E28000000F25D0EB6C8BB19A695968527A204601
:10E29000B847EB6C9A691968927A2046B847EB6CDC
:10E2A0009968DA68521A12112046B8476B6BA9694F
:10E2B0005A7A2046B8476B6BE9699A7A2046B84784
:10E2C00069692A6C521A12112046B8474D46D4E7A4
:10E2D000D6F840118D6825B118312046C04729462F
:10E2E000F8E7D6F8501131B18A69054B2046203144
:10E2F000BDE8F0471847BDE8F08700BFDDDE000845
:10E30000EDDE000870B50968044D06468C681CB146
:10E310003046A8472146F9E770BD00BF3DE200083E
:10E320002DE9F047514BC363514B0364ADF5856D47
:10E330000446002380F844304E4D083004AF0DF100
:10E340000408A84780220AA938464B4BC4F820800D
:10E3500067629847206AA847256A666A083D0AD01E
:10E360004EB1AE4207D0454B30469847AB68B360DC
:10E37000F560DE60AE60424B424D98474248434BE9
:10E380009847D5F89001866826B1E36B103098471E
:10E390003046F8E720463E4B3E4EDFF8189198474E
:10E3A0003D4B204698473D492046B0473C492046D2
:10E3B000B04704F14006D5F8A4113046C847D5F857
:10E3C000B0113046C84794F8443043B1354B20462D
:10E3D000984794F8443013B10120334B9847D5F84F
:10E3E0008451324EDFF894A0D5F80890B9F1000FAF
:10E3F00012D02B695B78DB070CD4E36B05F11000BE
:10E400009847B54206D02846D047F368EB60AE6027
:10E41000F5609D604D46E7E794F8443013B120461F
:10E42000204B9847236A434502D001201E4B984752
:10E43000636ABB4202D001201B4B98470F4F1C4E12
:10E44000236A9D68EB68002B636A08BF0025AB4216
:10E4500004D02846B8472846B047F1E70023236296
:10E4600063620DF5856DBDE8F08700BFC5EC00085F
:10E47000D9EA0008934C0208BDEA000829B7000851
:10E4800045E00008002E0020D42B0020A145010803
:10E49000B9E1000805E3000815E20008582F002044
:10E4A000642F002061E00008154C00088C2F00202C
:10E4B000594B0008DDDE00082DE9F041194B1A4CDC
:10E4C0001A4E98471A4B9847D4F84801856815B1F9
:10E4D000B0472846FAE7D4F85801164E856815B1BA
:10E4E000B0472846FAE7D4F86401124E856815B1A2
:10E4F000B0472846FAE7D4F87051DFF838800E4F5D
:10E50000AE682EB12846C0472846B8473546F7E7DB
:10E51000D4F8D400094D846814B1A8472046FAE71E
:10E52000BDE8F081A3FA0108002E0020FD77020863
:10E530003D6D020891000208F9FD01082926020834
:10E540008168F8B5122601278A68A2B14D6901F1E8
:10E550003003114615F1FF35F6D353F8082CCAB134
:10E56000146A1CB1647814F001040FD0547844F09C
:10E57000010454700EE0094B094D9847094BD3F83C
:10E580002801846844B1A8472046FAE743E90467B4
:10E5900043F8084C1033DDE7F8BD00BFB9E40008CC
:10E5A000FD7F0208002E002070B50C4BD3F8282107
:10E5B00000231946956865B1146AD669A41B2144E5
:10E5C00094692A46E568002DF4D0646823442C46FB
:10E5D000F8E71B0141618361184670BD002E0020E1
:10E5E0002DE9F04F4F4C504BF3B005469847236848
:10E5F000002B62DD4D4B984706460F464C4B4D486D
:10E60000984728464C4B984728464C4B98472846F5
:10E610004B4B98474B4B284698474B4B28469847BF
:10E620002368002B13DD414B9847801B474B484E16
:10E6300061EB070198476A69AB6900F51C500F3020
:10E6400042F21071D21A90FBF1F14248B0472368B0
:10E65000002B43DDE42200213F4CDFF80C91DFF872
:10E66000F0A068460DF1E408A047E42200214046EE
:10E67000A0473A4BD3F82871BB6823B3FE693C6AC4
:10E680001F46A642F8D23378382B12DC5DF82320DF
:10E690007068152B02444DF823200AD1317D3829AA
:10E6A0000EDC72AB03EB810151F8E43C034441F80A
:10E6B000E43C736806EB0316E3E7002600279DE7BA
:10E6C0004846D047F5E7DFF8A490DFF884A01C4661
:10E6D0005DF824305BB90134392CF9D1204B9847CF
:10E6E0002B68A86901332B6073B0BDE8F08F182741
:10E6F00007FB04921B0152691A482146D047152C8A
:10E70000E9D1DFF86CB0002658F8263033B107FBAA
:10E7100006921B01526931465846D0470136392EC0
:10E72000F2D1D8E7BC3500209DB800088D0E020854
:10E73000514A02080C2C002021E30008B9E000082F
:10E7400041E50008A9E500084DE100082D0E02088A
:10E75000754A01083D17030819020308002E00201E
:10E76000BDB800088B1703086C1703083055030861
:10E7700089170308164B2DE9F041D3F82851154E9F
:10E780004FF01808AB68EBB1EC692F6A1D46BC422C
:10E79000F8D22378A3F11102272A0FD80C2218FBF4
:10E7A00003239A199B59506800F0010203B92AB15A
:10E7B00040100AB12258D35820449847636804EBAC
:10E7C0000314E4E70248044BBDE8F041184700BFDA
:10E7D000002E00203055030821B9000870B5056BE4
:10E7E0000446DDB1836A93E806000020A84203F1E5
:10E7F00010030BD053F8106CB14228BF314653F8C8
:10E800000C6CB24238BF32460130EFE76163044B13
:10E81000A2630021204698470023236370BD00BFF8
:10E8200075E700082DE9F04FADF61C0D06AB8362CD
:10E830008023C362694B04930024D3F82821046326
:10E840008146029227460DF1180B029B9B68002B14
:10E850004BD0029BD9691B6A03934CB9049BD3F834
:10E860002871BB68002B40D03C69A268002A35D0D3
:10E870008C4281BF3B6A039321460297039B9942D6
:10E8800041D24B7813F00C0F39D1D9F830307F2BAF
:10E8900006D94846524B01919847D9F828B00199BA
:10E8A00063680193631ACBF80C30019BCBF80840E6
:10E8B00004EB03139942CBF800100D464FF0000A09
:10E8C0002AD0019B3BB1039B9D4204D295F8018065
:10E8D00018F00C0873D04FF0000826E01F46C0E780
:10E8E00029463446C4E7A6685CE0D9F8303013B155
:10E8F00048463B4B98470DF61C0DBDE8F08F4B6822
:10E9000001EB0311BAE7C0D1029B9B6802939CE71D
:10E910006B6805EB03159A44039B9D4203D26B7809
:10E9200013F00C0FF4D04FF00108BAF1000FDAD059
:10E93000039B9D4203D26B7813F00C0F4AD14FEA30
:10E940000A13CA18CBF80420E268A66802B19660E0
:10E9500006B1F2600022E260A26005931A462046EA
:10E96000204B9847019A059B22B1E11838461E4B6F
:10E9700098470646B8F1000F0DD15246DBF800105B
:10E980000298194B9847864205D9436800EB031358
:10E990009E4238BF0646D9F8303001330BF1100BD8
:10E9A000C9F83030B468002C9AD1BF68BB68002B1E
:10E9B000AAD03E69B268002A92D11F46F6E76B687A
:10E9C000019A9A42B1D3019AD21A019205EB03152A
:10E9D0009A4476E76B6805EB0315A9E7002E002043
:10E9E000DDE70008E5010308FD8002080A4B1B680B
:10E9F000002B10B5044602DD0848094B9847094B27
:10EA000098472046084B9847084B9847636801335E
:10EA10006360002010BD00BFBC350020AA170308AA
:10EA2000754A01089DB8000825E80008BDB800082F
:10EA30002DE9F0410F4E04460D4618274FF00C0803
:10EA4000B5B12378A3F11102272A0ED817FB03834F
:10EA50009A199B59506800F0010203B92AB140107D
:10EA60000AB12258D358204498471034013DE7E7B3
:10EA7000BDE8F081305503080F4A0368516B8B42A3
:10EA8000F0B518D3916B8B4215D2966A146B0021A6
:10EA90008C4210D9621852081701F519F759BB4278
:10EAA00004D369688B4203D3511CF1E71446EFE7A6
:10EAB000EA6813440360F0BDC02F002002F1005249
:10EAC000013A002301EBC2028360C360026141612D
:10EAD0000B604B60704700002DE9F74F734ED6F87E
:10EAE0002480D8F810A0D8F814500446894606F1BE
:10EAF000040BB9F1000F2FD16B6873B9D8F80C3043
:10EB0000DA68002A00F0C880726AC2F810A0556165
:10EB1000D3F810A05D69736298462C6804F1100365
:10EB20002B606B68013B6B6003B9083D637843F071
:10EB3000010363702378162B07D061D8142B00F2E1
:10EB40008180132B79D2122BD6D1A468002CD3D07C
:10EB50006378DB07D0D4E9E7B9F1010FE6D9554571
:10EB60000CD1D8F808309B6883B1736A1D615D6170
:10EB7000D8F810A0D8F81450C6F8248004F1100377
:10EB8000AB6009F1FF33EB600835CFE796F844300E
:10EB9000002B31D108238022D01C01934FF48061D7
:10EBA000434B0092C00098479DE80C000746F8B11F
:10EBB000736A00F11801C3F810A05D613D4BC6F8FF
:10EBC00024809847336A043B0CD098420AD0C1682D
:10EBD000826801B18A6002B1D160DA68FA60BB6014
:10EBE000DF6097607762D7F810A07D69B846C5E707
:10EBF000013B4FEA6202CFD1012386F844307BE724
:10EC00001E2B2FD006D81C2B9FD01D2B7FF474AF4A
:10EC100018348BE7202B1DD0372B7FF46DAFE068C5
:10EC200000283FF469AF244B9847024600288CD156
:10EC30000146224B204698475EE76368103403F193
:10EC4000FF3956E7A37D002B3FF456AFD4F8109060
:10EC500018344EE7A368002B3FF44EAF0120184B49
:10EC6000984749E7A369DA0712D50023A360E36058
:10EC7000BBF1000F3FF440AF5C453FF43DAFDBF824
:10EC80000C30E360C4F808B0CBF80C409C6033E76C
:10EC9000D4F8149020342CE7736A0120C3F810A034
:10ECA0005D61C6F8248003B0BDE8F08FC02F00205E
:10ECB0008D4B0008BDEA0008B9250208E55E020890
:10ECC000154C0008006828B14378DB0702D4012105
:10ECD000014B184701207047D9EA000813B502AB71
:10ECE00003E90300019CA3699B68986983699847BD
:10ECF000044B01462046984700234FF0FF30A365A0
:10ED000002B010BD2D85000813B502AB03E9030066
:10ED1000019CA3699A6899699069426990470028A3
:10ED200014BF4FF0774300234FF0FF30A36502B0CC
:10ED300010BD000013B502AB03E90300019CA369F9
:10ED40009B689869C36A9847044B014620469847D8
:10ED500000234FF0FF30A36502B010BD2D850008E1
:10ED600013B502AB03E90300019CA3699B68986992
:10ED7000436A9847044B01462046984700234FF0CA
:10ED8000FF30A36502B010BD2D85000813B502AB9E
:10ED900003E90300019CA3699B689869036A98478B
:10EDA000044B01462046984700234FF0FF30A365EF
:10EDB00002B010BD2D85000813B502AB03E90300B6
:10EDC000019CA3699B689869836A9847044B014634
:10EDD0002046984700234FF0FF30A36502B010BDD6
:10EDE0002D85000813B502AB03E90300019CA3695C
:10EDF0009A6899699069C2699047054B0146204617
:10EE0000984700234FF0FF30A36502B010BD00BF4C
:10EE10009D85000813B502AB03E90300019CA369BB
:10EE20009A689969906982689047002814BF4FF0EA
:10EE30007F4300234FF0FF30A36502B010BD13B530
:10EE400002AB03E90300019CA3699A689969906980
:10EE5000C2689047002814BF4FF07F4300234FF053
:10EE6000FF30A36502B010BD30B58B699A6885B0DC
:10EE70008DE8030090690D460469996903AAA047CB
:10EE8000044640B90399054B284698474FF0FF3098
:10EE9000AC6505B030BD4FF07F44F7E72D85000825
:10EEA00013B502AB03E90300019CA3699B68986951
:10EEB000036A9847044B01462046984700234FF0C9
:10EEC000FF30A36502B010BD2D85000813B502AB5D
:10EED00003E90300019CA3699B68986983699847CB
:10EEE000044B01462046984700234FF0FF30A365AE
:10EEF00002B010BD2D85000813B502AB03E9030075
:10EF0000019CA3699B68986943699847044B014633
:10EF10002046984700234FF0FF30A36502B010BD94
:10EF20002D85000813B502AB03E90300019CA3691A
:10EF30009B689869C3699847044B014620469847E7
:10EF400000234FF0FF30A36502B010BD2D850008EF
:10EF500013B502AB03E90300019CA3699A689969A0
:10EF6000906982689047002814BF4FF07F430023C8
:10EF70004FF0FF30A36502B010BD13B502AB03E93B
:10EF80000300019CA3699A6899699069C2689047D7
:10EF9000002814BF4FF07F4300234FF0FF30A365DC
:10EFA00002B010BD37B502AB03E90300019CA369B1
:10EFB0009A68996990699A6A0569A847002814BFF8
:10EFC0004FF07F4300234FF0FF30A36503B030BD07
:10EFD0002DE9F04F99B012AB83E80300139DAA69A5
:10EFE000936D0B93936F91680C93D2F888300D93C7
:10EFF000D2F898308E690E9392F8A8301193D2F817
:10F00000C83092F8288092F8389092F848A092F888
:10F0100068B0D2F8B8700F93B468D2F8D83092695B
:10F0200010933046A0470446002843D1109B089314
:10F030000F9B0793119B0697003318BF012305937D
:10F040000E9B04930D9B03930C9B02931BF10003F7
:10F0500018BF012301930B9B00931AF1000318BF03
:10F06000012319F1000218BF012218F1000118BF95
:10F07000012137693046B84790B9A9691696072229
:10F080000123CDE91423E03102460B4B14A8984725
:10F09000041E09DB01212846084B9847002403E0A1
:10F0A00021462846054B98474FF0FF30AC6519B014
:10F0B000BDE8F08F0021EEE7F95202089D850008B7
:10F0C00013B5064B1B6801461C6901AA1846A047E8
:10F0D0000198431E5842584102B010BD243400200C
:10F0E0002DE9F04F234D244C85B092469B46814636
:10F0F0000F46A84742F210720023A047CDE9000155
:10F10000A8470A220023A047002680465E452CDA45
:10F110005FFA89F0194B9847B8420CD0A8470023F2
:10F120000A22A047B7FA87F7A0EB08034AF826306F
:10F130007F09013680460E9B002BE7DBA84742F291
:10F1400010720023A047DDE90023821A61EB03035C
:10F15000CDE902230E9B1946DA1713460A46DDE96C
:10F1600002018B4208BF8242D0D2304605B0BDE8D2
:10F17000F08F00BF910F0208F5FC0208C1F00008F3
:10F180002DE9F3470AAC94E8B002884602A901E9E8
:10F190000C007B1C064623DB002C21DB002D1FDB33
:10F1A000019A631993421BD8DFF858A0DAF80030AF
:10F1B00023B9114B9847CAF80000C8B1F0B20F4B01
:10F1C0009847009A88F8000002EB84020C4C0A97DA
:10F1D00001462B463046A44602B0BDE8F0476047E2
:10F1E0004FF029430020C9F8003002B0BDE8F08795
:10F1F0004FF07F43F6E700BF0D5F0008C1F0000845
:10F20000E1F000082434002070B592B004AB83E82C
:10F210000300059C2B4B002508AA2946204607958C
:10F220009847A842079046DB09AB01220FA9204668
:10F23000254EB047A84207903DDB0D950E950DADCC
:10F240002A4602212046214B98470028079032DBAE
:10F250000AAA032120461E4EB047002807902ADB49
:10F260000BAA04212046B0470028079023DB0CAAF4
:10F2700005212046B047002807901CDB07AB03930D
:10F280000C9B02930B9B01930A9B009395E80C0047
:10F29000099908980F4DA847079B002B01460ADBE8
:10F2A00020460D4B984701220FA920460B4B98474B
:10F2B00000EAE0700790079BA3654FF0FF3012B0A3
:10F2C00070BD00BF3F7200087D740008F97200082D
:10F2D0006D72000881F1000841740008C5740008CF
:10F2E0002DE9F04F89B08146149C129FDDF84C80C7
:10F2F000159D8A46601C08A901E90C0059DB002F06
:10F3000057DBB8F1000F54DB079A07EB0803934271
:10F310004FD82B4E336823B92A4B984730600028CA
:10F320004BD0294E294DB04742F210720023A84716
:10F33000CDE9000102460B462046E117CDE9020166
:10F340005FFA89FBCDE904235846214B9847504585
:10F35000DDE9042317D0611CF4D0B04742F21072EB
:10F360000023A84702460B46DDE90001DDE902BCA7
:10F37000101A63EB01018C4508BF8345E0D20020E1
:10F3800009B0BDE8F08F631C05D00099521AA24263
:10F3900034BFA41A00241294069A0E4C434602EB82
:10F3A00087025FFA8AF14846A44609B0BDE8F04FEB
:10F3B00060474FF029432B60E1E74FF07F43FAE7C6
:10F3C000243400200D5F0008910F0208F5FC0208AC
:10F3D000C1F00008E1F00008F0B58FB004AB83E89D
:10F3E0000300059C284B002508AA294620460795BE
:10F3F0009847A842079040DB0DF11B0201212046EF
:10F40000224B9847A842079037DB0CAE32460221C8
:10F4100020461F4B0C950D959847A84207902CDB72
:10F4200009AA032120461B4FB847A842079024DBB6
:10F430000AAA04212046B847A84207901DDB0BAA60
:10F4400005212046B847A842079016DB07AB039377
:10F450000B9B02930A9B0193099B009396E80C0077
:10F460009DF91B1008980C4EB047079BAB42014614
:10F4700003DB2046094B98470795079BA3654FF090
:10F48000FF300FB0F0BD00BF3F7200084D720008A2
:10F49000F97200086D720008E1F20008417400087A
:10F4A00038B5064B064D0446984700230A22A84764
:10F4B0002368C01A034B186038BD00BF910F0208C3
:10F4C000F5FC02082C34002010B590F83920134BBD
:10F4D000B2FA82F25209044680F83920186821698C
:10F4E00043699847A368E26801339342A36008D256
:10F4F000204650F8182B52F82310094BBDE8104055
:10F50000184794F8383033B120460023A36050F8F0
:10F51000183B1968F1E784F83A3010BD2834002010
:10F52000558E0008F0B51C4B1C4C8BB0984700283A
:10F5300030D01B4F1B4EB8470A220023B047CDE9FD
:10F540000001B8470A220023B047009D1649012355
:10F550006A468DF82030451B144B02A89847B847DF
:10F560000A220023B047124BCDE90001642102A812
:10F5700098474FF0FF33236023680133FCD02068A5
:10F580006438401B20602368002B01DA00232360CD
:10F590000BB0F0BD2060FBE7B17401082C340020F3
:10F5A000910F0208F5FC0208A1F40008E990000898
:10F5B000558E000873B5144B144D044668469847A1
:10F5C00020460321124B98470468C4B104F1180681
:10F5D0003046104B984710B130460F4B98470F4EAE
:10F5E000216930680222036A984730682169C3683C
:10F5F0000B4E9847206800B1B0472046B047684698
:10F60000A84702B070BD00BF097501084175010827
:10F61000EF740008879000087D8E000828340020D1
:10F62000854B000830B585B08DE8030000250846FD
:10F630000A4B03950C46984740B94FF0214303937A
:10F64000039BA3654FF0FF3005B030BD044B03A909
:10F650009847039B002BA8BF0395F1E7E1740008CE
:10F66000B5F5000870B50D4B0D46022106469847CA
:10F6700090F900402CB14FF019432B600024204634
:10F6800070BD074B03213046984703681BB94FF004
:10F690004E432B60F3E793F93A40F0E7F774000824
:10F6A000EF74000830B585B08DE8030000250846EA
:10F6B0000C4B03950C46984740B94FF021430393F8
:10F6C000039BA3654FF0FF3005B030BD03A9064B87
:10F6D0009847039B002B0146F2DB2046034B9847DB
:10F6E0000395EDE7E174000865F600082974000849
:10F6F0002DE9F74F0E46DFF840810121174681467C
:10F70000C047424B056840209847044640B9404BEB
:10F7100098474FF07A433B60204603B0BDE8F08F36
:10F72000DFF818A1DAF80030D346002B3BD1394B73
:10F730009847CAF80000002835D14FF07F433B605E
:10F74000EBE7354B354F68469847B8478046B84792
:10F75000B0EB0808B8478146DBF80000216943692F
:10F76000324698472E4B0A2000219847B847643804
:10F77000A0EB0900B0EB080858BF45464FF00A0857
:10F7800095FBF8F308FB1352042ACCBF0135CAF8E5
:10F7900000306846234BC4BF95FBF8F5CAF800500B
:10F7A00098470120B9E7204BDFF894A09847DBF891
:10F7B0000000EDB22946036A012298470036DBF8C3
:10F7C000000018BF012629464369324698470127A1
:10F7D000256100252246154B1549256004F11800C6
:10F7E000E56084F830709847032184F83A50484621
:10F7F000C047104B04600221484698470570DAF86C
:10F80000003001339DD0384687E700BFE94B000840
:10F81000854B00080D5F000809750108910F02086B
:10F82000750F02084175010825F50008E9900008E8
:10F83000C9F40008F7740008EF74000828340020A9
:10F84000680A00207FB500258DE80300134B03955F
:10F8500008460C469847064640B94FF021430393AB
:10F86000039BA3654FF0FF3004B070BD0DF10B0298
:10F87000012120460A4B984700280390F0DB9DF9B0
:10F880000B10084B03AA30469847039B002B0146F8
:10F89000E6DB2046044B98470395E1E7E174000856
:10F8A0004D720008F1F6000829740008F7B5194BED
:10F8B000194D044668460F4616469847174B0221D5
:10F8C0002046984790F9003033B14FF01943336028
:10F8D0006846A84703B0F0BD20460321104B984767
:10F8E000046814B94FF04E43F1E704F118063046AE
:10F8F0000C4B984710B130460B4B9847002384F8C7
:10F900003A300A4B216918683A1C436918BF012232
:10F910009847DDE70975010841750108F77400088B
:10F92000EF740008879000087D8E000828340020BE
:10F930007FB500258DE80300114B039508460C4662
:10F940009847064640B94FF021430393039BA365B4
:10F950004FF0FF3004B070BD0DF10B0201212046C5
:10F96000084B984700280390F0DB074B9DF90B10DC
:10F9700003AA30469847039B002BA8BF0395E5E7F1
:10F98000E17400084D720008ADF800082DE9FF474A
:10F9900004468DE80C0002A83D4BDDF830900D9F29
:10F9A0000F9E88469847022120463A4B984790F987
:10F9B000005055B14FF019433360002502A8364B73
:10F9C0009847284604B0BDE8F087B9F1000F5CDB2A
:10F9D000002F5ADB019B09EB07029A4255D82046BB
:10F9E00003212E4B984704681CB94FF04E433360F7
:10F9F000E4E704F118063046294B984710B1304629
:10FA0000284B9847002384F83A30002F3BD02068D9
:10FA100008B1254B98474FEA870A5046234B984731
:10FA200020600028CAD00099214B524601EB890181
:10FA3000984700239DF93820A360E76084F83820B8
:10FA40000221E2689A4208D9226852F8230001286C
:10FA500098BF42F823100133F3E7164B84F839803E
:10FA600018682169436918F1000218BF01229847FC
:10FA70002368A268304653F822100F4B012598479F
:10FA800084F83A509AE7012598E74FF02543AEE70E
:10FA900009750108F774000841750108EF74000842
:10FAA000879000087D8E0008854B0008E94B000810
:10FAB000CF01030828340020558E00082DE9F043BB
:10FAC0008DB004AB83E80300059C2B4B002520463A
:10FAD00007959847074648B94FF021430793079B7E
:10FAE000A3654FF0FF300DB0BDE8F0830DF11A02B1
:10FAF00001212046DFF89080C04700280790EEDB08
:10FB00000AAE3246022120461C4B0A950B959847B7
:10FB100000280790E3DB08AA03212046DFF86C9059
:10FB2000C84700280790DADB09AA04212046C84705
:10FB300000280790D3DB0DF11B0205212046C047AA
:10FB400000280790CBDB07AB03939DF91B30029392
:10FB5000099B0193089B009396E80C009DF91A10ED
:10FB6000074E3846B047079B002B0146B7DB2046BF
:10FB7000044B98470795B2E7E1740008F972000852
:10FB80008DF90008297400084D7200086D72000894
:10FB90002DE9F04F89B00F46129E169CDDF85C806F
:10FBA00004A981E80C00002E9DF954300293C0F2A4
:10FBB000B980139B002BC0F2B580F218059B9A42C6
:10FBC00000F2B0800321594B9847056825B94FF0E2
:10FBD0004E43C8F800307CE0554B06A805F11808E4
:10FBE00098474046534B984710B14046524B984770
:10FBF000002385F83A3006A8504B9847049B03EB46
:10FC0000860A44B14E4A4F4BB3FBF4F31468A34247
:10FC100094BF01341C1B029B33B14B4B984720B35C
:10FC20004A4B984701230193494E296930683A1C91
:10FC3000436918BF012298474FF00008B146139B53
:10FC4000984538D007B194B95AF82800414B0021A3
:10FC50009847D9F8000029694369B7FA87F2520931
:10FC600057B208F101089847E9E70190DCE7344B07
:10FC70005AF828201B684FF0000B2344B2FBF3F323
:10FC80000393039B9B45E4DAD9F800002969436993
:10FC900001229847204600212E4B9847D9F80000B2
:10FCA000296943690022984720460021294B98473B
:10FCB0000BF1020BE5E7149B2BB107B164B9149863
:10FCC000244B00219847029B1BB1019B0BB1224B97
:10FCD000984709B0BDE8F08F194BDFF878901F689E
:10FCE000149B4FF000082744B3FBF7F7B84512DA2E
:10FCF0003068296943690122984720460021C84796
:10FD00003068296943690022984720460021C84786
:10FD100008F10208EAE70E4B2969186801224369D5
:10FD20009847D0E74FF0254353E700BFEF74000832
:10FD300009750108879000087D8E0008417501084B
:10FD4000680A002020A10700B1740108C9740108E5
:10FD500028340020750F0208DD7401082DE9F043F6
:10FD600091B006AB83E80300079C334B0025204687
:10FD700009959847074648B94FF021430993099BD5
:10FD8000A3654FF0FF3011B0BDE8F0830DF1220202
:10FD900001212046DFF8AC90C84700280990EEDB2F
:10FDA0000EAE324602212046244B0E950F95984701
:10FDB00000280990E3DB0AAA03212046DFF88880A7
:10FDC000C04700280990DADB0BAA04212046C0476F
:10FDD00000280990D3DB0CAA05212046DFF86C80AF
:10FDE000C04700280990CADB0DF1230206212046F6
:10FDF000C84700280990C2DB0DAA07212046C0474A
:10FE000000280990BBDB09AB05930D9B04939DF97A
:10FE1000233003930C9B02930B9B01930A9B00934B
:10FE200096E80C009DF92210054E3846B047099B14
:10FE3000002BA8BF0995A2E7E1740008F972000839
:10FE400091FB00084D7200086D7200083F720008B7
:10FE500013B5064B1B6801461C6901AA1846A0474A
:10FE60000198431E5842584102B010BD3034002062
:10FE70002DE9F04F364B374D85B00E46062104462E
:10FE80009847032107782046A847334BD0F800B0A5
:10FE9000042120469847092190F900902046A84760
:10FEA0000221D0F800A020462C4CA8472368D0F8A7
:10FEB00000802546B3B92A4B9847206090B94FF08F
:10FEC0007F433360002000213EE0B8F1FF3F29D09E
:10FED000DDE90023A242AB4124DA4FF0FF304FF0BE
:10FEE000FF3131E028681F4C036A1F4E012239465A
:10FEF000984758461D4BDFF878B0C1179847A04780
:10FF00000A220023B04710EB080241EBE873CDE969
:10FF10000023A047CDE9020128685246036A39460A
:10FF20009847A246D0470A220023B04704463846E5
:10FF30000D46D8474845C8D00A220023DDE9020112
:10FF4000B047201A65EB010105B0BDE8F08F00BF96
:10FF5000E7740008FF740008F774000830340020CC
:10FF60000D5F0008910F0208F5FC0208590F020806
:10FF700051FE000830B585B08DE803000025084625
:10FF80000D4B03950C46984740B94FF0214303931E
:10FF9000039BA3654FF0FF3005B030BD074B03A9AD
:10FFA00098470B46039900290246F1DB2046044995
:10FFB00088470395ECE700BFE174000871FE000874
:10FFC000597400082DE9F04F87B0DFF8C0A1049103
:10FFD000062104461646D047654F0578DFF8B091F4
:10FFE00003212046B8470421D0F800B02046C84776
:10FFF000072190F900802046D047052190F800A005
:020000040801F1
:100000002046C847092190F9003005932046B8479B
:100010000221D0F800902046B84703680093554F5E
:10002000554B98473B68CDE902013C46002B71D106
:10003000524B9847386000286CD14FF07F433360B3
:100040000020002137E04C4B98470A220023B0479C
:1000500004460D46009B4A4FDFF81CB11946DA17DB
:10006000CDE9001200230A22DDE90201B047DDE9F3
:10007000002312184B41CDE90223B9465046B84738
:10008000059B9842804619D0DDE90023013308BF63
:10009000B2F1FF3FF2D0D847DFF8EC800A2200230C
:1000A000C047DDE902238B4208BF8242E6D24FF00F
:1000B000FF304FF0FF3107B0BDE8F08F049B2E4FAB
:1000C00073B9B847BB4604460D465046C8478045FD
:1000D0000ED0204629460A220023B04704460D468A
:1000E000B8470A220023B047001B61EB0501E2E795
:1000F000DDE90023013308BFB2F1FF3FE5D0D84767
:100100000A220023B047DDE902238B4208BF824266
:10011000DBD2CCE720681B4F036A012229469847AF
:10012000B8FA88F620687609324643692946984726
:100130000A200021B847206818F1000218BF0122E8
:100140004369294698475846C117B8472068324640
:1001500043690D4E2946984720684A46036A51462E
:100160009847049B002B7FF46EAF0024002571E7B5
:10017000FF74000830340020910F02080D5F000862
:1001800051FE0008590F0208F5FC0208E774000848
:10019000F77400087FB500258DE80300144B039524
:1001A00008460C469847064640B94FF02143039352
:1001B000039BA3654FF0FF3004B070BD0DF10B023F
:1001C000012120460B4B984700280390F0DB03AA3F
:1001D000094B9DF90B10304698470B4603990029AF
:1001E0000246E5DB2046054988470395E0E700BF66
:1001F000E17400084D720008C5FF0008597400083A
:1002000070B506210F4C0546A04707210678284601
:10021000A0470D4C057820680222036A31469847B2
:1002200020683146C3689847AE420AD02068294604
:10023000036A0222984720682946C368BDE87040D7
:10024000184770BDE77400083034002030B585B021
:100250008DE80300002508460A4B03950C46984795
:1002600040B94FF021430393039BA3654FF0FF3048
:1002700005B030BD044B03A99847039B002BA8BFD2
:100280000395F1E7E17400080102010813B502AB20
:1002900003E90300019CA3699B689869036B984775
:1002A000044B01462046984700234FF0FF30A365DA
:1002B00002B010BD2D85000810B502F1FF3E86B0DA
:1002C000DEF1000242EB0E02002304680493029266
:1002D00003930A46CB17CDE90023044943686268BB
:1002E0000348044CA04706B010BD00BF67210308B7
:1002F000042B0020DD88000830B58B699B6893F9DA
:10030000284085B08DE803000D46B4B9986F996B0D
:10031000426A904742F2107280FB022304A961E90D
:1003200002232846064B98472B6C102203F8102C0A
:100330004FF0FF30AC6505B030BD4FF01944F7E722
:1003400045850008F7B502AB03E90300019CA169EC
:100350008D6895F92830ABB942F210720023886994
:100360000B4FC969AE6FB847B36AA96B02463046F6
:10037000984750B92046074B9847A0654FF0FF308B
:1003800003B0F0BD4FF01940F7E74FF07D40F4E7C0
:1003900055FC0208258700087FB58B699B6893F997
:1003A00028408DE803000D466CB9986F996B06697B
:1003B00003AAB0470399054B284698474FF0FF30F2
:1003C000AC6504B070BD4FF01944F7E72D85000807
:1003D00073B502AB03E90300019DAA69936893F921
:1003E00028408CB991699965996C986F012906D15B
:1003F00092694669996B003218BF0122B0474FF0ED
:10040000FF30AC6502B070BD4FF01944F7E7000053
:10041000F7B502AB03E90300019DAB699E689F69D4
:10042000B06F394683689847044648B9B7630121DD
:100430002846054B98474FF0FF30AC6503B0F0BD40
:100440004FF05644F7E700BF9D85000813B502AB97
:1004500003E90300019CA3699B68986F996BC268CC
:10046000904700234FF0FF30A36502B010BD00009D
:100470002DE9F34102AB03E90300DDF80480D8F86D
:1004800018309F689B69BC6FBD6B032B2BD8DFE8CE
:1004900003F014022427236A0122294620469847A4
:1004A0000646002E14BF4FF0564300234FF0FF3096
:1004B000C8F8583002B0BDE8F081236A002229460E
:1004C00020469847BA6EE36A002A0646074A29463C
:1004D00008BF002220469847E3E7236A0222EEE79E
:1004E000236A0322EBE74FF07D43DFE7B9020108FF
:1004F00070B5074D044628682146036A01229847D3
:100500002868214643690122BDE87040184700BFB2
:1005100034340020074B427B1B6810B41C6A002A4D
:10052000184618BF0222234608BF00225DF8044B7C
:10053000184700BF3434002013B5074B0C469847CA
:10054000064B186801AA0369214698470198431E83
:100550005842584102B010BD15050108343400203E
:10056000F8B5104C104E2068104D0168104FB04780
:1005700001200021A84720684168B04728B9013F01
:1005800003D001200021A847F5E720680168B047A3
:10059000002106460120A84723685868054B984764
:1005A0003046F8BD3834002039050108750F0208BF
:1005B00041420F00F10401082DE9F0418046164C3C
:1005C000164EF0B120680168B04701200021144D9B
:1005D000144FA84720684168B04708B9013F15D1BA
:1005E000B8F1000F03D020680168B04790B1002136
:1005F0000120A847236858680B4B98470120BDE8A5
:10060000F08123681868084B9847DEE70120002135
:10061000A847DFE7BDE8F08138340020390501083C
:10062000750F020841420F00F10401082DE9F04165
:10063000164E174C3378DFF86880A3B9206801683C
:10064000C047054660B12368124F1868B8470120BB
:100650000021114B984723685868B847012333702D
:100660002846BDE8F08120680B4D01680B4FC0475C
:1006700001200021A84720684168C0470028DDD13B
:10068000013FDBD001200021A847F4E73C340020E3
:1006900038340020F1040108750F020841420F00B0
:1006A000390501082DE9F041114C124D2368124F14
:1006B0001868124B124E984701200021A847B846EF
:1006C00020684168B84708B9013E0DD1206801682B
:1006D000C047044628B101200021A847094B002249
:1006E0001A702046BDE8F08101200021A847E7E705
:1006F00038340020750F020839050108F10401089B
:1007000041420F003C340020F8B50E46144608B1B3
:10071000084B9847084F0825E009B8476400013D99
:10072000E4B2F9D1054B984704460EB1044B984703
:100730002046F8BD2D060108B9050108610501082C
:10074000A50601082DE9F041DFF8348007460E4682
:10075000082500246400E4B2C04708B144F0010455
:10076000013DF7D187F00100034B98470EB1034BD1
:1007700098472046BDE8F081B9050108A5060108A3
:1007800061050108064A38B50021064D1170064C76
:1007900001682860A04728684168A047012038BD4B
:1007A0003C34002038340020150501082DE9F84FAD
:1007B00098460C9B0A9D00241C600B9B16461C60EF
:1007C0002E4B89469847002E43D02D4B2D4F1B684A
:1007D0001A7B520002F0FE0221460120B847002891
:1007E00042D1CA46044606F1FF3BAAEB09029345F3
:1007F00008D900211AF8012B0846B8470028F4D17F
:100800000134F2E7B5FA85F119F80B204909002007
:10081000B84700B901340B9B1C601DB3184B1B6813
:100820001A7B184B520042F00102D2B20021012083
:10083000984708BBDFF850A0474605F1FF39A7EB02
:1008400008034B4507D200210120D04707F8010BD0
:10085000F5E73446E1E701210020D0470C9B08F87A
:1008600009001D60294600E0214670190C44231A36
:1008700058425841BDE8F88F0021F6E78507010886
:100880003834002009070108450701082DE9F04F19
:100890008FB006AB83E80300DFF8C090DDF81C8062
:1008A000D9F80020D8F818400023A168D4F818A07F
:1008B00094F828B094F93870A56CA66D0893099344
:1008C000002A40D1224A059190470599C9F80000B5
:1008D000002838D14FF07F432CE02A69002E30D019
:1008E00033690B9164210C9109A90037029108A981
:1008F00018BF01270191009305F1180106F11803B3
:100900000AA8144D8DF83570CDF828A08DF834B0B4
:10091000A847A36E089A9A6008260127C3E90067D2
:10092000A36F099A9A60C3E9006701460A4B4046E3
:10093000984700234FF0FF30C8F858300FB0BDE89B
:10094000F08F3346CDE7002DC7D12A46C6E700BF5A
:100950000D5F0008AD070108217400083434002041
:1009600013B502AB03E90300019CA3699B68986976
:1009700083689847002814BF4FF07F4300234FF04F
:10098000FF30A36502B010BD13B502AB03E903004D
:10099000019CA3699B689869C3689847002814BFA5
:1009A0004FF07F4300234FF0FF30A36502B010BD2E
:1009B0002DE9F0418A6988B093688DE803000C4600
:1009C0000021029193F828109D69002933D196697E
:1009D000002E33D09B6B99699A6A3369029328463B
:1009E0002B6998476F69284603AB02AA06F11801E4
:1009F000B847054628BBA169029BDFF84C800693E7
:100A0000024607260127203104A8CDE90467C04724
:100A100000280ADBA169039B06932A46303104A80B
:100A2000CDE90467C04700EAE070A0654FF0FF30F1
:100A300008B0BDE8F0814FF01940F6E74FF056409E
:100A4000F3E74FF07F40F0E7F95202082DE9F0415B
:100A50008A6988B093688DE803000C4600210291F2
:100A600093F828109D69002933D19669002E33D060
:100A70009B6B99699A6A3369029328462B69984758
:100A8000AF69284603AB02AA06F11801B84705462C
:100A900028BBA169029BDFF84C800693024607261B
:100AA0000127203104A8CDE90467C04700280ADBEC
:100AB000A169039B06932A46303104A8CDE9046757
:100AC000C04700EAE070A0654FF0FF3008B0BDE815
:100AD000F0814FF01940F6E74FF05640F3E74FF042
:100AE0007F40F0E7F95202082DE9F0418CB002ABEB
:100AF00083E80300039CA269936800210591069195
:100B000093F828109D69002940D19669976A002EB4
:100B10003FD0002F3DD09B6B99699A6A336905934A
:100B20003B69069328462B69984707AB019306ABB0
:100B30000093D5F81C80284607F1180305AA06F192
:100B40001801C047054638BB069A059BA169DFF826
:100B500050801344072602460127203108A8CDE91A
:100B600008670A93C04700280ADBA169079B0A931C
:100B70002A46303108A8CDE90867C04700EAE0708E
:100B8000A0654FF0FF300CB0BDE8F0814FF0194088
:100B9000F6E74FF05640F3E74FF07F40F0E700BF35
:100BA000F952020882B003788DF8003043788DF84E
:100BB000013083788DF8023002ABC27803F8052D3E
:100BC000021D0830904204D012F8011B03F8011FE7
:100BD000F8E79DED000B02B07047000013B502ABC3
:100BE00003E90300019CA3699B689869436A9847DD
:100BF0002046044B984700234FF0FF30A36502B016
:100C000010BD00BFD584000813B502AB03E9030093
:100C1000019CA3699B689869036A98472046044B26
:100C2000984700234FF0FF30A36502B010BD00BF0E
:100C3000D584000813B502AB03E90300019CA36946
:100C40009B689869C36A9847044B014620469847B9
:100C500000234FF0FF30A36502B010BD2D850008C2
:100C600013B502AB03E90300019CA3699A68996973
:100C700090694269904700234FF0FF30A36502B0AE
:100C800010BD13B502AB03E90300019CA3699A6888
:100C9000996990690269904700234FF0FF30A3657E
:100CA00002B010BD13B502AB03E90300019CA369B8
:100CB0009A68996990698268904700234FF0FF30E5
:100CC000A36502B010BD13B502AB03E90300019C9C
:100CD000A3699A6899699069C268904700234FF0A8
:100CE000FF30A36502B010BD30B585B08DE80300BC
:100CF0008869836818309D69094B0C46984704A998
:100D000021ED020BEB692846984720469DED020B2A
:100D1000044B984700234FF0FF30A36505B030BD6A
:100D2000A50B0108D584000873B502AB03E90300E5
:100D3000019DAC69A36804F128009E69084B98479F
:100D400094F93820B369A169003218BF01223046F6
:100D5000984700234FF0FF30AB6502B070BD00BF75
:100D6000A50B010830B5002387B0002400250268D8
:100D70000493CDE902458DE80A00044C43685268AB
:100D800003490448A04707B030BD00BFDD88000814
:100D9000A1210308042B002030B5002387B00024D4
:100DA000002502680493CDE902458DE80A00044C51
:100DB0004368526803490448A04707B030BD00BFEC
:100DC000DD880008D9210308042B0020026C436948
:100DD0009A4210B5044602D80120034B9847206C74
:100DE0001038206410BD00BF154C00082DE9FF47E6
:100DF00004AB03E90300039DA86983689C692CB3D5
:100E0000866CD0F858A08769D0F82890D0F8388040
:100E1000A368204698478DE8400442464B46394631
:100E200026692046B047236A0A4920469847636AE4
:100E3000094920469847A36A084920469847002355
:100E40004FF0FF30AB6504B0BDE8F0874FF077435B
:100E5000F6E700BF650D0108990D0108ED5C00087B
:100E600013B502AB03E90300019CA3699B68986971
:100E7000C368984700234FF0FF30A36502B010BD50
:100E800013B502AB03E90300019CA3699B68986951
:100E90004369984700234FF0FF30A36502B010BDAF
:100EA0002DE9F04788B002AB83E80300039CA169F9
:100EB0008B68D1F83880D3F81890D1F818A08D6AD3
:100EC00001238DF8173006AA40312046214B984760
:100ED00000282CDBA36C012B05D11F4B00212046E1
:100EE00098470223A36463699F693D4418355544BC
:100EF000A8EB0706DFF868A0DFF868809DF81730D8
:100F0000E3B1DEB1D9F81830079607AA294648465A
:100F10009847079B8BB96369069A9F610DF1170388
:100F20000093216902235046C0470028E6DAA065F5
:100F30004FF0FF3008B0BDE8F0871F44074D204652
:100F4000A8472046A84720463946034B984700202B
:100F5000EDE700BF158600082D850008CD0D0108BE
:100F6000002E0020E1CB00082DE9F04788B002AB4D
:100F700083E80300039CA1698B68D1F83880D3F81B
:100F80001890D1F818A08D6A01238DF8173006AAA1
:100F900040312046224B984700282CDBA36C012BC4
:100FA00005D1204B0021204698470223A3646369A2
:100FB0009F693D4418355544A8EB0706DFF86CA03F
:100FC000DFF86C809DF81730FBB1F6B1D9F81C3012
:100FD000079607AA294648469847079B8BB9636935
:100FE000069A9F610DF11703009321690223404681
:100FF000D0470028E6DAA0654FF0FF3008B0BDE822
:10100000F0871D441F44F61ADCE7074D2046A84729
:101010002046A84720463946024B98470020EAE779
:10102000158600082D850008CD0D0108E1CB0008CC
:10103000002E002013B502AB03E90300019CA36955
:101040009B68986983689847002814BF4FF07F43D6
:1010500000234FF0FF30A36502B010BD13B502AB03
:1010600003E90300019CA3699B689869C3689847DA
:10107000002814BF4FF07F4300234FF0FF30A365DB
:1010800002B010BD2DE9F04186B002AB83E8030049
:10109000DDF80C80D8F818209368002104910591A0
:1010A00093F838109C6931BB9569966A35B32EB3B5
:1010B000986A8169826B836A876C286904903069B9
:1010C0000097059027692046B84705AB0093E7696C
:1010D00006F1180304AA05F118012046B8470028B4
:1010E00014BF4FF07F4300234FF0FF30C8F8583053
:1010F00006B0BDE8F0814FF01943F5E74FF05643D5
:10110000F2E72DE9F04186B002AB83E80300DDF899
:101110000C80D8F81820936800210491059193F869
:1011200038109C6931BB9569966A35B32EB3986ABD
:101130008169826B836A876C2869049030690097A3
:10114000059027692046B84705AB0093276A06F14A
:10115000180304AA05F118012046B847002814BF57
:101160004FF07F4300234FF0FF30C8F8583006B0EF
:10117000BDE8F0814FF01943F5E74FF05643F2E731
:101180002DE9F04186B002AB83E80300DDF80C8066
:10119000D8F8182093680021059193F838109C69BD
:1011A00001BB95690DB3986A06AE8169826B836A4B
:1011B000876C286946F8040D009727692046B847D0
:1011C000A369324605F1180120469847002814BF4C
:1011D0004FF07F4300234FF0FF30C8F8583006B07F
:1011E000BDE8F0814FF01943F5E74FF05643F2E7C1
:1011F0002DE9F04186B002AB83E80300DDF80C80F6
:10120000D8F8182093680021059193F838109C694C
:1012100001BB95690DB3986A06AE8169826B836ADA
:10122000876C286946F8040D009727692046B8475F
:101230006369324605F1180120469847002814BF1B
:101240004FF07F4300234FF0FF30C8F8583006B00E
:10125000BDE8F0814FF01943F5E74FF05643F2E750
:10126000F0B58B699C689D698FB08DE803000E46D0
:10127000002C34D0AB6A28469847A062EB6A284617
:101280009847A0636B6A284698470EAAA0610A2374
:1012900004AF42F82C3D39462B6B28469847002571
:1012A00012220123C4E91023A5640E4A03990E4BB0
:1012B00004F14000984700280CDBA26C039814321C
:1012C0002B46834205D057F8231042F8041F013300
:1012D000F7E70020B0654FF0FF300FB0F0BD4FF0E2
:1012E0002140F7E7B03100205961020838B50D46BA
:1012F00090B1846884B12378372B05D120460A4BFE
:10130000984700280EDBA468A36913B11A78202A35
:1013100005D04FF07D4038BD4FF0214038BD183327
:101320002B60002038BD00BFED5E02088069014BD4
:10133000184700BFED12010810B50C468AB08DE8C1
:1013400003000D4B03A92046984700280EDBA36934
:101350000398198B094B04AA98479DF8101009B1FE
:10136000BDF81A10064B204698470020A0654FF0A4
:10137000FF300AB010BD00BF2D130108E588020838
:101380002D8500081FB50C468DE80300084B03A906
:1013900020469847002805DB039B20461988054B0B
:1013A00098470020A0654FF0FF3004B010BD00BF8B
:1013B0002D1301082D8500081FB50C468DE803008C
:1013C000084B03A920469847002806DB039B2046CC
:1013D000B3F90C10044B98470020A0654FF0FF3084
:1013E00004B010BD2D1301082D8500081FB50C4653
:1013F0008DE80300084B03A920469847002806DB28
:10140000039B2046B3F90E10044B98470020A065BB
:101410004FF0FF3004B010BD2D1301082D850008DA
:101420001FB50C468DE80300084B03A920469847DA
:10143000002806DB039B2046B3F90410044B9847B1
:101440000020A0654FF0FF3004B010BD2D1301083F
:101450002D8500081FB50C468DE80300084B03A935
:1014600020469847002806DB039B2046B3F9061068
:10147000044B98470020A0654FF0FF3004B010BD2A
:101480002D1301082D8500081FB50C468DE80300BB
:10149000084B03A920469847002806DB039B2046FB
:1014A000B3F90810044B98470020A0654FF0FF30B7
:1014B00004B010BD2D1301082D8500081FB50C4682
:1014C0008DE80300084B03A920469847002806DB57
:1014D000039B2046B3F90A10044B98470020A065EF
:1014E0004FF0FF3004B010BD2D1301082D8500080A
:1014F0002DE9F04391B004AB83E80300DDF81480DC
:101500001F4B07A94046984700282FDBD8F81850F2
:101510002B7C122B31D1AB69002B2ED0996800297E
:101520002BD000240394029401940094AB6C154ECC
:101530000798DFF854904FF0FF32B04701270A9028
:101540000726224605F1200108A8CDE90867C8470B
:1015500000280BDB079B22461B880E9305F1300108
:101560000CA8CDE90C67C84700EAE070C8F858003D
:101570004FF0FF3011B0BDE8F0834FF02140F5E7A8
:101580002D130108A18A0208F95202082DE9F0433F
:101590009BB00AAB83E80300DDF82C80294B0CA933
:1015A00040469847002840DBD8F81840237C122B8F
:1015B00042D1A36903B19B680D93002B3ED0A36C6D
:1015C0001093A36D119300250C9B08930795D4F8F5
:1015D00088300693A36F0593A36E04930FAB00931B
:1015E0000395029501950EAB11AA10A90DA8164EF0
:1015F000B047002819DB0E9BDFF8509014930726A4
:1016000001272A4604F1200112A8CDE91267C84734
:1016100000280ADB0F9B18932A4604F1300116A814
:10162000CDE91667C84700EAE070C8F858004FF0E7
:10163000FF301BB0BDE8F0830023BDE74FF0214031
:10164000F3E700BF2D130108692B0108F9520208C6
:10165000F7B502AB03E90300019DAB69AA6C9E6874
:101660002AB90122AA64AA6A42F02002AA629C69ED
:1016700054B393F82870637843F0080363702378B9
:10168000152B02D00120164B9847237D032B02D047
:101690000120134B9847637D012B02D00120104B92
:1016A00098473B4622690F4F04F1180106F11000DC
:1016B000B84700280ADBB3691B78202B02D13046DB
:1016C000094B9847002001E04FF02140637823F058
:1016D00008036370A8654FF0FF3003B0F0BD00BF92
:1016E000154C0008B9260108A96B020870B50C4614
:1016F00086B08DE80300A36C89698D682BB901233E
:10170000A364A36A43F02003A3628A6A0E4E896928
:10171000002303A8B04778B103A905F110000B4BD3
:10172000984700280ADBAB691B78202B02D128469A
:10173000074B9847002001E04FF07F40A0654FF035
:10174000FF3006B070BD00BF81260108892801085E
:10175000A96B020837B502AB03E90300019DAB6931
:101760009C68A06958B104F11000074B9847002805
:1017700005DB12220123C4E904230020A061A8652F
:101780004FF0FF3003B030BD19270108F0B58B6969
:101790009C688BB08DE803000D4634B3E3692046A6
:1017A000984707260127236A0490CDE9026720465F
:1017B0009847A9690890CDE906670022103102A870
:1017C0000C4EB047041E0BDBA9690022203106A88D
:1017D000B047041E04DB01212846074B984700242C
:1017E0004FF0FF30AC650BB0F0BD21462846024BF0
:1017F0009847F5E7F95202089D85000870B50E4636
:101800001546E8B18468DCB12378372B05D1204632
:101810000E4B9847002818DBA4680D4B294604F1AD
:1018200010009847002810DB2B681B89DA0700D5C9
:101830004EB913F0020F14BF4FF07D40002070BD71
:101840004FF0214070BD4FF07D4070BDED5E02084D
:10185000E52601088069014B184700BFFD17010804
:101860001FB50C468DE8030003AA00212046074B54
:101870009847002805DB039B20461968044B9847CE
:101880000020A0654FF0FF3004B010BD55180108CE
:101890002D8500081FB50C468DE8030003AA002122
:1018A0002046074B9847002805DB039B20465968D4
:1018B000044B98470020A0654FF0FF3004B010BDE6
:1018C000551801082D8500081FB50C468DE803004A
:1018D00003AA01212046064B9847002803DB039802
:1018E000044B98470020A0654FF0FF3004B010BDB6
:1018F00055180108112A010830B589B004AB83E8F6
:101900000300059C0C4B07AA00212046984700289D
:101910000DDBA36907999B6902938B8801930B8860
:10192000009300230548064D1A46A8470020A065ED
:101930004FF0FF3009B030BD55180108D42B0020FE
:10194000A146010830B587B002AB83E80300039DD0
:10195000134BAC6904AA012128469847002817DBDD
:1019600005A904F120000F4B9847002810DB237CC9
:10197000122B12D1A36983B1996871B1A36D019340
:10198000A36C0093A36B0498059A074CA047002012
:10199000A8654FF0FF3007B030BD4FF02140F7E7AA
:1019A00055180108ED120108412B0108F0B58FB060
:1019B00002AB83E80300039C214BA56904AA012123
:1019C00020469847002836DB05AA002105F13000A3
:1019D0001C4B984700282EDB0498059A904205D0AE
:1019E000A96E002902DBAB6F002B02DA4FF07D40BD
:1019F00021E0D5F828E0D5F818C0AE6DAF6CCDF871
:101A000018C073446144013B01390993A3EB0E03F1
:101A100008913344A1EB0C0139440D93B5F888309B
:101A20000C91009306A90AAB074DCDF81CE00A976C
:101A30000B96A8470020A0654FF0FF300FB0F0BD17
:101A400055180108FD170108B52A010830B591B0F5
:101A500004AB83E80300059C194B06AA012120462C
:101A60009847002826DBA36906989A6907929A6A24
:101A700008929A6F0992D3F888200A92D3F8982096
:101A80000B92D3F8A8200C92D3F8B8200D92D3F87B
:101A9000C8200E92B3F8D820ADF83C209A6E02927E
:101AA0009A6D01929A6C00929B6B064D09AA07A948
:101AB000A8470020A0654FF0FF3011B030BD00BF37
:101AC00055180108A12A010830B589B002AB83E896
:101AD0000300039C0D4B05AA0121204698470028CE
:101AE0000FDBA269059893690693936A0793936E37
:101AF0000193936D0093936C054D926B06A9A847D3
:101B00000020A0654FF0FF3009B030BD5518010826
:101B1000F12A010870B592B002AB83E80300039C80
:101B20002A4B04AA01212046984700283CDBA369E0
:101B30009A6905929A6A0692D3F898200B92D3F884
:101B4000A8200C92D3F8B8200D92D3F8C8200E929A
:101B5000D3F8D8200F92D3F8E8201092B3F8F820E9
:101B60009D6B986C996DADF844209A6E9E6F0795A9
:101B7000294402440139013A002E089009910A9241
:101B8000D3F888300CDC002B13DD5EB9019300968E
:101B900007AB0BAA05A904980D4DA847002003E048
:101BA000002BF3DA4FF07D40A0654FF0FF3012B00C
:101BB00070BD491B0131F5DB121A0132F2DB07ABB4
:101BC0000BAA05A90498034DA847E7E75518010893
:101BD000192B0108052B01082DE9F04389B004AB4E
:101BE00083E80300059D114BAA690021D2F81880F3
:101BF000D2F82890966B976C284607AA9847041E3F
